:020000040000FA
:1000000092EF01F01200FFFF10EF04F01200FFFF6B
:1000100000000901C80E926F66806650010B06E071
:100020000901925103E009019207F7D7120000007D
:100030000901C80E926F66846650040B06E0090140
:10004000925103E009019207F7D71200D9CFE6FFDA
:10005000E1CFD9FF3F0E6816676A666AFE0EDB5075
:100060006712FD0EDB506812678AE552E7CFD9FFB1
:100070001200D9CFE6FFE1CFD9FFFE0EDB506A6E4A
:1000800067AE02D0FF0E30D00F0E671408080CE0E8
:100090000F0E67140B0808E06850040B03E168506A
:1000A000010B1FE0000E20D00F0E6714080804E0BB
:1000B0000F0E67140B0818E10901C80E926F685003
:1000C000010B04E0925102E09207F9D76850040B4B
:1000D00001E0010E4B6E1F0E66144B10F7E166AC8B
:1000E00002D0FE0E01D0000EE552E7CFD9FF12007C
:1000F000D9CFE6FFE1CFD9FF0000FE0EDBCFE6FF50
:10010000B8DFE552006E005003E091DF005000D0F0
:10011000E552E7CFD9FF120000007ADF700EE66EDD
:10012000E7DFE552000901E028D0800EE66EE0DF4F
:10013000E552000901E021D0E66ADADFE552000964
:1001400001E01BD0400EE66ED3DFE552000901E06E
:1001500014D0016A1E0E015C0FE20150EA6A000F22
:10016000E96E060EEA22EF50E66EC2DFE5520009A4
:1001700001E003D0012AEED75ADF12000000016A25
:100180001E0E015C09E20150EA6A000FE96E060EDC
:10019000EA22EF68012AF4D712000000016A1E0E5D
:1001A000015C09E20150EA6A000FE96E060EEA22DC
:1001B000EF6A012AF4D712000000EFDFE66A080EAA
:1001C000E66E44DFE552E552090E696E21DF700EDE
:1001D000E66E8EDFE552000901E01CD0800EE66E6F
:1001E00087DFE552000901E015D0C80EE66E80DF1A
:1001F000E552000901E00ED0E66A7ADFE552000917
:1002000001E008D0E00EE66E73DFE552000901E080
:1002100001D00DDF12000000CFDF0601050E026FD6
:100220000601340E036F0601460E146F0601050E1B
:10023000176F0601040E186F0601640E196F060190
:10024000010E1A6F0601670E1B6F0601020E1C6F6E
:100250000601600E1D6F60DF1200000037D836D82F
:100260008D8A8D8C84848C80120009018E6B09012B
:100270008A07000E8B5B09018D5109018C5D04E03A
:1002800084948C908D9A8D9C8E2FFED709018D5170
:1002900009018C5D06E009018CB18C8009018CB3E9
:1002A00084848E2FFED78CC98DF9120000000900BE
:1002B000F5CF89F90900F5CF88F9090188510901BD
:1002C00086270901895109018723120000000901CD
:1002D000886B896B0901540E885D3D0E895905E2D2
:1002E0000901882B000E8923F5D7120000000901AF
:1002F000886B896B0901220E885D060E895905E21B
:100300000901882B000E8923F5D7120000008250C6
:10031000010B03E08250020B02E1010E02D0000E3D
:1003200000D01200C16A0F01DF0E256F0F01F70E1A
:10033000246F0F01E00E236F3A0EC06EEF0E896E30
:100340008A6A8B6A9E0E8C6E900E8D6E8E6A8F6A94
:10035000010E906E916AEF0E926E070E936E930EE1
:10036000946E600E956E030E966E7D0E976E060E61
:10037000986EFE0E996E9A688A8AC79EC698C78C38
:10038000F00EC616C680C68A240EAC6E190EAF6E6D
:10039000900EAB6EF29EA698636AFE0E626E010E20
:1003A000616E7F9E7F9C7F84550E7E6EAA0E7E6E50
:1003B0007F82F28E01DFB0DE50DF0901916BA6DF94
:1003C000000904E10A0E0901915D09E2640E0901C8
:1003D000915D05E27BDF7ADF0901912BF0D77F94F5
:1003E00009019151630802E216EF02F00901866BE0
:1003F000876BF66A080EF76EF86A58DF000009018D
:100400008851891102E102EF04F050DF800EF618E6
:1004100005E1FD0EF71802E1010EF81801E0F5D72D
:1004200009018651871102E102EF04F001D81200A0
:10043000F2DE09018C6B09018BA703D00901010EC3
:100440008C6F13DF9EAA17D0AECF8FF9490E09012A
:100450008F5D0AE14B0EAD6E49DF580EAD6E46DF83
:10046000330EAD6E43DF02D08FC9ADFF440E0901DC
:100470008F5D01E101D0DDD709018A6B8B6B09012A
:10048000020E8C6F09018AA902D009018C6BEDDE86
:100490002FD8020EF85C05E1420EAD6EF86A0ED858
:1004A000FF000CD8410EAD6EEAD712000000550EC9
:1004B0007E6EAA0E7E6E7F8200001200940E7F6E0A
:1004C000F5DF000EE96E090EEA6E0A000901100E52
:1004D000846F0901080E856FEE50F56E0F00852FB1
:1004E000FBD7840E7F6EE2DF842FF3D77F94120058
:1004F00000000901906B0901846B090184514B6E66
:100500004C6AD8904C5004E6840E4B5C000E4C585C
:1005100014E29EAAFED7AECF8FF909018451EA6A90
:10052000000FE96E090EEA228FC9EFFF09018F5112
:10053000090190270901842BE0D7090190510BE1B3
:10054000030E0901825D07E280C9F6FF81C9F7FF4A
:1005500082C9F8FF03D04E0EAD6ECBD71200FFFF5D
:10056000FFFFFFFFFFFFFFFFFFFFFFFFFFFFFFFF9B
:10057000FFFFFFFFFFFFFFFFFFFFFFFFFFFFFFFF8B
:10058000FFFFFFFFFFFFFFFFFFFFFFFFFFFFFFFF7B
:10059000FFFFFFFFFFFFFFFFFFFFFFFFFFFFFFFF6B
:1008000000001200280EE66E4EECFAF0E552ECEF16
:10081000F9F01200FFFFFFFFFFFFFFFFFFFFFFFFE9
:1008200068EF22F01200FFFFFFFFFFFFFFFFFFFF57
:10083000000025EC73F0C00E4B6EAF0E4C6E010E37
:10084000DAEC79F02AEF73F025EC73F0270E4B6E9B
:10085000B00E4C6E010EDAEC79F02AEF73F025EC55
:1008600073F00A0E4D6EB10E4E6E010E4F6EFE0EFF
:10087000DBCF50F05AEC74F003EC7CF02AEF73F00D
:1008800025EC73F0950E4B6EAE0E4C6E010EDAEC4D
:1008900079F02AEF73F025EC73F0800E4B6EAE0EFC
:1008A0004C6E010EDAEC79F02AEF73F025EC73F060
:1008B000D70E4B6E860E4C6E010EDAEC79F02AEFF5
:1008C00073F027EC7AF0050D22EC7BF00A0E4B2634
:1008D0000A0E4C22FD0EDB504B24E96E000E4C201C
:1008E000EA6EEF502AEF73F02FC1E6FFB8DFE55252
:1008F0001200400E012408EF79F025EC73F0000E91
:100900004B6E880E4C6E010EDAEC79F02AEF73F024
:100910009AC1C0F19BC1C1F19CC1C2F19DC1C3F19B
:100920009EC1C4F112004AEC78F09AEF7AF0640E9E
:100930004B6E4C6A9AEF7AF0E80E4B6E030E4C6EDB
:100940009AEF7AF0010156513C0DF3CF15F2F4CF36
:1009500016F21200640E4B6E4C6A38C23FF039C278
:1009600040F027EF7BF0E66A1DEC25F0E55212001F
:10097000010ED5EF73F0020ED5EF73F0650EE66E43
:10098000E60EE66E010EC8EF74F09FEC77F019E307
:10099000DDEC7AF002E60DEC79F013E29FEC77F0F3
:1009A00010E3DDEC7AF002E60DEC79F00AE29FEC60
:1009B00077F007E3DDEC7AF002E60DEC79F001E286
:1009C000010C000C020E0101815D0BE2815102E07D
:1009D000010E01D0000EE8B08A88E8B003D08A98F2
:1009E00001D08A98070E936EF18E8151010803E2BF
:1009F000F19E170E936E12002250100B08E06E0E3F
:100A000002010B5D04E3FEEC76F001E02298120097
:100A10008BEC79F00101A86BB19F1200020E01016D
:100A2000815D03E18150100B06E0030E815D04E15E
:100A30008150100B01E0000C010CF0DF000901E116
:100A4000000C010157A1010CD70E96EC75F0005077
:100A50001E0803E2F00E005C01E3000C010C610EC5
:100A6000E66EE60EE66E010EC8EC74F08EEC79F0E0
:100A700006E102EC77F003E001011E0EA86F67C1EA
:100A800000F073EC76F00A0E675D02E2200E1B6F39
:100A900012005A0EE66EE60EE66E010EC8EC74F019
:100AA0008EEC79F006E102EC77F003E001011E0E16
:100AB000A86F68C100F000500FE00101030E016F44
:100AC000ADECE6F001012D0E1A6F0A0E685D04E22E
:100AD000200E1A6F2D0E1B6F1200530EE66EE60EDF
:100AE000E66E010EC8EC74F069C100F000500AE037
:100AF0000101030E016F73EC76F00A0E695D02E2EC
:100B0000200E1B6F12000101495112002092E3ECEC
:100B10000CF0A0EC2CF01394139604907EEC3EF0B5
:100B200001018F51400B09E14A51320806E2320EB1
:100B30004A6F75EC61F0020106870101D0510BE1AB
:100B40008FAD07D00A01D76BE66AC5EC70F0E552AD
:100B5000120037EC37F01200800E081406E0215026
:100B6000010B03E10201205101E0000C010C010125
:100B7000D05109E18F51400B06E03550800B03E165
:100B80002150800B01E0000C010C37EC37F0A0EC99
:100B90002CF0B1EF16F027EC7AF004080FE071ECBE
:100BA00074F00EE0FE0EDB500A0808E0FE0EDB508B
:100BB0000D0804E0FE0EDB50090802E1010E01D031
:100BC000000E2AEF73F00701BC51D880BB5502E23A
:100BD000BBC7BCF7BB07B951B92BEA6A000FE96E76
:100BE0000C0EEA22EF501200D9CFE6FFE1CFD9FF79
:100BF000FE0EDB50D80805E1300EF36EFE0EF3CF8B
:100C0000DBFF060EAB1405E0AB980000000000000F
:100C1000AB88200EF36EFE0EDBCFF4FFF350F45CD6
:100C200004E3FE0EDB507E0807E2FE0EDBCFE6FF9C
:100C3000B2DFE552000939E00401F0514B6E4C6A15
:100C4000D8904C5004E6FF0E4B5C000E4C582DE241
:100C5000FE0EDB503B0804E0FE0EDB507C0802E198
:100C60000401F92BFE0EDB50210804E0FE0EDB50E0
:100C700040080AE13B0E0401FE5D04E07C0E040125
:100C8000FE5D02E10401F92BFE0EDBCFFEF4040150
:100C9000F151EA6A000FE96E0B0EEA22FE0EDBCF7D
:100CA000EFFF0401F12B0401F02BE552E7CFD9FF50
:100CB0001200ACA212000401F851EA6A000FE96EBA
:100CC000040EEA22EF50006E0050E66EBEECF9F022
:100CD000E5523B0E005C03E07C0E005C01E12A90D3
:100CE0000401F82B120025EC73F0ACA2FED715EC32
:100CF0007AF0BEECF9F0E5522AEF73F0A7EC0FF0B2
:100D0000010EE66EB6EC0FF0E55284948C908D9A4D
:100D10008D9CF29E0000F66A080EF76EF86A940E3B
:100D20007F6E550E7E6EAA0E7E6E7F82000000ECF6
:100D300000F012000401F007F251EA6A000FE96EB8
:100D40000B0EEA22EF50006EF22B1200E9EC73F06A
:100D50000AE12050020B07E102019C51020B04E161
:100D60009C51010B01E1000C010C4EEC78F003E109
:100D7000CE51080B01E1000C010CD9CFE6FFE1CF09
:100D8000D9FFE6522150200B01E176D08250010BB1
:100D900003E18250020B03E03050400B6DE0010193
:100DA000E3890601880EFD6F130EFE6F34AE45D049
:100DB000A7EC0FF00601880EFD6F130EFE6F010EFB
:100DC000E66EB6EC0FF0E55255EC9AF034AE2DD04D
:100DD0000601880EFD6F130EFE6F0101016B4B0EB5
:100DE000E66EE60EE66E010EE66E5BECE7F0E552AF
:100DF000E552E552AEECE4F0010EE66E6EECEFF07B
:100E0000E552000901E0FF00500EE66EA7ECF9F094
:100E1000E5528250010B08E18250020B05E101010D
:100E2000E39955EC9AF0FF00D1D70601880EFD6FCB
:100E3000130EFE6FE1EC0FF01FD0309CA7EC0FF00B
:100E4000010EE66EB6EC0FF0E552ADECE0F0BDEC55
:100E5000E0F0430EE66EE60EE66E010EE66E5BEC2B
:100E6000E7F0E552E552E552AEECE4F00101E3991A
:100E700055EC9AF0E1EC0FF0E552E552E7CFD9FFDF
:100E80001200D6EC79F0DF6AFC0E4E6E890E4F6EC2
:100E9000010E506EFD0EDBCF51F0526A536A090EFF
:100EA000FCEC73F0DFCF54F0556A566A75EC74F0C1
:100EB0000800F5CF00F0F5500DE0090EDF5C0AE206
:100EC000FE0EDB5003E11BECE7F002D045ECE7F04F
:100ED000DF2ADAD7E5522AEF73F02850200B06E01C
:100EE00005011051020118112C1101E1000C010C37
:100EF0003AEC20F012EC79F02C6B3851391102E009
:100F0000219454DAE6EF61F00701E351010B07E0A9
:100F10004DEC75F004E0050ED05D01E0000C010C15
:100F20000101279D010E0E6E27BF0E681200030EF1
:100F3000D5EC73F0268E12006A0E55EF73F06B0E2F
:100F400055EF73F001018F51010B08E041EC0EF0F9
:100F5000000904E001013C51800B01E0000C010C90
:100F6000040ED5EC73F001013C0EA86F12000101D4
:100F7000A8510DE12EAC08D0C90EE66E8D0EE66EBE
:100F8000010E74EC78F001D0EBDF268E2E8C12006F
:100F9000268E050ED5EF73F0FEEC74F000010F6E97
:100FA000E66A90EC7AF0106E12004FEC7AF0076A65
:100FB00088C1E6FFA80E4FEC73F094C100F000501A
:100FC000E66EA90E4FEC73F053EF7AF025EC73F058
:100FD000FE0EDB5048EC74F0EF500AE1EFEC77F0D6
:100FE00007E36BEC77F048EC74F0100EEF6EF0D77F
:100FF0002AEF73F025EC73F0FE0EDB5071EC77F006
:10100000EF5030080AE1EFEC77F007E36BEC77F094
:1010100071EC77F0200EEF6EEFD72AEF73F0830EAE
:101020000A6EFA0ED6EC74F000500F6E0FC010F07E
:101030000F6AFB0ED6EC74F00A6A0050B6EF75F03A
:101040000101CC51800B01E0010EF7EF77F00101B7
:101050003B51130804E2010E3B6F2CA63B6B3BEFA8
:10106000D9F027EC7AF0020802E1DFC7DEF7FE0EC6
:10107000DB0402E1DEC7DFF72AEF73F0075003E17C
:101080000101D05112000101D15112002CEC7BF072
:10109000FFEF77F043C1C9F243C1C8F22CEC7BF0FB
:1010A000EF50400B03E00201020EC86F0101D15165
:1010B000F2EC73F0EF50400B03E00201020EC96F37
:1010C0001200D6EC79F02950010B17E177EC77F09C
:1010D00016E14C5014E11850010B03E01C0E165C95
:1010E0000CE01850100B03E0150E165C06E02050C3
:1010F000100B05E00C0E165C02E1000E01D0010E93
:10110000DF6E2D50800B03E12D50400B02E0010EED
:10111000DF6E2990DF50E5522AEF73F01B9C248A82
:1011200012000101DF8B11C512F50501106B289A21
:10113000120037EC77F01EE00901BD511BE0B8EC5E
:101140007AF0BDC9E6FF8FEC0FF0E5520901BE5100
:1011500005E0BEC9E6FF8FEC0FF0E5520901BE6B5A
:10116000BEC9BDF9010137990450010B01E037896F
:101170009CEF07F0010137AF05D004A002D01B8817
:1011800012001B8A120025EC73F037EC77F00CE0AC
:10119000FE0EDB5009E0C5DFF7EC7AF00901BDAFC8
:1011A00002D001013789C8DE2AEF73F025EC73F015
:1011B00037EC77F011E0FE0EDB500EE0FD0EDB5059
:1011C0000BE0AFDFF7EC7AF078EC78F0FE0EDBAEF8
:1011D00002D001013789B0DE2AEF73F025EC73F0FD
:1011E000010137AD12D0B8EC7AF0F7EC7AF0FD0ED1
:1011F000DB5002E078EC78F001013799FE0EDBBE9F
:101200003789DB5008E098DE06D0FE0EDBAE02D058
:101210001B8801D01B8A2AEF73F080EC7CF0DBCFB7
:10122000FBF60201F45101E105D80201190EF46F39
:101230002AEF73F0E0EC79F0010EFBC6DBFF37EC30
:1012400077F063E02150200B60E00601FB51FC5D6C
:101250005CE067DF71DE01013789890EDAEC73F03B
:101260000101DFA50BD0530EDAEC73F0570EDAEC68
:1012700073F0520EDAEC73F00101DF95640E31EC7D
:1012800074F04050300FDF6EDF50300805E2DFCFE2
:10129000E6FF8FEC0FF0E552640E31EC74F0010EB6
:1012A0003CC0DBFF0A0E31EC74F04050300FDF6EB3
:1012B0000101E3A503D0520EDAEC73F0DF503008E1
:1012C00008E30601FB51630804E30101E351040B49
:1012D00008E0300EDF5C02E1540E01D0DF50DAECA2
:1012E00073F00101E3A303D0520EDAEC73F00A0E9F
:1012F00031EC74F03C50300FDF6E300EDF5C02E1F9
:10130000540E01D0DF50DAEC73F0FBC6FCF6020E8F
:10131000E15C02E2E16AE552E16E2AEF73F0690EE8
:1013200055EF73F0060E94EC7AF0280E64EC73F02F
:101330008FEF09F0010137BFF5DF12000601980EAB
:10134000D880B0553A0EB15509E20F50B05D010199
:10135000D46F10500601B159010108D0B0510F24CB
:101360000101D46F0601B15110200101D56F1200A7
:10137000190E3F6E406A0FC044F010C045F091EC6A
:10138000F5F03DC038F23EC039F2180E446E456AA1
:1013900038C23FF039C240F002ECFAF03FC038F2F8
:1013A00040C039F21200EB0E55EF73F00101E293E9
:1013B0001A9A149282EC17F0F6DF0201386B396B3F
:1013C0001A94D7EF0BF013ECAFF0320E64EC73F01D
:1013D000E30E9BEC74F0006E0050F5E1120025EC7A
:1013E00073F0F1DFEC0E08EC7CF0A0EC6FF000C7BE
:1013F0000AF0FC0E016E10C000F077EC38F0012A04
:101400000FC000F077EC38F00A6A2AEF73F0660E2E
:1014100055EC73F01A801200670E55EC73F01A90B9
:101420001200D6EC79F0A0EC1EF0DF6ED0EC77F075
:1014300007E01AA00ED0F0DFDF500BE1006A07D002
:101440001AB007D0E4DFDF5004E1010E006ED6ECE5
:1014500070F0E5522AEF73F02CC161F117EC79F0CE
:10146000EBEF1FF097EC73F003E03550800B07E0D3
:1014700001015851040B04E14BEC76F001E1000C42
:10148000010CD6EC79F001018BA10AD0A0EC1EF082
:10149000DF6EDF0403E0020EDF5C02E1010E01D02B
:1014A000000EE5522AEF73F0ECDF000905E1A0EC35
:1014B0001EF0040801E0000C010CF6DF000904E155
:1014C00092EC79F001E0000C010CD6EC79F01F50A1
:1014D000010B0EE083EC75F00BE097EC73F003E08A
:1014E000D4EC77F005E11A50020B02E1000E01D0B6
:1014F000010EDF6EDF5002E0A2EC04F0DF50E55297
:101500002AEF73F0D6EC79F01E50040B1AE01E504F
:10151000080B17E01F50010B14E083EC75F011E08D
:10152000050110510EE12150040B0BE12150010B7C
:1015300008E197EC73F003E0D4EC77F002E1000EE1
:1015400001D0010EDF6EDF5002E0A2EC04F0DF50AC
:10155000E5522AEF73F0870E56EC78F0010137ADB3
:1015600008D0410EE66E4E0EE66E38DEE552E552CC
:10157000120037BF268E120002C2E6FF01C2E6FF4C
:10158000740E38EF73F01E9C1CEC79F0D8DCE90E79
:1015900056EC78F0268E120027EC7AF00A0DF3CF85
:1015A0005AF3F4CF5BF3000E03015A27030E5B23BB
:1015B0002AEF73F06B0E005C05E20201C8510101D5
:1015C000255F1200DDEC7AF004E6990E4B5C000E0C
:1015D0004C5804E20201C8510101252712001200F3
:1015E00007C0AFF2076A280E0101D8806955040DC3
:1015F000F328016E0150E66EAA0E4FEC73F0AFC2F5
:1016000007F01200075003E00201995112000A018D
:10161000D55112000201630EAB6F010EAC6F075083
:1016200004E05D0EAB6F010EAC6F120025EC73F0A1
:101630002BA40AD0A0EC74F013EC25F05FEC7CF046
:101640000101500EA86F2B942AEF73F0159E0A012A
:10165000DA51800B06E1E9EC73F003E04BEC76F035
:1016600001E0158E12000101D051080DF3CF4DF0AD
:10167000F4CF4EF0010ED8904D364E36E806FBE121
:1016800002509FEC7BF04B50016E12000A01DA8F82
:10169000DDDF0201845156EC74F01CE24B509608D9
:1016A000000E4C5417E20268830501E1026A030E42
:1016B000835D02E1010E026EFF0E025C14E0670E14
:1016C0000A6ED1DF080EE66ED40EE66E0A0EFCEC52
:1016D0007AF009D07BEC77F01FAC03D002010989C6
:1016E00002D00201068B0201836B0101B18F500E03
:1016F000A86F2596328C12000201AE69AEC2ADF21F
:10170000AEC2B0F7AEC2AFF7AEC2AEF7AEC2ADF783
:10171000AEC2ACF7AEC2ABF70701B769B869B5693D
:10172000B669B5C7B3F7B6C7B4F7B5C7B1F7B6C7AB
:10173000B2F71200040E0101815D03E18150100B2C
:1017400007E0050E815D03E18150100B01E1000C03
:10175000010C1200D6EC79F00101A45103E19A5179
:10176000200821E2DF6A090EDF5C10E2DF50AAECFC
:1017700074F0EF50040B08E0100EDF24E66E74ECFA
:101780002BF0E552000902E1DF2AEDD7090EDF5CFC
:101790000AE2100EDF262A86DFCFE6FF31EC2BF0BF
:1017A000E552DF5001D0000EE5522AEF73F020869B
:1017B0001CEC79F0B199B19B2682248A1200D9CF12
:1017C000E6FFE1CFD9FFE6528C9600000000FE0E46
:1017D000DBCFE6FF41EC59F0E5520000C950DF6E67
:1017E00000008C86030EE66E77ECFAF0E552DF50CF
:1017F00000D0E552E552E7CFD9FF12004EEC59F088
:10180000F00EC616C680C68A1200800EE66EE66A24
:10181000010EE66E0BECF9F05FEC7CF0FEEF0BF0E6
:10182000138213800601019102011E0E2F6F120018
:10183000139020A21380139220B2138212009FEC07
:101840007CF0EF50E840E8403F0BDF6E000EDF9485
:10185000DF96DF98DF9ADF9CDF9E0A0E006EFE0E99
:10186000DB5009E1030EDF5C02E2050E006EDF5083
:1018700044E1010E41D0FE0EDB50030804E1DF50CD
:1018800002E1010E006EFE0EDB5004080EE1DF04E3
:1018900002E1320E006E020EDF5C02E15A0E006EB3
:1018A000030EDF5C02E1640E006EFE0EDB500508E5
:1018B00010E1320E006EDF0402E1640E006E020ED3
:1018C000DF5C02E17D0E006E030EDF5C02E1FA0ECA
:1018D000006EFE0EDB0404E0FE0EDB5002080DE19C
:1018E000DF5002E1010E006EDF0402E1050E006E22
:1018F000030EDF5C02E1190E006EE5522AEF73F071
:10190000020E64EC73F0C0C100F0000406E10101B6
:10191000C151460802E2020E006E030E005C06E1B1
:101920000101C151280802E2040E006ED5CA03F07D
:1019300096EC79F005E03851080B02E0040E036ED6
:10194000840E4C6E850E4D6E010EA6EC7BF0190FC9
:10195000E96E0A0EEA22EF504B24016EBB0E4C6E6C
:10196000850E4D6E010EA6EC7BF01E0FE96E0A0E81
:10197000EA22EF504B24026E02504FEC76F0E66AFA
:101980007D0EBCEC74F0020E64EC73F0280E026E57
:10199000016E96EC79F00EE03851080B0BE01CCA92
:1019A00001F021CA02F0015002E0025003E1280ECA
:1019B000026E016E02504FEC76F07C0E38EC73F044
:1019C000020E64EF73F0139A20B2138A31DF37EC02
:1019D00037F0B1EC16F02050020B06E00101D151B6
:1019E000D05D02E01B8C12001BAC02D08EEC08F024
:1019F0001200080E0C5C01E3000C010C0A5004E01C
:101A00000701010E58EC7AF00A6AC5EC04F00009EF
:101A100007E0700EE66E290EE66E010E0CEC7CF00F
:101A20001200C5EC04F0000909E07E0E0A6E080EF3
:101A3000E66ED80EE66E020E0CEC7CF00A6A12001E
:101A400080EC7CF0DBCF49F10BEC22F0F0EC76F08F
:101A5000C1EC1FF012EC79F02AEF73F007017B5113
:101A600006E1080E9BEC74F00501261501E1000C5F
:101A7000010C2D9E2D9CA0EC2CF0ACEF9AF025ECE7
:101A800073F0020143514211411107E12C50010B47
:101A900004E101018B51200B09E143C246F242C22D
:101AA00045F241C244F27FEC78F009D0FE0EDB50E3
:101AB00006E046C243F245C242F244C241F204800B
:101AC0002CA002D004902C907EEC3EF00101320E4E
:101AD000A86F2AEF73F026B41200199A18B8198A61
:101AE00012000301916B926B936B946B91C38DF316
:101AF00092C38EF393C38FF394C390F3030E016EDE
:101B0000FF0E015C32E0056A030E026EFF0E025CFE
:101B100022E00250EA6A890FE96E030EEA22EF50D2
:101B20004D6E4E6A0150EA6A850FE96E030EEA2295
:101B3000EF50E3EC7AF03FEC77F0EF50B6EC75F055
:101B40000550B6EC75F03FEC77F00FC0EFFF10C01A
:101B500005F00206DBD70150EA6A8D0FE96E030E2D
:101B6000EA2205C0EFFF0106CBD7120027EC7AF07E
:101B7000006E00AE04D0006C01010E0E126F010168
:101B8000040E006F90ECE6F0010113510AE112C15E
:101B900013F1100E126F145104E113C114F1100E61
:101BA000136F130E166F2AEF73F04DEC75F003E10F
:101BB000030E0B5C01E0000C010C4DEC75F005E12F
:101BC000020E0B5C03E00B0401E0000C010C4DEC79
:101BD00075F003E1020E0B5C01E0000C010C4DEC12
:101BE00075F007E10B5005E1CB51040B01E0020C4D
:101BF000010C000C4DEC75F005E1020E0B5C03E0EE
:101C00000B0401E0000C010C0601EC5106E04DEC68
:101C100075F003E10B50000801E3000C010C4DECE2
:101C200075F004E10B0403E00B5001E0000C010C23
:101C30004DEC75F006E1020E0B5C04E0030E0B5C4C
:101C400001E0000C010C01013D51080B03E0030E03
:101C5000D05D09E03D51040B05E0D00504E0020E23
:101C6000D05D01E0000C010CD5DC3EEC76F0EF9C81
:101C7000EADF000905E03EEC76F0EF8C0701D66B59
:101C8000120097EC73F003E059EC78F001E1000CDE
:101C9000010C0101D05104E10A01DA51040B01E108
:101CA000000C010C0101D05104E10A01DA51080BCA
:101CB00001E1000C010CD8EC77F009E00301D051F0
:101CC0004DEC7CF0D1EC74F0210E38EC73F0120086
:101CD000D8EC77F002E05BEF0EF0E66AE66A210EE0
:101CE00038EF73F04DEC75F010E1CC51040B05E0CA
:101CF0000B040CE0020E0B5C09E0CB51040B05E079
:101D00000B5004E0030E0B5C01E0000C010C010120
:101D1000D05103E1CC51400B04E1E4DF000901E1C3
:101D2000000C010CDCEC77F001E0030C9AEC79F08C
:101D300001E0080C4EEC78F001E11B0CD05109E0F9
:101D4000030ED05D05E10B5004E0030E0B5C01E0D7
:101D5000030C010CDCEC77F001E00A0C9AEC79F052
:101D600001E0380C4EEC78F001E1640CD05101E058
:101D7000500C380CEFDFE66ED5DFE66ED60EE66E61
:101D80000A0E80EF73F01FEC3FF0190E01240A01D8
:101D9000D880D75503E2190E0124D76F9EEC79F055
:101DA000D75D03E29EEC79F0D76FD46B348A010ED5
:101DB00086EF78F04BEC76F00DE1DCEC77F00AE1A1
:101DC0009AEC79F007E13FDF000904E153EC76F08B
:101DD00001E1000C010CEF0E896E8A6A8B6A9E0E7F
:101DE0008C6E900E8D6E8E6A8F6A010E906E916A67
:101DF000EF0E926E070E936E930E946E600E956EBC
:101E0000030E966E7D0E976E060E986EFE0E996E00
:101E10009A6812002098268A0101B19B020119518B
:101E200020E0020E6B5D04E1210E0101B55D19E0B9
:101E30000701E39BE39B33BEE38B46EC08F006010E
:101E4000EA05EB6F020EEA5D01E2EB6BEBC600F018
:101E50000101D05102E0EDC600F00050E66E48EC02
:101E60007AF00201196B26821200C08EA70E96EC42
:101E700075F021EC79F0A70E96EC75F0C3500F26A3
:101E8000C45010220FC04FF010C050F0D890503204
:101E90004F320FC051F010C052F0D8905232513230
:101EA000D890523251324F5051244D6E50505220E2
:101EB0004E6E0FC053F010C054F0040ED890543240
:101EC0005332E804FBE153504D5C4B6E54504E5876
:101ED0004C6E0FC055F010C056F0060ED89056321A
:101EE0005532E804FBE14B5055240F6E4C50562000
:101EF000106E0FC0EFF210C0F0F2C09E1200EFC2E1
:101F00000FF0F0C210F0E66AD0EC24F0E5520101C7
:101F1000200E176F1D6F198F410E1C6F120025ECDC
:101F200073F005011151EA6A000FE96E080E10EC1A
:101F30007CF0112B11516EEC73F004E6000E4B5C3B
:101F4000010E4C5801E3116B102B2AEF73F0C5EC16
:101F500004F000090AE026EC79F050DD1AEC46F0B6
:101F600060DD25EC46F035EC7EF0120025EC73F0D8
:101F70000101E3890601880EFD6F130EFE6F2DEC43
:101F800015F08A988A867EEC23F00101776BFE0EAD
:101F9000DB500CE00CEC0AF08FEC09F0F1ECF0F007
:101FA00084ECF1F0BCECE7F0FFECE5F00601506BDF
:101FB000F7EC3AF00601516B0101B56B89982AEFF5
:101FC00073F0F29E82ECFAF0F26AF06AB96A9D6AE6
:101FD000000EA66EA16E9E6E8D8C8D8A8C90848470
:101FE000070E936E0000000000008A9A00000000B7
:101FF00000000000270E936E4E0E996E0000000048
:10200000000003000000000000000000FF001200BC
:10201000D6EC79F021AA3DD02BEC79F006E38FECD9
:102020007BF037E2A4EC77F034E21C50080B31E18E
:102030002BEC79F006E38FEC7BF02BE2A4EC77F04D
:1020400028E22BEC79F006E38FEC7BF022E2A4ECA3
:1020500077F01FE20050DF6EDF5056EC74F015E2AF
:10206000A4EC77F012E2DF504D6E4E6AD8904E50DD
:1020700004E6B40E4D5C000E4E5807E23B0EE66ED1
:10208000E60EE66E010E8AEC78F0E66A6FDFE55246
:1020900098DFE5522AEF73F025EC73F0BDECE0F029
:1020A000A0EC74F0F8EC73F0AEECE4F087EC75F0B3
:1020B00087EC75F087EC75F002EC7BF002EC7BF0BE
:1020C0002AEF73F0010C21EC79F05DEC78F05DEC17
:1020D00078F0460E48EC77F010504B6E4C6A9F0E2D
:1020E000D8804B56000E4C564B50006E0050800866
:1020F00001E2006A0201FC0ED880EF55080EF0558F
:1021000002E2040E0FD0080ED880EF55070EF055EE
:1021100002E2030E07D0140ED880EF55050EF055DD
:1021200003E2020E002607D0200ED880EF55030EE2
:10213000F05501E2002A0050800801E2006A080E12
:10214000D880EF55070EF05502E2030E07D0140EAB
:10215000D880EF55050EF05503E2020E002612005E
:10216000200ED880EF55030EF05501E2002A120030
:10217000E0EC79F0C08EAF0E96EC75F0010158A935
:10218000D0D0500ED880C354050EC45401E3C5D03E
:10219000D00EC35C0A0EC45801E3BFD03C0E4B6E98
:1021A0004C6AEFC23FF0F0C240F027EC7BF00050E9
:1021B0003C0802E23C0E006EB4EC7AF007014B5092
:1021C000C35CF46F4C50C458F56F140EF45F050EE9
:1021D000F55B010158ABA5D0F4C7D4F1F5C7D5F133
:1021E000D4C14BF0D5C14CF0070EA9EC77F0FDE15E
:1021F0006A0E4B240A6ED4C14BF0D5C14CF00001DD
:102200004C6A4B9E4B50E824D6EC74F0AEEC75F063
:102210000101E3AF10D0E39FC80EA2EC79F004E314
:10222000840E30EC79F002E2070119D00FC0F6F706
:1022300010C0F7F76FD0C80EA2EC79F004E3840E5B
:1022400030EC79F011E20701C80EF65D000EF75987
:1022500006E3840ED880F655030EF75562E2260E8B
:10226000F66F020EF76F56D0010E07014C6AF62585
:102270004B6EF7514C220F504B5C10504C580CE3F6
:10228000F6C74DF0F7C74EF04D06000E4E5A4D50B2
:102290000F5C4E50105845E20101D0510CE107018E
:1022A0000F50F65D1050F75903E2F62B000E1CD0CC
:1022B000F607000E2ED007010F50F65D1050F759AB
:1022C00015E2F6510F5C0101D46F0701F751105868
:1022D00007EC78F003E2050ED46FD56BD4510701FB
:1022E000F6270101D5510701F72314D00F50F65DF1
:1022F0000101D46F10500701F75907EC78F003E2A1
:10230000050ED46FD56BD4510701F65F0101D5518D
:102310000701F75B0FEC30F004D00701060E58EC14
:102320007AF0D9EC74F00701CE274C50CF23CEC7FA
:102330004BF0CFC74CF030EC7BF00701CE5F4C5038
:10234000CF5B080ED880C354090EC45462E321EC5D
:1023500079F00B0E48EC77F0040E5DEC78F0E804B1
:10236000FCE1360ED8800F56060E1056EFC24BF029
:10237000F0C24CF0A9EC77F0FDE14B500F264C5029
:10238000102221BA0ED0D4C24BF0D5C24CF030ECA2
:102390007BF00201D45F4C50D55B0F50D427105016
:1023A00013D0D4C24BF0D5C24CF0640E48EC73F09D
:1023B0004B500201D45F4C50D55BAAEC7AF030EC64
:1023C0007BF00201D4274C50D523020E4C6AD6254F
:1023D0004B6ED7514C22D4514B5CD5514C5813E322
:1023E000020ED880D655000ED75513E2D6C24DF056
:1023F000D7C24EF0020E4D5E000E4E5A4D50D45DC7
:102400004E50D55906E20FEC30F0D4C2D6F2D5C208
:10241000D7F2C09E17EC75F002E2E16AE552E16E78
:102420002AEF73F0E0EC79F0C08EAB0E96EC75F00D
:10243000D9EC74F00701D0274C50D123D0C74BF012
:10244000D1C74CF030EC7BF00701D05F4C50D15B32
:10245000C09E17EC75F002E2E16AE552E16E2AEFE8
:1024600073F0C00E016E010160A302D0E00E016E98
:102470000D510126BCEF38F0D6EC79F07CEC0BF076
:10248000E9EC73F008E10701D66B0A01D56BDA932A
:102490007BEC77F016D0BCEC75F0EFCFD6F7D0C15F
:1024A000DFFFD5CA00F0080EE66EE66ADF506BEC7F
:1024B00075F0ADEC7BF0D40EE66E0A0EE66E3DECE8
:1024C00075F04BEC76F004E00A01D76BCFEC17F017
:1024D000159C0101D05103E0030ED05D06E1030E0F
:1024E0000A01D45D07E1158C05D0020E0A01D45D06
:1024F00001E1158CDAA304D0D8CADBF7D9CADCF71E
:1025000095EC17F02CEC7BF0EFCFE3F70701E39F9E
:102510000101D05103E0030ED05D02E10701E38F1A
:102520009EEC1DF035EC7BF0C3ECE4F089EC23F07D
:102530004AEC08F0E5522AEF73F064EC7AF0ADEC67
:102540007BF03DEF75F02CEC7BF0FFEC77F0E9ECE5
:1025500073F00FE00A01DAA306D0DBC7D8FADCC7B4
:10256000D9FA95EC17F0E9DF0101BCEC75F0D6C79C
:10257000EFFF1200D6EC79F0DF6A080EDF5C04E2B0
:10258000B2EC7BF0DF2AF9D7E5522AEF73F0D6ECF4
:1025900079F0DF6A080EDF5C0CE2C9EC73F0EFCF74
:1025A0004BF0FE0EDB504B5C02E1010E03D0DF2A44
:1025B000F1D7000EE5522AEF73F025EC73F015EC1D
:1025C0007AF07DEC04F0E5527F0BE4EC73F02AEF37
:1025D00073F025EC73F02AA003D059EC06F0FBD77A
:1025E0005BEC76F00FE05BEC76F0E4EC73F0D95046
:1025F000FC0FE96EFF0EDA20EA6EEE2A000EEE22E4
:10260000EE22EED72AEF73F025EC73F02AA003D068
:1026100059EC06F0FBD739EC7AF0E80E446E030E65
:10262000456E33EC7AF040C04CF09DEC7AF0E80E49
:10263000446E030E456EB5EC73F0640E48EC73F017
:102640009DEC7AF0640E446E456AB5EC73F00A0EA8
:1026500048EC73F09DEC7AF00A0E446E456AB5ECD6
:1026600073F0300E4B24E4EC73F02AEF73F025EC9A
:1026700073F01FAE0FD0360EE66EE60EE66E010E5C
:10268000E66EA7DF5FEC7CF0A0EC74F0A2DFE55211
:10269000E552E5522AEF73F0D6EC79F00201F12B06
:1026A0001FAE19D06D0EE66EE60EE66E010ED0EC92
:1026B00073F015EC7AF081DFE552FE0EDB28E66E52
:1026C0007CDFE552FE0EDB50020FE66E76DFE55250
:1026D0003B0EE4EC73F015EC7AF059DFE55200099B
:1026E00015E1DF6A080EDF5C11E2C9EC73F0EF5010
:1026F000FF080AE1C9EC73F0FE0EDBCFEFFFC3EC7D
:1027000075F026C7EFFF02D0DF2AECD70701266954
:10271000E5522AEF73F0D6EC79F0DF6A080EDF5C41
:102720000FE2C9EC73F0EF50FF0808E0C3EC75F05E
:10273000EF50016EC9EC73F0EF5003D0DF2AEED7F3
:10274000FF0EE5522AEF73F0E0EC79F0DF6A080E35
:10275000DF5C0FE2C9EC73F0010EEFCFDBFFDB5063
:10276000FF0805E0B2EC7BF0010EDB5003D0DF2A5E
:10277000EED7000EA6EC79F002E2E16AE552E16ED6
:102780004B502AEF73F0D6EC79F03350200B04E174
:10279000020E07017B5D02E1DF6A03D054EC7BF09F
:1027A000319ADF50E5522AEF73F0E0EC79F03350C4
:1027B000200B04E1020E07017B5D03E1DE6ADD6AA6
:1027C00008D054EC7BF0E66A90EC7AF03AEC79F0C1
:1027D000319A17EC75F002E2E16AE552E16E2AEFF8
:1027E00073F0D6EC79F007017F6B806B2EA802D0D6
:1027F000010E27D0080E9BEC74F0DF6E07017F2BD3
:10280000000E8023200EDF1405E0580E7F5D020EBF
:102810008059F0E37F51815D8051825904E27FC786
:1028200081F780C782F7580E7F5D020E805908E35A
:1028300001018C5103E1330E51EC74F0000E01D014
:10284000010EE5522AEF73F025EC73F08EEC78F070
:102850002AEF73F008EC7BF004E2FE0EDB50300F41
:1028600004D0FE0EDB50F60F410F2AEF73F0010E7D
:10287000006E02017CB9008E002A0050E66E060E42
:1028800001013603F350E66E780E38EF73F0D6ECA4
:1028900079F0A0EC1EF0DF6E0F0EE66EDF5007E061
:1028A000030EDF5C04E001018B51020B02E1000E1C
:1028B00001D0010E000905E00A0E01017B03F3506F
:1028C00001D0000EE66E7E0E38EC73F0E5522AEF72
:1028D00073F065C17CF259EC78F002E166C17CF2DC
:1028E000120059EC78F003E17CC266F102D07CC2A0
:1028F00065F1EFDF37EF14F0A0C20FF0A1C210F0C6
:10290000B9EC7BF05E0E38EC73F0A2C20FF0A3C2FC
:1029100010F0B9EC7BF05F0E38EC73F0A5C2E6FF67
:10292000A4C2E6FFE66A7B0EBCEF74F00601B46B4E
:10293000B56B020EF5EC76F00601B42B000EB52354
:10294000B451B65DB551B75904E2B4C6B6F6B5C6D2
:10295000B7F6E80ED880B455030EB55509E2310E2E
:10296000E66EE60EE66E010EC8EC74F03286010CDF
:1029700084B0DFD7000CD6EC79F02E50100B03E1B9
:102980003250100B02E1000E20D032A604D00A0E05
:10299000F5EC76F001D0CADF15EC7AF0DFEC0BF045
:1029A000E552DF6EE66ADFEC0BF0E55201013951CA
:1029B000100B0AE03150200B07E1E3A102D02E0EEC
:1029C00001D0210E19EC7AF0DF50E5522AEF73F0B6
:1029D000F5EC79F00101E3912AEF73F0F5EC79F071
:1029E000FC0E60EC73F00101E3912AEF73F0F5EC5B
:1029F00079F0BFEC7BF00101E3912AEF73F0F5EC85
:102A000079F0BFEC7BF0FA0E60EC73F0F90E60EC3D
:102A100073F00101E3912AEF73F084EC7CF0D4C1F0
:102A2000E6FF90EC7AF0D5C1E6FF90EC7AF00FC0AB
:102A3000E6FF90EC7AF010C0E6FF90EC7AF001012E
:102A4000E3912AEF73F01D0E08EF7CF01E0E08EFE5
:102A50007CF0D9CFE6FF2AEF73F02BB203D0600EE3
:102A600055EC73F02B8212002BA203D0610E55ECB3
:102A700073F02B9212002BB203D0600E55EC73F062
:102A80002B8212002BA203D0610E55EC73F02B9217
:102A9000120025EC73F032B206D0620E55EC73F0E2
:102AA000FE0EDBCF1AF22AEF73F025EC73F0B00EB6
:102AB00055EC73F0FE0EDBCF1BF22AEF73F025EC22
:102AC00073F00701A851320D3FEC79F0AAEC79F0D0
:102AD00012E1FE0EDB500FE10101D05104E12A5159
:102AE0000A0D3FEC79F0E0EC77F005E00101E80E2B
:102AF000D46F030ED56F2AEF73F0D6EC79F0D6CAF7
:102B0000A7F707011E0EA86F0101D05106E1050EBF
:102B1000C2EC74F040C0A8F710D0030ED05D0DE1F8
:102B2000030E0B5C03E10701140E06D018EC76F0DF
:102B300004E00DEC7BF00701A86FD7CA00F0070195
:102B4000E3AF10D0190E006E0A01D75D06E261EC0A
:102B500078F015EC7CF0005E05D0190ED75D15EC11
:102B60007CF00026190E005C05E3190E005C0701DD
:102B7000A82705D0190ED88000540701A85F080EB9
:102B8000006E22A20FD00101D05102E1020E18D036
:102B9000D00506E0020ED05D03E0040ED05D11E129
:102BA000010E0ED00101D05102E1080E09D0D0056E
:102BB00006E0020ED05D03E0040ED05D02E1070ED8
:102BC000006E0701A751FE0BE8420024056EDF6A84
:102BD0000550A85D13E2DF2AA751FE0BE842A825A5
:102BE000016E01500024FE0BE842A86F0050015C0A
:102BF00002E20050016E0050015CA76FA7C7A6F764
:102C00004EEC78F004E10701A751E824A66FE9EC47
:102C100073F006E10701320EA76F1F0EA86FA669B9
:102C20000750E96EEA6AD890E936EA36AC0EE92632
:102C3000060EEA22EECFA9F7EDCFAAF74EEC78F018
:102C400021E2DFCFE6FF3BDFE552020E0101D05D5E
:102C500008E0EFEC0DF0020804E087EC0EF000094C
:102C600009E00101D4510701A9270101D55107014C
:102C7000AA2308D00101D4510701A95F0101D55150
:102C80000701AA5BAEEC79F062E00701E351800B2B
:102C900029E0DF5027E1F4DA0FC0D4F110C0D5F1FC
:102CA0000A01D751190808E2190ED75D93EC7CF0A0
:102CB0000101D4274C50D523AAEC79F008E261EC4D
:102CC00078F093EC7CF00101D45F4C50D55B0101AE
:102CD0000A0ED503F3CFD5F1D403F3CFD4F1F450DA
:102CE000D52704D0DFCFE6FFEADEE5520701A75182
:102CF000320DDFEC73F03EEC08F0030802E1010155
:102D0000D58F200E006E0701AD51005C10E1B3516C
:102D10000101D4190CE10701B4510101D51907E1F2
:102D20000701B5510F1802E1B65110180DE000C0AF
:102D3000ADF7D4C1B3F7D5C1B4F70FC0B5F710C024
:102D4000B6F700505CEC7BF04CDD5BEC0EF080ECF9
:102D50000CF062EC4BF00701042B0407E5522AEF5C
:102D600073F01CEC76F0005001E11200AEEC79F04B
:102D700067E00101DC0ED46F050ED56FF00E0F6E0B
:102D80000A0E106E030E005C01E1D58F000403E013
:102D9000020E005C47E141EC0AF0000917E0010176
:102DA0008A51640DDFEC73F00FC0D4F110C0D5F17F
:102DB000010E0F0B05E0D890D533D433E806FBE1C4
:102DC000640E0101D427000ED5232CD0010135510A
:102DD00029E03551080DF3CFD2F1F4CFD3F15C0ED9
:102DE000D227000ED323D2C14BF0D3C14CF0F00E4A
:102DF000D8804B560A0E4C56010E0F0B03E044ECE4
:102E000079F0FDE14B500101D225D46F4C50D32114
:102E1000D56FD2C10FF0D3C110F0F00ED8800F568D
:102E20000A0E1056050ED05D08E10E0ED46F060E88
:102E3000D56FC40E0F6E090E106E300E5CEC7BF079
:102E4000F1EF13F01200640E55EF73F0E0EC79F03F
:102E500097EC73F022E071EC74F01FE107017B51F5
:102E60001CE102013851391118E1185116E1010134
:102E70003C51800B03E1050ED05D0FE1080E9BEC89
:102E800074F0DF6EE9EC73F003E1E09FDFA8E08F00
:102E90003CAF03D0010EDF1401D0000EA6EC79F098
:102EA00002E2E16AE552E16E4B502AEF73F0010154
:102EB0003C51800B06E097EC73F003E071EC74F08A
:102EC00001E0000C010C54C1E6FFF1DF000903E052
:102ED00001016F5101D0000EE66E340E38EC73F034
:102EE00070C1E6FF350E4FEF73F0650E55EF73F0CE
:102EF0002150400B06E00101E151040B02E1E185A4
:102F000001D81200D6EC79F055C1DFFF59EC78F00A
:102F100002E159C1DFFF080EDF02F350E66E750EC5
:102F20004FEC73F0E5522AEF73F00701DB510C0808
:102F300003E3DC510C0805E2DB6B0C0EDC6F0A01CD
:102F4000DA931200016A0D0E015C07E067EC76F07F
:102F500002E001501200012AF6D7000C0C0E016E9F
:102F6000015007E067EC76F002E001501200010624
:102F7000F7D7000C0701D96BDA6BD7DFDBC701F09D
:102F80000701DC51D880015409E379EC04F0F350D7
:102F90000701D913F450DA13012AF2D71200016A9B
:102FA000DCEC77F00BE045EC7AF006E24B500508DC
:102FB000000E4C5401E2012A4D0E0DD09AEC79F02E
:102FC00012E045EC7AF006E24B501408000E4C5427
:102FD00001E2012A4F0E012408EC79F0F3CFD9F772
:102FE000F4CFDAF7120045EC7AF017E24B504608BE
:102FF000000E4C5412E253EC76F00FE10701F40E90
:10300000D96FDA69E9EC73F001E1BAD00701DB6B43
:103010000C0EDC6F0A01DA83B3D0006A0A01D751C3
:1030200056EC74F006E24B500D08000E4C5401E2D1
:10303000002AD75156EC74F006E24B501308000EEC
:103040004C5401E2002AD751180801E2002AD75156
:10305000190801E2002AD75156EC74F006E24B50F1
:103060001F08000E4C5401E2002AD75156EC74F0B0
:1030700006E24B502508000E4C5401E2002A53ECA6
:1030800076F007E0020E006E0101CEA302D0040E1E
:10309000006E0101D05103E0030ED05D1CE145EC50
:1030A0007AF006E24B500508000E4C5401E2012A6A
:1030B000B1EC7CF006E24B500A08000E4C5401E2E1
:1030C000012AB1EC7CF022E24B501308000E4C5464
:1030D0001DE2012A1BD045EC7AF006E24B501E0897
:1030E000000E4C5401E2012AB1EC7CF006E24B5098
:1030F0002808000E4C5401E2012AB1EC7CF006E2F3
:103100004B503208000E4C5401E2012A4D0E4E6E17
:10311000AF0E4F6E010E506E0050516E526A536AE0
:10312000030ED890513652365336E806FAE1C1EC18
:103130007AF00150546E556A566AD8905436553616
:10314000563675EC74F00900F5CFD9F70A00F5CFC3
:10315000DAF7D8EC77F005E00701D985DA89D99D4F
:10316000DA9B030E0A01D45D02E0D45109E1EADEE4
:103170000701DB6FF3DE0701DC6F0A01DA83D5DEBE
:103180000A01D40514E10701DC05056E0A0EDC5DB9
:1031900001E20506D7DE0701DB6F0550D880DB555D
:1031A00002E205C0DBF7E6DE0A01DA831200020E56
:1031B000D45D12E10701DB29056EDB51020801E253
:1031C000052ACCDE0701DC6F0550DC5D02E205C09C
:1031D000DCF7D0DE0A01DA8312001E0E006E010158
:1031E000D05105E1050EC2EC74F040500AD0E0EC7D
:1031F00077F002E0140E05D018EC76F003E00DEC49
:103200007BF0006E0A01D651FE0BE842056E1200FB
:10321000170E44EC75F0050E0A01D803F350006E4A
:103220000101012B73EC76F01C8F12001A0E44EC96
:1032300075F00A01D9514DEC7CF063EC7BF01C8FEA
:103240001200E4EC77F00101960EA86F3C51200BC0
:1032500006E102EC77F003E001011E0EA86F6FECAF
:1032600060F071EC75F0300E01011A5D02E1200E84
:103270001A6F1C8F016B660E006E248848EF24F0D5
:103280000101D05102E12A510BD0030ED05D11E1B2
:10329000030E0B5C02E1640E03D00B5004E1960EAA
:1032A0000F6E106A1200240E2F258CEC75F00F6E35
:1032B000106A120092DF0701E3AF17D000504DEC07
:1032C0007CF0DEDF0A01D751190804E2190ED75D40
:1032D000B6EC75F0190ED75D1CE261EC78F093EC5A
:1032E0007CF00F5E4C50105A12000A01D751190899
:1032F00003E2190ED75D0026190ED75D03E261ECDB
:1033000078F0005E00504DEC7CF0190ED75D01E1C5
:10331000B7DF120053EC76F00AE00101CE930A0108
:10332000D751190802E20101CE830A01D76B1200BE
:1033300053EC76F009E00A0ED5EC73F00101CEA350
:1033400034D00B0ED5EF73F0A10E44EC75F08EEC7B
:1033500079F006E102EC77F003E001011E0EA86FA0
:10336000A9DFD8EC77F00BE00101410E176F500E8A
:10337000186F0301D051106AE8307F0B0F6E63ECB9
:103380007BF0D8EC77F009E00101460E196F2A5165
:10339000E8240301D05D07E103D0AAEC79F003E152
:1033A00001012A0E1A6F01011C8F120025EC73F027
:1033B000070EE12692EC0EF00A01D65D04E292ECD3
:1033C0000EF00A01D66FAAEC0EF00A01D880D6558D
:1033D00004E2AAEC0EF00A01D66FDAEC0EF0000956
:1033E00003E00A01190ED76FF8DEAAEC79F004E3C6
:1033F000190ED75D002603D061EC78F00526055044
:10340000005C03E30550005E0AD0006AD40507E1C2
:10341000DC51D75D04E2DCCAD7FADDCAD6FA00C0B7
:10342000D8FADBDE05500026AAEC79F004E3190E89
:10343000D75D002609D061EC78F0056E0550D88084
:10344000005402E20550005E8FEC7BF00BE24B5023
:103450005408000E4C5406E2540E006EDCCAD7FA33
:10346000DDCAD6FA00C0D9FA00C0E9F7190ED75D57
:1034700003E3190ED75D03D0190ED880D755070185
:10348000D76FD86BE3AF02D00A0E01D0320ED8034B
:10349000F3CFD8F7D703F3CFD7F7F450D8274BECB7
:1034A00076F0FE0EDB501EE02150800B1BE10A017E
:1034B000D45102E1C6DE0AD0D40502E1A9DE06D06D
:1034C000020ED45D02E1B2DE01D032DF0101960EC0
:1034D000A86F3C51200B06E102EC77F003E00101FC
:1034E0001E0EA86F3550080B13E10A01DA51020BCA
:1034F0000FE04BEC76F00CE1DCEC77F009E19AECB4
:1035000079F006E1D8EC77F003E153EC76F003E0D4
:1035100046DD359601D02EDD0701010ED56F010184
:103520002BA303D00701070ED56FD5CADFFF0A0111
:10353000D56B0701D551010858E201013C51100B30
:1035400054E1CE51010B51E1050ED05D4EE0040E69
:10355000D05D4BE0D00503E0020ED05D11E10A0121
:1035600092EC7BF002E6B7EC77F00AE2D52B92EC16
:103570007BF004E61E0E4B5C000E4C5836E220D069
:103580000101D0511FE10A0192EC7BF004E61F0E0D
:103590004B5C000E4C5801E2D52B92EC7BF004E61C
:1035A0000F0E4B5C000E4C580BE3D6514D6E4E6A1D
:1035B000D8904E5004E60B0E4D5C000E4E5815E2AE
:1035C000D52B13D00A0192EC7BF004E62D0E4B5C58
:1035D000000E4C5801E2D52B92EC7BF004E60F0E66
:1035E0004B5C000E4C5801E2D52BDF500A01D55D33
:1035F00011E0D5CADFFFC3ECE4F0D5CAE6FFAB0E9D
:103600004FEC73F0258A1FAC03D00201098902D068
:103610000201068B37EC37F0070EE15C02E2E16A4B
:10362000E552E16E2AEF73F0006A800E066E056EB9
:1036300005500502F350015CF4500258D8B008D090
:1036400000C005F006420650051206BE09D0F0D7AC
:1036500005C000F006420650051206BE01D0E8D7AC
:1036600000D0120025EC73F02B8431EC12F000C076
:10367000E5F749C102F0B2EC79F00250E3EC7AF0E0
:103680000F50016E10C002F0CFDF0A0E516E51C014
:1036900045F00BC240F095EC7BF04F6E506AB2ECF7
:1036A00079F0720E3F6E010E406E19EC7CF093ECD7
:1036B00078F07BEC7CF04FC044F050C045F0E2EC79
:1036C00076F0036A3DDB016E1D50040B31E001040E
:1036D00003E0020E015C2CE13550800B29E1FE0E67
:1036E000DB5026E002C202F0025022E002506EECF3
:1036F00073F004E6800E4B5C000E4C5819E2025049
:10370000FE0BE842D880005413E20250E824005C2B
:103710000FE2FE0EDB0406E10C0E02010127000E93
:10372000022305D00C0E0201015F000E025B032A8A
:1037300003500EE1880ED8800F54130E105404E28B
:10374000880E0F6E130E106E0FC001F210C002F241
:103750002550020B06E12350400B03E03250800B52
:103760000AE0036A006A32AE06D0000E0201036F5F
:10377000046B016F026BBCEC0AF02AEF73F025ECCE
:1037800073F0D1EC74F015EC7AF0EEEC14F05FEC21
:103790007CF02AEF73F025EC73F012EC7BF0770EDF
:1037A000BCEC77F0FE0EDB5005E0075003E1100E95
:1037B000BCEC77F02AEF73F01CEC76F0050E005CA1
:1037C00005E0B6EC79F002E1000E01D0010E00092F
:1037D00002E0000E03D001013551E824E66E3C0EF4
:1037E0004FEF73F01EEC3DF0E7DF0201C65103E03E
:1037F0000101355106E00201C65105E101013551D3
:1038000002E0B1EC16F02B841200016A65EC78F04E
:1038100001E1012A006A329084EC76F0020E97EC06
:103820007CF0800B05E084EC76F0EF50006E328087
:103830001200D6EC79F0FE0EDB5003E001012951B5
:1038400001D0000EDF6E22B204D0040EDF02F3CFEF
:10385000DFFFDFCFE6FF760E4FEC73F0DF90DF4245
:10386000DF5005E1FE0EDB5002E0010EDF6EDFCF20
:10387000E6FF790E4FEC73F0E5522AEF73F025EC7A
:1038800073F0016A080E015C15E2FE0EDB500124A4
:10389000E66EDAEC7CF0E552026E100E025C040D6E
:1038A000F350006E010E64EC73F0005055EC73F0B1
:1038B000012AE8D7140E64EC73F02AEF73F0AEEC33
:1038C00079F00DE0220E55EC73F03EEC08F00009A3
:1038D00002E1180E01D0080EE66ED1DFE552F1EFDD
:1038E00013F0AEEC79F00DE0310E55EC73F05DECB9
:1038F0000AF0000902E0100E01D0000EE66EBFDFF4
:10390000E552F1EF13F04FEC7AF0240E0101B55DB2
:1039100003E1076AD4DF01D0E4DF53EF7AF00AEC69
:103920000BF03EEC76F0EFCF4BF09AEC78F0EF50E6
:103930004B5C20E03EEC76F0EF50E66E9AEC78F0CF
:10394000E552E750EF6E01016351020B05E1CC51E6
:10395000200B02E1000E01D0010E000902E0000E72
:1039600001D0380EE66E0F0EE66EC80EE66EA10EA2
:10397000BCEC74F01200120077EC75F02B922DEC79
:1039800015F0E66A720E4FEC73F03C0EE66E710EA7
:103990004FEC73F07DEC15F075EC17F0F0EC0AF0DD
:1039A000075002E1D5EC07F0C9D87BEC7AF0E66A63
:1039B000130E4FEC73F0010163855D9534EC0EF04E
:1039C000AEDFA7EC4BF0E668B30E4FEC73F0075098
:1039D00001E144D862EC4BF0D3EC4CF09FEC07F0E3
:1039E0007CEC14F069EC14F037EC14F082EC17F076
:1039F00078DFF0EC76F0E0DE47EC14F063EC17F0E3
:103A000004DF22EC17F0010EE66EC5DEE55277EC1E
:103A100075F00601B26B090EB36F51DF0101605101
:103A2000200B02E0640E01D0320EE66E1F0E4FEC4A
:103A300073F0010EE66E0F0E4FEF73F01200046A82
:103A4000010160AF04D012BC048012BE04823DB9F3
:103A5000048453EC76F001E004881200010113980D
:103A60003C51100B01E013883C51100B19E022501F
:103A7000020B16E01F50200B13E0CE51010B10E19A
:103A8000050ED05D0DE0040ED05D0AE03C9B228463
:103A9000060150955087248A2682030E006E06D0B8
:103AA00032C100F0B6EC79F001E0006A0050E66E39
:103AB000A60E4FEF73F0016A0701E3B302D04CC1C9
:103AC00001F04DC102F0E351020B09E00101D051B8
:103AD00004E10601EA51010802E34EC102F00F0EB3
:103AE0000101D8804255E66E02504FEC76F07EC15F
:103AF000E6FF48C1E6FFA00EE66EFFEC14F04B6E49
:103B0000060EE15E4B500701E3B10FD00101CEADCF
:103B100003D0CE9D62EC4BF01550100B06E0155013
:103B2000200B03E11598D3EC4CF00701E351010B96
:103B300002E0AE0E01D0AD0E55EF73F05BEF1DF05D
:103B4000D6EC79F01CEC76F0000403E0020E005C89
:103B500008E1E66A3450080B02E0030E15D0000EAF
:103B600013D0005005E1010EE66E15DEE5522DD0B2
:103B7000050E005C0BE102019C51040B02E09A511E
:103B800001D0000EE66E040EE66E21D0030E005C3E
:103B90001CE171EC74F019E0020E0B5C03E181ECA6
:103BA00077F00CD0E80E0F6E030E106ED1EC74F0AF
:103BB0003E0E38EC73F0E66A020EE66E140E38EC38
:103BC00073F00501040E266F05D0E66AE66A140E4E
:103BD00038EC73F0E5522AEF73F0D6EC79F00AEC8A
:103BE0000BF002012E6B0601BF6BBFC6BEF6349010
:103BF0000101D05124E10601EA51010803E3145008
:103C0000010B17E0016AEA05EB6F020EEA5D03E3C0
:103C10000201195102E00601EB6BEBC6E6FF48EC2E
:103C20007AF0E66A030EE66E120E38EC73F034801A
:103C300004D07BEC7AF00601EB6B80DF58D0030EEA
:103C4000D05D53E13EEC76F0EF981450010B06E1A5
:103C5000DCEC77F003E1BAEC79F043E018EC76F0B5
:103C60000AE02D0EDF6E010E016E026A14A00ED066
:103C700002012E6F0BD0E0EC77F006E0020E016E31
:103C8000026A1F0EDF6E02D0016A026AE66A015004
:103C9000E66E120E38EC73F0EDC6E6FF48EC7AF0F3
:103CA0003480DCEC77F003E03EEC76F0EF8807013F
:103CB000200E726F3F0EDF5C02E1100E726F640E19
:103CC000DF5C02E10A0E726F4B0EDF5C02E10D0E4B
:103CD000726F2D0EDF5C02E1160E726F6F6B736BED
:103CE00002D07BEC7AF01BDE02D07BEC7AF0B0ECF9
:103CF00036F0E5522AEF73F0BF0E96EC75F00050E7
:103D0000E840E8403F0B005C02010B6F060E00C06C
:103D1000E7FF070B04E0E742E79EE806FCE1E75017
:103D200002010B5F0B076E0E0B5D07E22250100BBA
:103D300004E1228870DBF0EC76F00BC200F0120098
:103D400020B203D00101D05112000101D151120063
:103D50000C0E55EC73F0FEEC74F00F6E106AFF0E53
:103D60000F1804E1105002E10F6810681200466B52
:103D7000476B486B496B400E4A6FD89041374037CC
:103D80003F373E373D373C373B373A37493748377F
:103D9000473746374551495D445148594351475982
:103DA0004251465909E34551495F4451485B4351EB
:103DB000475B4251465B412B4A2FE0D7120001017D
:103DC000CC9712BECC87CD9912BCCD8912000A0EB9
:103DD00047EC79F001010490CC51080B01E004801C
:103DE0000492CD51100B01E00482129E04B0128E99
:103DF000129C04B2128C07010A970A990A8504A042
:103E00000ED00101CC5107010A99010B01E00A898A
:103E10000101CC5107010A97020B01E00A870A5100
:103E2000100B06E10101785103E10450020B02E09E
:103E300007010A9507010A9104B20A8155ECF1F0D5
:103E40001FEF1DF0D6EC79F0C5EC7BF0200EE0EC16
:103E50007AF00050026E0F0EE0EC7AF001012C5166
:103E6000005C33E1250E025C30E1050EE8EC7AF0EF
:103E70004DEC75F01DE2010EE66E0A0EDF24E66ED3
:103E8000060EE66E010E3DEC73F00F0E01010617F3
:103E9000D051065D0DE0298206C1D0F1B0EC36F0BC
:103EA000FFECE5F035EC61F0B0EC36F02682248AC8
:103EB000E9EC73F007E1030EE66E100EDF24E66E08
:103EC0006BEC7BF00A6A010E02D00A6A000EE55222
:103ED0002AEF73F025EC73F01FAC03D002010981C7
:103EE00002D0020106832C8C2D8A000EB06FB16BBC
:103EF0008D6F8E6B9BEC73F0EE50ED1013E00101B3
:103F0000452B640E455D03E29DDF00091DE10101C3
:103F10004507FF0E455D03E095DF0009F8E101016B
:103F2000452B12D001014507FF0E455D03E08ADFF6
:103F300000090AE10101452B640E455D03E282DFC1
:103F40000009F8E1010145072AEF73F02A50800BC0
:103F50000DE001013851400B09E02C50100B06E137
:103F60002B50010B03E1100E2C5D01E3000C010C42
:103F7000EDDF000905E001014951780801E2010C7B
:103F8000000C258A120025EC73F0540E4B6E8F0E38
:103F90004C6E010EDAEC79F07F0B006EFE0EDB50FA
:103FA000040806E1FD0EDB50310802E2020E006E4D
:103FB0002AEF73F0040E0101445D01E3446B160E19
:103FC00044251EEC7CF0E66EE66A3C0EE66EBAEC2A
:103FD000F7F0E5EF79F022900201320E236F2851BD
:103FE00002E0140E236FC80E376F640E3D6F1EACD7
:103FF0002A981E50400B03E02B50800B02E12DEC61
:1040000015F0020109870985098309817E6B120079
:1040100025EC73F0FE0EDB500EE02AA006D0FE0E5B
:10402000DB50030B02E159EC06F0280EF5EC76F0BC
:10403000FE0EDB06EFD72AEF73F011C512F505016E
:10404000106B289C0101E091120028BA09D013C519
:104050004AF114C52AF1259224BC258275EC61F041
:10406000288A010137999FEC07F00201206B249AFE
:104070002692120051EC79F0E0DF2850200B05E089
:1040800071EC74F002E0080E086EDFDF3098120069
:104090000850220A01E1A3D1030A01E184D1010AF7
:1040A00001E1F5D03F0A39E0010A01E0B2D1288CE4
:1040B0004AC113F52AC114F5249C25B2248C28BAD0
:1040C00015D0010137AD11D0E3B706D03751070B3A
:1040D000050DF3500A0F4A6F640E2A6F37B902D0EC
:1040E000430E2A6F5DEC61F001D0C4DFBAEC79F0C9
:1040F00007E0200E06014A5D03E0200E48EC75F053
:104100001E901F0E086E02012C5101E183D1285030
:10411000200B01E17FD1086A1AD00501105101E19D
:104120008CD071EC74F016E02850200B13E00501E0
:10413000235107E1020E265D0DE12EEC0DF0000982
:1041400009E102012C5101E12C2B080E086E1F0E13
:10415000096E1200050110071251EA6A000FE96E9C
:10416000080EEA22EFCF02F7122B12516EEC73F019
:1041700004E6000E4B5C010E4C5801E3126B71EC2F
:1041800074F009E02850200B06E002C7E6FFDCECE3
:1041900039F0E5524FD03C0E0701025D04E1258263
:1041A000248C239C12003E0E025D06E12592249C85
:1041B0001FBC30D1238C1200740E025D67E0060133
:1041C000EA510AE02850200B07E02A8A02C7E6FFDE
:1041D00048EC6BF0E5522A9A800E0701025D0FE26F
:1041E0003F0E4B6EAE0E4C6E010E4D6E200E025DFC
:1041F00057EC76F02EEC73F00800F5CF02F7800E46
:10420000025D03E10201040E556F070102518008AF
:1042100005E2800E025DFD0F0201556F800E070161
:10422000025D06E3220E086E05011F0E156F1200D7
:1042300002512CE0200E086E120028BA02D03AEF8C
:1042400020F0C1EC77F007E007010251800803E39A
:10425000200E48EC75F00EDF71EC74F005E0289C40
:10426000080E086E100E096E2850200B01E1D2D006
:104270000201585101E1CED0199A58BF198A186B22
:10428000010EE66E7F0E58150FEC78F012001850F4
:10429000800B06E02850200B09E10B0E165C06E0AF
:1042A0001E50040B03E01E50080B56E12850200B53
:1042B00009E01850800B06E0BEEC79F003E00B0E2D
:1042C000165C1DE1E6EC61F0D5DE219428AAA2D0AF
:1042D00071EC74F003E00201010E2C6F12EC79F026
:1042E0000601EA5101E196D007010251800801E27E
:1042F00091D03088200EE66E48EC6BF027D0230E6C
:10430000165C0EE1010EE66E3FEC0DF0E5521FACBF
:1043100003D00201098702D002010681189E120013
:1043200061EC9AF0000914E02850200B11E00D50C8
:10433000006E020EE66EF1EC2AF0E5520D50026EB0
:1043400000500D6E0250E66EFEEC6FF0E55212006A
:1043500028AA28D0D3EF9CF071EC74F008E0285024
:10436000200B05E0080E086E1F0E096E1200FE0EEF
:10437000070102150FE0238E010E016F02A102D08A
:10438000030E016F02910243210E086E0501200EFB
:10439000156F12000201020E556F220E086E050104
:1043A0001F0E156F12000701015112E00107248052
:1043B0008FEC61F0086A1EA006D0020E086E28BAC3
:1043C00002D043EC76F0210E096E1E80239E12006F
:1043D0000201010E556F238E220E086E120002019B
:1043E000555114E0249055078FEC61F0030E086ED0
:1043F0001EB007D0070E086E28BA03D0006AD6ECAC
:1044000070F0220E096E239E1E90120015C508F052
:10441000120030DE1200020174510101D8804955AA
:1044200002E274C249F12C510A080EE2100E2C5D12
:10443000AAEC74F0060E97EC7CF0016E0150D88067
:10444000495502E201C049F10A0E2C5D05E14951CE
:10445000640802E2640E496F02010B516EEC73F0C6
:1044600004E6820E4B5C000E4C5806E201014951F5
:10447000640802E2640E496F6E0E02010B5D05E2F4
:10448000E7EC77F002E2320E496F2250100B05E0A4
:10449000E7EC77F002E2320E496F010149511E0844
:1044A0000AE26E0E02010B5D0CE3E7EC77F009E324
:1044B000C2EC79F006E0010160B309D0608384EFBB
:1044C000F1F0010160A303D0609384ECF1F01200DD
:1044D000DACFE4FFE2CFDAFFE9CFE4FFEACFE4FF8F
:1044E000E652FC0EB36EF30EB26E0201110702012A
:1044F000115105E10201320E116F0101228101010A
:10450000E3A92CD00601FD07000EFE5B0601FD515C
:10451000FE1124E1F29EF26AF06AB96A9D6A000E09
:10452000A66EA16E9E6E8D8C8D8A8C908494070EE3
:10453000936E0000000000008A9A00000000000056
:104540000000270E936E4E0E996E000000000000D2
:1045500003000000000000000000FF001F801E8616
:104560001E8481B20BD0010150A302D01F9006D04F
:10457000010150A102D01E9601D01E9481B40BD02F
:10458000010150A302D01F9006D0010150A102D01A
:104590001E9401D01E9687B60BD0010150AB02D0FD
:1045A0001F9006D0010150A902D01E9601D01E9482
:1045B00081B00BD0010150AB02D01F9006D0010199
:1045C00050A902D01E9401D01E96020112070201CA
:1045D000125137E10201050E126F0101AC5116E0D4
:1045E0000101AC07020102015451020B05E01E500B
:1045F000040B02E102015481020102015451080B33
:1046000005E01E50080B02E1020154850101AD5185
:1046100006E0FF0E0101AD5D02E00101AD2B20AE11
:1046200004D00601DE2B000EDF230701715109E0E3
:10463000070171070701715104E172C771F70101A8
:1046400022830101AB5102E00101AB070101279771
:1046500001012795010127A102D001012785010150
:1046600027A302D001012787010127930101279188
:1046700088A202D00101278188A002D001012783EE
:104680000F0E010127150101246F01012451EA6A6F
:10469000C50FE96E060EEA22EFCF23F1010E0101EC
:1046A000231513E02050080B05E0010101013C51E6
:1046B000010B0BE12150200B08E0010123AF03D0D7
:1046C0000101250702D00101252B9EAA0CD007016C
:1046D000BB2B0701BA51BA2BEA6A000FE96E0C0E28
:1046E000EA22AECFEFFFA19207014B07E552E5CFDB
:1046F000EAFFE5CFE9FFE5CFDAFF110001013CABAE
:1047000007D03C9B248A0601425102E0426B436B76
:1047100012000701E3B103D0129A12981200129806
:10472000E3A31288129AE3B3128A1200220E44EC19
:1047300075F0268E1200ABEF0AF097EC73F003E0F1
:1047400071EC74F006E01494010157A30ED01484A8
:104750000CD0149402013F5107E10101E251800B9A
:1047600003E13C51040B01E01484149614A4148654
:1047700014981450040B05E1B8EC1FF0000901E097
:1047800014881200E7C1E9FFE8C1EAFFEECF4BF061
:10479000EECF4CF0EECF4DF0EECF4EF0EFCF4FF02E
:1047A000E5C1E9FFE6C1EAFF4BC0EEFF4CC0EEFFFA
:1047B0004DC0EEFF4EC0EEFF4FC0EEFF120025ECE5
:1047C00073F0FD0EDBCFE7F1FE0EDBCFE8F1010168
:1047D0009A0EE56F010EE66FD5DFFB0EDBCFE7F13A
:1047E000FC0EDBCFE8F101019F0EE56F010EE66FD5
:1047F000C9DFEBEC2FF0D8A002D0010E01D0000EE3
:104800002AEF73F0E0EC79F00050E66E18ECFAF065
:10481000E552140EE66E77ECFAF0E5528CECFAF005
:1048200087ECFAF00009FCE1C450006E0050F80873
:1048300012E2C20410E0050EC25C0DE0090EC25C7B
:104840000AE00D0EC25C07E0110EC25C04E0390EF6
:10485000C25C01E00006020EE15C02E2E16AE552A0
:10486000E16E2AEF73F0D6EC79F00050DF6E020EA5
:104870004B6E870E4C6E010EA4EC7CF00150006E66
:10488000009E1BECE7F001AEF2D7E5522AEF73F081
:10489000D6EC79F00050DF6E2450100B12E100507E
:1048A000E66E7DEC04F0E552800B0BE00101450E55
:1048B000176F520E196F19C118F1200E1A6F040EDE
:1048C000016F2B8824A808D0FE0E4B6E880E4C6E0C
:1048D000010EA4EC7CF007D0DFCFE6FF7DEC04F006
:1048E000E552016EDF2A2BA802D0019E2B980150C1
:1048F000006E009E45ECE7F001AEE4D72498E55247
:104900002AEF73F008EC7BF004E2FE0EDB50300F70
:1049100004D0FE0EDB50410FF60F006E1BECE7F0EB
:104920002AEF73F008EC7BF004E2FE0EDB50300F50
:1049300004D0FE0EDB50410FF60F006E45ECE7F0A1
:104940002AEF73F025EC73F0ADEC77F0DBDFE55286
:10495000B2EC77F0D7DFE5522AEF73F025EC73F075
:10496000ADEC77F0DFDFE552B2EC77F0DBDFE5525C
:104970002AEF73F025EC73F0A1EC78F0020E010140
:10498000002790ECE6F0DF50006E050E0101005F9D
:1049900090ECE6F0030E0101005FE5522AEF73F0A0
:1049A00025EC73F0A1EC78F0FE0EDB50020F010154
:1049B000016FADECE6F0DF50006EFE0EDBCF01F1D3
:1049C000ADECE6F0E5522AEF73F000C05CF2ADEC1E
:1049D000E0F0FF0E005C01E046DF0101B18912004A
:1049E00000C05DF2BDECE0F0FF0E005C01E050DFC6
:1049F0000101B18B1200ADECE0F0FF0E005C01E0B4
:104A000032DF0101B18D640EA86F25961200BDEC56
:104A1000E0F0FF0E005C01E03BDF0101B18F640EAE
:104A2000A86F2596120025EC73F0E4EC77F0A0EC6B
:104A300074F0F8EC73F02AEF73F025EC73F0E4EC0B
:104A400077F015EC7AF0010EE66E41EC07F0E552D6
:104A5000E5522AEF73F025EC73F005EC6BF00101E1
:104A6000190EAA6FFC0EDBCFAEF1FD0EDBCFAFF15E
:104A7000FE0EDBCFB0F12AEF73F0830E0A6EE00E6C
:104A8000D6EC74F00A6A800E005C08E205EC6BF06C
:104A90000101190EAA6F0201E00EC76F120080EC2F
:104AA0007CF0DBCF4CF0800E4C1407E039EC7AF050
:104AB0004B6C4C1E000E4C2202D039EC7AF003EC09
:104AC0007CF02AEF73F025EC73F013A614D00601E6
:104AD00050B508D001013C9B2294060150855097A7
:104AE000248A2682298ABCBF299AFE0EDB5001E067
:104AF000297A8EEC3EF02AEF73F080EC7CF0DBAE8E
:104B000008D0DB50FF0DFE0EF3CFDBFF51EC77F04A
:104B100007D051EC77F0DB50FF0DFE0EF3CFDBFF3B
:104B2000DB502AEF73F0D6EC79F007017B5101E0FE
:104B300061D11E50400B01E05DD13350040B01E107
:104B400058D10101D05104E18450020B01E151D14F
:104B50000B0E9BEC74F00601BC6F18EC76F001E0D4
:104B6000A9D0140E0601E76EBC19E8AE02D0BC3520
:104B700003D0E750D880BC5502E2140EBC6FEC0E97
:104B8000E76EBC19E8AE02D0E73402D0E750BC5D56
:104B900002E2EC0EBC6FBE51E76EBC19E8AE02D06B
:104BA000BC3503D0E750D880BC5502E2BE2B0BD0F9
:104BB000BE51E76EBC19E8AE02D0E73402D0E75030
:104BC000BC5D03E2BE07BEC6BCF6200E4B6E4C6A4F
:104BD000C1C63FF0C2C640F0A8EC78F03FC0C0F6B6
:104BE000C0C64BF04C6A4BBE4C684B500601C15FCF
:104BF0004C50C25BBCC64BF04C6A4BBE4C684B5031
:104C0000C1274C50C223C0C6E6FF77DFE552016ED4
:104C1000010EE66E0E0E012404EC75F0020119512E
:104C200001E1E7D01CAA05D0BCC6E6FF2EEC71F06E
:104C3000E552E5EC75F02EE01350080B03E1040E8D
:104C400019152CE01A9EC6EC79F002E0000E01D096
:104C5000010E4B6E0101D05103E1CC51400B07E036
:104C6000D05103E0CB51040B02E0000E01D0010E45
:104C70004B1809E013A602D0E66A09D00601BC5120
:104C8000010125270BD013A605D0010EE66E1BDF10
:104C9000E55204D00601BC510101255F0601BC515B
:104CA00001E0A7D002011951320801E3A2D0320E6F
:104CB000196F9FD01B0EE66ED5EC13F0E552F3CFC3
:104CC000BCF6F4CFBDF6026A016A0601BC51E76E7C
:104CD000BD19E8AE02D0BD3503D0E750D880BD5530
:104CE00005E2BC51BD5D8DEC76F0026E0601BD5152
:104CF000E76EBC19E8AE02D0BC3503D0E750D880CF
:104D0000BC5505E2BD51BC5D8DEC76F0016E06012F
:104D1000BF51D880025402E202C0BFF6BE51D88013
:104D2000015402E201C0BEF6000EE76EBF19E8AE04
:104D300002D0BF3503D0E750D880BF5505E2010E41
:104D4000E66E0D0E04EC75F0010E0601E76EBF195C
:104D5000E8AE02D0BF3503D0E750D880BF5505E29A
:104D6000010EE66E0C0E04EC75F0020E0601E76E05
:104D7000BF19E8AE02D0BF3503D0E750D880BF5589
:104D800005E2010EE66E0B0E04EC75F0000E060156
:104D9000E76EBE19E8AE02D0BE3503D0E750D8802A
:104DA000BE5505E2010EE66E0F0E04EC75F0010E25
:104DB0000601E76EBE19E8AE02D0BE3503D0E7505B
:104DC000D880BE5505E2010EE66E100E04EC75F0BB
:104DD000020E0601E76EBE19E8AE02D0BE3503D062
:104DE000E750D880BE5505E2010EE66E110E04ECC8
:104DF00075F03394E5522AEF73F0E0EC79F0FC0E95
:104E0000DB506BE10201295168E10490FE0EDB509A
:104E1000140804E2140E46EC76F00480FE0EDBCF9C
:104E20004BF05951D8804B5403E2FE0EDBCF59F2C0
:104E300001012B51100B03E0050ED05D05E104507C
:104E4000010B02E0FE0EDB2A010E68C1DBFF050E3E
:104E5000D05D02E1010EDB6A010EDB50280803E29F
:104E6000DE52280EDD6E050E31EC74F0010E40C0EE
:104E7000DBFFDF6A150EDF5C22E2006AFE0EDB500C
:104E800004E0FE0EDB50DF5C13E301012B51100B3D
:104E900007E0050ED05D04E002015951DF5C08E037
:104EA00001016851040806E2010EDB50DF5C02E1FB
:104EB000010E006E005028EC76F0DF2ADBD714508C
:104EC000010B6BE00201205168E10101D05103E0C8
:104ED000030ED05D62E1338460D0FC0EDB0431E16F
:104EE0000201295106E0FD0EDB5003E12350400B87
:104EF00057E1FE0EDB50080803E2080E46EC76F0A0
:104F0000FD0EDB500C0805E20C0EF36EFD0EF3CF28
:104F1000DBFFE9EC75F0150EDF5C3FE2FE0EDB50C7
:104F200004E0FE0EDB50DF5C07E3090EDF5C07E305
:104F3000FD0EDB50DF5C03E2010E28EC76F0DF2A89
:104F4000EAD7FC0EDB50020828E1FE0EDB50080811
:104F500003E2080E46EC76F0FD0EDB500C0805E28D
:104F60000B0EF36EFD0EF3CFDBFFE9EC75F0150EC3
:104F7000DF5C13E2FE0EDB5004E0FE0EDB50DF5C74
:104F800007E3090EDF5C07E3FD0EDB50DF5C03E2A5
:104F9000010E28EC76F0DF2AEAD7FE0EDBCF0AF20C
:104FA000020EE15C02E2E16AE552E16E2AEF73F083
:104FB0000101D1512FEC76F01EEC75F00150080D77
:104FC0004B50F3240A01DF6F4C50F420E06F1200C5
:104FD0000101C551C05D0CE1C651C15D09E1C75178
:104FE000C25D06E1C851C35D03E1C951C45D01E082
:104FF000000C010C0101D151D05D01E0000CD05139
:105000000BE1CC51400B01E0010E4B6ED951400B2E
:1050100001E0010E4B5C2DE0030ED05D23E1D85181
:105020003CEC74F00B5C1EE118EC76F00CE0010136
:10503000CC51040B01E0010E4C6ED951040B01E080
:10504000010E4C5C16E018EC76F00CE10101CB513E
:10505000040B01E0010E4D6ED851040B01E0010E6E
:105060004D5C07E00101D05103E0030ED05D01E18A
:10507000000C010CADDF000903E0BCDF000901E119
:10508000000C010CF7DF000932E0E9EC73F001E1FC
:10509000010CD1512FEC76F0080EE66EE66AD15184
:1050A0006BEC75F056EC79F00150EDEC73F0D051EB
:1050B000100DF3CF51F0F4CF52F02A0E51260A0E04
:1050C00052220701D651080D5150F3244F6E525011
:1050D000F420506E4FC0E6FF50C0E6FF6CECF6F0D7
:1050E000536E060EE15E5350000901E1010C000C05
:1050F0002CC161F10DC10EF11BB20AD0C0C1C5F1C6
:10510000C1C1C6F1C2C1C7F1C3C1C8F1C4C1C9F1AF
:10511000D0C1D1F135AC15D0010139A306D0DA9355
:10512000CDB3DA83DA95CDB5DA85D99DCCBDD98DED
:10513000D995CCB5D985D895CBB5D885EEEC7AF094
:1051400018D00101D15103E1D99DCCBDD98D030EF9
:10515000D15D0FE1EEEC7AF018EC76F006E001019B
:10516000D995CCA506D0D98504D00101D895CBB569
:10517000D88535AC0DD0500EE66EE66A2A0EE66E86
:105180000A0EE66E7A0EE66E0A0E63EC75F00FD02C
:10519000050ED05D0CE0100EE66EE66A99EC75F037
:1051A000D1516BEC75F056EC79F0CAEC7BF0050E42
:1051B0000101D15D08E0D151EA6ACF0FE96E0A0E14
:1051C000EA22D6C7EFFF120061C12CF10EC10DF12A
:1051D000C5C1C0F1C6C1C1F1C7C1C2F1C8C1C3F1E7
:1051E000C9C1C4F1D1C1D0F135AC08D017EC78F009
:1051F0002A0EE66E0A0E63EC75F011D0E9EC73F03E
:105200000EE0100EE66EE66A1EEC75F05CEC7AF0CD
:10521000D0516BEC75F035EC79F0CAEC7BF0E9EC31
:1052200073F004E0BCEC75F0D6C7EFFF120025EC7C
:1052300073F028DF000913E1A3EC12F0FE0EDB503F
:1052400002E156DF01D0C0DF5BEC79F0258A1FACAC
:1052500004D002010983098102D0020106832AEFEA
:1052600073F0A3EC12F001012C51615D0EE1C0510D
:105270000CE0C00503E13C0EC15D07E3C55105E04C
:10528000C50518E13C0EC65D15E226EC79F0358CBB
:1052900014D8359C3CEC12F01D8A26EC79F01D9A4E
:1052A000198417EC79F01994EBEC1FF00201010E50
:1052B000236F120002D83CEF12F061C102F00EC160
:1052C00003F0C5C1B7F2C6C1B8F2C7C1B9F2C8C1CF
:1052D000BAF2C9C1BBF2D1C100F0D8C1DCF1D9C169
:1052E000DDF1DAC1DEF135AC08D017EC78F0540E00
:1052F000E66E060E63EC75F011D0050E005C0EE054
:10530000100EE66EE66A01011EEC75F05CEC7AF0B8
:10531000540EE66E060EE66EABEC78F0016A050EF2
:10532000005C03E000502FEC76F0E2DE02C02CF1CE
:1053300003C00DF1B7C2C0F1B8C2C1F1B9C2C2F128
:10534000BAC2C3F1BBC2C4F100C0D0F135AC21D0A8
:10535000010139A30ED0CD93DEB3CD83CD95DEB55B
:10536000CD851396CDB313861394CDB513841BEC62
:10537000A5F00101CC9DDDBDCC8DCC95DDB5CC85F6
:10538000CB95DCB5CB85DC513CEC74F0A3EC75F02F
:105390001BD00101D05103E1CC9DDDBDCC8D030EAE
:1053A000D05D12E1DC513CEC74F0A3EC75F018EC2C
:1053B00076F006E00101CC95DDA506D0CC8504D0C1
:1053C0000101CB95DCB5CB8535AC09D0500EB2ECE4
:1053D00078F02A0EE66E0A0E63EC75F00AD0050E20
:1053E000005C07E0100EB2EC78F099EC75F0ABECD5
:1053F00078F001C0D6F7E9EC73F004E0BCEC75F08E
:1054000001C0EFFF04903CB104803C913CB33C816F
:105410003C9304B03C83139C3CB1138C139E3CB36F
:10542000138E5BEC79F0258A14DB1FAC06D00201E9
:105430000987098509830981120002010683120088
:1054400027EC7AF00AE0076A010163958FEC1CF003
:10545000010E076E01015D8509D0010E076E010185
:105460005D958FEC1CF0076A010163858FEC1CF0E1
:105470002AEF73F0370E005C02E2370E006E005028
:105480009F0802E29F0E006E630E005C08E2370E7A
:10549000005CE8244B6E090EA2EC73F005D0630E9D
:1054A000005C15EC7CF0090F006E0201F25102E085
:1054B000030E00260050150802E2150E006E1200C1
:1054C00039EC7BF0020120510EE12150010B0BE180
:1054D000235109E13350200B06E12850200B03E053
:1054E00031A003D03190000E72D0FE0EDB5002E0EE
:1054F000990E01D00A0E9BEC74F03AEC79F08C0E08
:1055000091EC75F00201F25103E0790E91EC75F027
:105510002B512CE1020EDB50CDEC74F027E30A0E88
:105520009BEC74F04B6E020EDB504B5C1FE312AE33
:1055300010D0129EDFEC1EF00201068D090ED5EC94
:1055400073F0E7EC1EF055ECF1F00201780E2B6FD2
:105550000DD00201F25107E107010A9355ECF1F079
:105560002FEC50F012840201FA0EF26F010EDB50A4
:10557000006E00509F0802E29F0E006EB2EC79F0C0
:1055800005011851070DB9EC78F0030E0F0B03E07D
:1055900044EC79F0FDE14BC018F56CDF0050DF6E94
:1055A00000C0C9F7090E016E01012BB901061450A4
:1055B000010B06E00150D880005402E20150006E59
:1055C000E66AE66A0050E66EDCEC75F0DF504B6E82
:1055D000030EE15C02E2E16AE552E16E4B502AEF14
:1055E00073F025EC73F0016A0A0E015C19E2FE0EFD
:1055F000DB50010B06E0210E0124E0EC75F0165C97
:105600000AE0FE0EDB50020B09E02B0E0124E0EC59
:1056100075F0165C03E101500D6E02D0012AE4D74B
:105620002AEF73F025EC73F0800E0D6E18AE17D0D4
:10563000189E1850010B03E11850100B10E0100ECB
:105640000D6E15EC7AF0CDDFE5522C0E165C02E102
:10565000200E0D6E0B0E165C02E1400E0D6E2AEF51
:1056600073F025EC73F095EC76F015EC7AF080ECA5
:105670007AF0030EEB500101A46FA451640DDFEC2E
:1056800073F023EC7CF05C0F8CEC75F0006E73EC27
:1056900073F0020EEB50C0EC78F0B2EC79F001013F
:1056A0004D504B5CD46F4E504C58D56F2AA60BD042
:1056B0009A51C0EC78F00101D4514B5C0F6ED5517A
:1056C0004C58106E06D09A51106AD4250F6ED551E1
:1056D0001022640E4B6E4C6AAAEC7CF03FC0A4F121
:1056E0003BC09AF12AEF73F025EC73F095EC76F05D
:1056F000DB50AAEC74F0030E97EC7CF00101A45D82
:1057000002E0000E11D0FE0EDB50AAEC74F0020E87
:1057100097EC7CF09A5D006E00BE006C040E005C9D
:1057200002E2010E01D0000E2AEF73F050EC7BF084
:10573000920E4B1811E14C500FE1006AE5EC24F099
:10574000B50E006EF0EC24F00101A86B2286020178
:105750007B6B6C6B299E082A50EC7BF0930E4B18E8
:105760005CE14C505AE1010EE66E5CDFE5520A0E38
:105770000D5C32E202017B51050833E36C510208F3
:1057800030E37B2B29BE6C2B010E016E070E015CF2
:1057900013E2012848EC74F0EF50006E060E015C35
:1057A00005E1800E010116150D10006E99EC7BF0DD
:1057B00000C0EFFF012AEAD70101169F37AD2DD0B7
:1057C0000D5002E1540E02D0300E0D24006E800EFA
:1057D0000010C6EC77F010D0200E0D5C12E129AE5F
:1057E00002D0268E1AD0298E0101168FD20EC6EC59
:1057F00077F0010137AD11D00501930E4F6F1E0EEA
:105800000BD0400E0D5C04E1980E086E1B8805D08D
:10581000100E0D5C02E19A0E086E50EC7BF0980EB3
:105820004B1801E07FD04C5001E07CD0010E016E9E
:10583000070E015C0DE299EC7BF0EF9E99EC7BF09A
:10584000EF500E0803E199EC7BF0EF6A012AF0D7E4
:1058500010C1A4F10A0E01011103F35012259A6F31
:105860000A0E1303F35014259B6F0A0E1503F3CF92
:105870009CF19E6B9EC19DF1040E02017B5D0DE2C9
:105880006C510BE113C1A4F10A0E01011403F35092
:1058900015259A6F9C6B9CC19BF102016C0508E178
:1058A00012C1A4F19BC19AF19CC19BF101019C6BB7
:1058B000020E02016C5D0EE111C1A4F10A0E01019C
:1058C0001203F35013259A6F0A0E1403F350152593
:1058D0009B6F9C6B9A0E086EAAEC0BF0006E00504A
:1058E00013E10101A45103E19A51370802E2268E27
:1058F00012005AEC77F00A0E005C06E10101DF515C
:10590000010B02E0C8EF07F000C02CF117EC79F0B2
:1059100088EC04F0EBEC1FF0000E0201B06FB16BED
:105920008D6F8E6B50EC7BF09A0E4B1808E14C504B
:1059300006E10101B19BB19903D80C0E086E12006B
:1059400088D86DDB2682248A120041C2A3F142C2AC
:10595000A2F143C2A1F10101A06B9F6B20A402D070
:10596000C7EF2FF0EBEF2FF004902D50100B01E05C
:105970000480FAECF1F02D50100B01E0010E4B6E9B
:105980000450010B4B5C02E0FAEC76F01200D6EC0E
:1059900079F0DF6A01018EA715D0FE0EDB5008E01A
:1059A000FD0EDB5005E1DF68CBA102D0010EDF6EFA
:1059B000FE0EDB5007E1FD0EDB5004E0010EDF6E52
:1059C000CBB1DF68DF5023E027EC75F0A36BA3C1F8
:1059D000A0F1A3C19FF172EC7BF0C6EC79F002E07C
:1059E000000E01D0010E4B6EDF0402E0000E01D06C
:1059F000010E4B1802E0CBDA01D0EDDA88EC04F0AE
:105A00001FAC03D00201098102D002010683E552D6
:105A10002AEF73F00101A36BA26BA16B02019B51F2
:105A2000E8244B6E640E17EC7BF05CECFAF03CC0A3
:105A3000A0F1320EB4EC7CF09BC240F05CECFAF0CA
:105A400040C09FF102019CA102D0C7EF2FF0EBEF05
:105A50002FF008AE6ED02C50400B03E02D50200BE1
:105A600031E0800E0101C01505E1C0510CE11F0EAF
:105A7000C15D09E2C06B1F0EC16FC46BC4C1C3F12D
:105A8000C4C1C2F11FD0100E2C5D1CE2360E006E98
:105A90000050C05D03E300C0C0F10DD0200EC05D1A
:105AA00011E32C0EC05D0EE2260EC05D02E2200E58
:105AB00001D02C0EC06FC46BC4C1C3F1C4C1C2F10C
:105AC000C4C1C1F12C50400B03E02D50200B31E13B
:105AD000800E0101C51505E1C5510CE11F0EC65D23
:105AE00009E2C56B1F0EC66FC96BC9C1C8F1C9C138
:105AF000C7F11FD0100E615D1CE2360E006E005023
:105B0000C55D03E300C0C5F10DD0200EC55D11E3F6
:105B10002C0EC55D0EE2260EC55D02E2200E01D000
:105B20002C0EC56FC96BC9C1C8F1C9C1C7F1C9C1C4
:105B3000C6F12C50400B03E02D50200B1DE02150EE
:105B4000400B03E11350080B0FE12150400B12E012
:105B50002050020B03E11350040B06E12050020B0E
:105B600009E01350080B06E027EC75F0EEDEA0EC20
:105B700076F002D0ABEC76F02C50400B03E02D50C9
:105B8000200B16E12050020B11E01350040B0EE025
:105B9000B6EC76F0DADE9AC1BBF19BC1BCF19CC1D8
:105BA000BDF19DC1BEF19EC1BFF102D0C1EC76F046
:105BB0002050020B18E102019C51010B03E19C51A2
:105BC000020B11E0E9EC73F006E02150800B0BE0D2
:105BD000050E995D08E12150400B05E032EC75F0AF
:105BE00019DFA0EC76F001013CA9B4D0B6C1ECF706
:105BF0000701ED6BEE6BEF6B1FEC78F0ECC73DF03F
:105C0000EDC73EF0EEC73FF0EFC740F0F3ECF7F022
:105C100039C0ECF73AC0EDF73BC0EEF73CC0EFF708
:105C2000B7C13DF0D0EC7BF07FEC74F0B8C13DF033
:105C300069EC78F0640E426E436A7FEC74F0B9C18F
:105C40003DF069EC78F00A0E426E436A7FEC74F026
:105C50000101BA510701EC27000EED23EE23EF23DB
:105C6000BBC1F0F7F16BF26BF36B1FEC78F0F0C790
:105C70003DF0F1C73EF0F2C73FF0F3C740F0F3EC60
:105C8000F7F039C0F0F73AC0F1F73BC0F2F73CC08B
:105C9000F3F7BCC13DF0D0EC7BF08DEC74F0BDC1EE
:105CA0003DF069EC78F0640E426E436A8DEC74F05E
:105CB000BEC13DF069EC78F00A0E426E436A8DEC8D
:105CC00074F00101BF510701F027000EF123F22308
:105CD000F323EC51F05FED51F15BEE51F25BEF51CC
:105CE000F35B049C1F50200B01E0048CD880F3511F
:105CF000FF0A08E6680EF05DC50EF159FF0EF25975
:105D0000FF0EF35919E3F335000EF31909E6D880B5
:105D1000980EF0553A0EF155000EF255000EF3555F
:105D20000BE3F0C70FF0F1C710F0D1EC74F0A50E43
:105D300038EC73F01F8A01D01F9A0450400B01E029
:105D4000010E4B6E1F50200B01E0010E4B5C02E078
:105D500035EC7BF02CACADD02CC100F02C50400BBE
:105D600005E02D50200B02E161C100F02CC161F172
:105D7000800E081401E19DD0100E005C01E399D063
:105D80002DBA0DD0CCEC76F0C5C19FF1C6C1A0F103
:105D9000C7C1A1F1C8C1A2F1C9C1A3F10CD032ECB5
:105DA00075F0C0C19FF1C1C1A0F1C2C1A1F1C3C1D1
:105DB000A2F1C4C1A3F15AEC77F02D50200B04E0FE
:105DC000005001012C5D07E12D50200B33E1005004
:105DD0000101615D2FE000C00EF100C00DF100C0B7
:105DE00061F100C02CF12CC1CFF120EC76F02CC178
:105DF000E6FF79EC76F0056E2DAA06D0050EE66E6C
:105E000005245FEC79F005D0050EE66E055064ECD4
:105E100079F03DEC73F00E0E0524D6EC74F0010120
:105E2000CE9B00BACE8B0A6AB7DB21820201010E3B
:105E3000236F01D099DD0701E6510101C05D04E047
:105E400080EC0CF0C0C1E6F701012C5132E12C507E
:105E5000080B2FE0020E3B5D2CE1F7EC75F004E03F
:105E60005DEC78F0E806FCE10701EA510F1802E169
:105E7000EB5110181EE0006A5A0E0F1807E110507F
:105E800005E1590EEA1901E1EB510AE0590E0F182C
:105E900008E1105006E15A0EEA1903E1EB5101E165
:105EA000002A0FC0EAF710C0EBF70050E66E02D8E8
:105EB000E552120025EC73F001012C5166E12C50E3
:105EC000080B63E0FE0EDB5003E1020E3B5D5DE17B
:105ED000F7EC75F004E05DEC78F0E806FCE10FC04B
:105EE000EAF710C0EBF7190EA2EC79F003E20368B1
:105EF00002681FD0410EA2EC79F017E2AAEC7AF00A
:105F0000190E4B5E000E4C5A4B50016E2AEC7AF083
:105F10000800F550026E2AEC7AF0F62A000EF722FD
:105F2000F8220800F550036E04D069C302F06AC37A
:105F300003F0FE0EDB5007E10701E751025C03E1CD
:105F4000E851035C22E002C0E7F703C0E8F7410E26
:105F5000A2EC79F012E2010EE66EE66A0350E66EFC
:105F60000250E66E94ECD9F05FEC7CF0E5520B0E3B
:105F7000E66E63ECD9F0E55205D0FE0EDB5002E090
:105F8000C7EC78F00A0E47EC79F02AEF73F00101C4
:105F9000A3519E279E51090803E20A0E9E5F9D2B86
:105FA000A2519D279D51090803E20A0E9D5F9C2B7B
:105FB000A1519C279C51630803E2640E9C5F9B2BBC
:105FC000A0519B279B51630803E2640E9B5F9A2BB1
:105FD0009F519A2712000101A3519E5F9E510A080A
:105FE00003E20A0E9E279D07A2519D5F9D510A085C
:105FF00003E20A0E9D279C07A1519C5F9C516408F7
:1060000003E2640E9C279B07A0519B5F9B51640891
:1060100003E2640E9B279A079F519A5F12004FEC90
:106020007AF02CBC04D0076A15D8309E11D02DAA66
:1060300007D02150400B0AE02050020B09E106D0A6
:106040002150400B05E02050020B02E0076A02D805
:1060500053EF7AF02050020B06E02150400B03E092
:10606000CCEC76F002D032EC75F00101A36BA3C149
:10607000A2F1A3C1A1F1A3C1A0F1A3C19FF121503D
:10608000400B09E1D05107E172EC7BF087EC0EF098
:10609000000947E044D02150400B12E1D00503E055
:1060A000020ED05D0DE128EC7CF002E6B7EC77F053
:1060B00007E201010F0EA16F020ED05D30E131D079
:1060C000CAEC79F00CE00101090EA16F010EA26F7C
:1060D000050EA36F87EC0EF0000921E122D02150BC
:1060E000400B0BE1E0EC77F008E001010A0EA16F34
:1060F00087EC0EF0000913E114D02150400B12E19F
:10610000E9EC73F003E0040ED05D0CE1010EA06F2A
:106110000A0EA16F040ED05D04E0E1AF02D05BDF98
:1061200001D035DF96EC79F011E02150400B0EE103
:10613000050ED05D0BE0040ED05D08E09F6BA06BF8
:10614000500EA16FA36BA3C1A2F145DF010158A9B5
:1061500043D058AB64D0F6C70FF0F7C710F0260E47
:10616000D8800F54020E105406E20480260E0F5EF3
:10617000020E105A06D00490260ED8800F56020E3A
:1061800010569B514B6E4C6A9A51640DF3504B2440
:10619000D46FF4504C20D56FD4C14FF0D5C150F01E
:1061A0000FEC74F039C03DF03AC03EF03BC03FF018
:1061B0003CC040F0880E426E130E436E446A456A3E
:1061C00031ECF9F03DC00FF03EC010F051EC75F02D
:1061D00004A024D000DF23D09AC100F0000405E120
:1061E0009B51310802E2020E006E030E005C05E1D5
:1061F0009B51310802E2040E006EB2EC79F04AECD9
:1062000078F0D4C23FF0D5C240F05CEC73F013ECF0
:1062100075F01E0ED6EC7BF051EC75F0B8DEE5ECB7
:1062200075F004E1210E0101B55D19E00601F051A0
:1062300001019C5D14E10601EF5101019B5D0FE13D
:106240000601F15101019D5D0AE10601F2510101D2
:106250009E5D05E10601EE5101019A5D0CE09AC1D7
:10626000EEF69BC1EFF69CC1F0F69DC1F1F69EC122
:10627000F2F623ECE8F01200D9CFE6FFE1CFD9FF28
:10628000B6C19AF1B7C19BF1B8C19CF1B9C19DF1FA
:10629000BAC19EF10101A46BFE0EDB500A0807E2B1
:1062A0002A96FE0EDBCFE6FF31EC2BF0E552010122
:1062B000006B800E01011415036E800E0101111593
:1062C000026E010EEA6E9A5105D89B5103D89C517B
:1062D00001D814D0076B066F0A0E065DD8A003D054
:1062E000066F072BF9D700510F0FE96E0751EF6EBC
:1062F000E92A0651EF6E002B002B000C9DC115F111
:106300009EC116F10101A45107E10A0E01019A5D37
:1063100003E20101100E0F6F0701E3BB03D001017F
:10632000100E166F0701E3AD05D00101100E156FB9
:1063300015C116F11EBC03D00101118F03D002500C
:10634000010111130101148F0101A45109081AE27E
:106350000201375117E0ADECE0F00101020E006FD1
:106360009AC100F090ECE6F0A4C100F00101006BCE
:1063700090ECE6F0010EE66EE66AE6EC07F0E55218
:10638000E55223D00101A4511FE007010701E351A9
:10639000200B1AE1298C15C116F114C115F113C196
:1063A00014F112C113F111C112F110C111F10FC199
:1063B00010F10A0E4B6E4BC045F0A4C140F05CECEE
:1063C000FAF03CC00FF101D0299CE552E7CFD9FF8C
:1063D0001200D9CFE6FFE1CFD9FF020EE126010E70
:1063E000A4C1DBFF61C1DFFF0101D151EA6ADD0F0A
:1063F000E96E070EEA22EFCFE4F7BBC19AF1BCC108
:106400009BF1BDC19CF1BEC19DF1BFC19EF10101D7
:10641000A46BDF500A0806E22A96DFCFE6FF31ECD4
:106420002BF0E5520101016B800E01011C15026E7B
:10643000010EEA6E9A5105D89B5103D89C5101D8A0
:1064400016D0076B066F0A0E065DD8A003D0066F44
:10645000072BF9D70151170FE96E0751300FEF6E77
:10646000E92A0651300FEF6E012B012B000C300E84
:1064700001019D2501011D6F0101A45107E10A0ED3
:1064800001019A5D03E20101200E176F0701E4ADDF
:1064900003D00101200E1D6F0101198F01011C8F16
:1064A0000101A4511DE007010701E451200B18E18F
:1064B0001CC11DF11BC11CF11AC11BF119C11AF13C
:1064C00018C119F117C118F10A0E4B6E4BC045F0F7
:1064D000A4C140F05CECFAF03C50300F0101176FA2
:1064E000A4C1A5F1010EDBCFA4F1020EE15C02E232
:1064F000E16AE552E16EE552E7CFD9FF1200D6EC32
:1065000079F0830E0A6E0A0EE66E01010D03F35058
:10651000E66E610EE66E020E3DEC73F0DE0ED6EC1A
:1065200074F00050DF6EFE0ED6EC74F00A6A0101C2
:10653000E19D2F9EB90E005C05E1FF0E0201615D39
:1065400001E02F8EA30EDF5C02E10101E18DE55237
:106550002AEF73F08C0E0201A01909E10A0EA119AD
:1065600006E18C0EA21902E10A0EA31907E0800EC3
:10657000A11504E1800EA31501E1000C010C02013C
:10658000A45102E1A55107E0FF0EA45D04E0FF0E57
:10659000A55D01E0000C010C4FEC7AF007504CE1D6
:1065A0001950010B49E10DC1E6FF66EC57F0E552C9
:1065B000D1DF000902E006EC77F00DC1E6FF82ECC6
:1065C00057F0E552DCDF000903E00201A46BA56B84
:1065D0007CEC14F094DF01015751080B03E12C51BE
:1065E000090809E2FF0E02019D5D02E1320E9D6F76
:1065F0009DC249F108D0FF0E8D5D03E1320E8D6F13
:1066000002D08DC149F15BEC3FF0F0EC76F02B84C9
:10661000C1EC1FF005EC1CF02C50080B0DE0010143
:10662000E251040B09E12C5105E1010EE66E42DC5A
:10663000E55202D0C7EC78F05BEC79F053EF7AF0DA
:10664000D6EC79F0FD0EDB50100DF350DF6E010E2D
:106650000A6E0201680EAA6FFD0EDB500A080AE2FC
:10666000020E0A6E690EAA6FFD0EDB50F00F100DC0
:10667000F350DF6ECEEC79F002E0CBEC7AF0DF5035
:10668000E5522AEF73F002019A5103E09A51320861
:1066900002E20D0E9A6F9B5156EC74F007E24B50DC
:1066A000FA08000E4C5402E21E0E9B6F9CBF9C6BBE
:1066B000A6510E0803E2A66B0101CC9B1200E0EC90
:1066C00079F0CEEC79F01BE0CBEC7AF00F0EE0EC39
:1066D0007AF00A0E005C07E10101DF51010B03E0D3
:1066E0000A6A000ED7D100C02CF101018B51100BAA
:1066F00006E00A0E58EC73F002E2FE0EDB682CC1D5
:106700000DF10201796B0101E2952C510A0821E299
:10671000100E2C5D8CEC7CF014E023EC7CF001017D
:106720000D6F73EC73F0EF380F0B0201796F73ECA0
:1067300073F0090E97EC7CF0800B0BE00101E28511
:1067400008D0FE0EDB680101090E0D6F0DC12CF1A2
:10675000268E0101E2A507D007011397140EE66EFD
:106760007AECD9F006D007011387140EE66E63ECBD
:10677000D9F0E55207010B890101E2A502D007011A
:106780000B9954ECF1F027EC74F0100EE8EC7AF071
:106790000F0E0101CA15D06FCA390F0BD16FD1513D
:1067A000060802E2D0C1D1F1D00501E1CB91020E81
:1067B000D05D01E1CB81CB513CEC74F00B6E2CC170
:1067C00061F10DC10EF161C10EF161510A0815E2CE
:1067D000100E615D8CEC7CF005E023EC7CF0010197
:1067E0000E6F08D0FE0EDB680101090E0E6F0EC1A0
:1067F00061F1268E61C100F006D0C6C1E6FFC5C1B9
:10680000E6FF2CEC7CF000500101615D03E12C51AE
:10681000615D13E061C1E6FF79EC76F0DF6E050E95
:10682000E66EDF245FEC79F03DEC73F00A0EE0ECED
:106830007AF000380F0B0101D16F040EE66E0B0EDB
:10684000DF24E66ED80EE66E010E3DEC73F027EC09
:1068500074F0CEEC79F003E1AAC20AF002D0100E77
:10686000DF26100E9BEC7CF06BEC7BF0CEEC79F02D
:1068700057E02CC1E6FF79EC76F0DF6E0B0EE0EC12
:106880007AF04DEC75F009E01F0ECB17E00E001406
:10689000CB13CB513CEC74F00B6E0C0EE0EC7AF0A9
:1068A000440E0101CC17BB0E0014CC1350EC7CF04D
:1068B000470E0101CD17B80E0014CD1350EC7CF03B
:1068C0009E0E0101CE17610E0014CE13AAC20AF06B
:1068D0000A0EE66E030EDF24E66E9D0EE66E020ED5
:1068E0003DEC73F061C1E6FF79EC76F0DF6E0C0EE3
:1068F000E0EC7AF0440E0101D917BB0E0014D91355
:1069000050EC7CF0470E0101DA17B80E0014DA13D0
:1069100050EC7CF09E0E0101DB17610E0014DB13BE
:106920000A6AC0C119F5C1C11AF5C2C11BF5C3C1BC
:106930001CF5C4C11DF5C5C11EF5C6C11FF5C7C1F3
:1069400020F5C8C121F5C9C122F519B42DD0139481
:106950001396139A209201013951020B1CE04BEC63
:1069600076F019E10101CD51010B04E008EC9DF036
:10697000000911E10101CD51010B05E02C51615DD0
:1069800002E1138A20821396CDB313861394CDA50A
:1069900009D0138407D07FEC78F00101DA95DA93FF
:1069A000CD95CD931BECA5F001012C510A0819E2FD
:1069B0005C0E0D251EEC7CF00101C05D016E01AE88
:1069C00003D0C051005C016E015003080AE2050EBD
:1069D000EBEC77F0C00EE66E010EADEC73F000C08C
:1069E000C0F1010161510A0819E25C0E0E251EEC8E
:1069F0007CF00101C55D026E02AE03D0C551005CA2
:106A0000026E025003080AE2050EEBEC77F0C50EA9
:106A1000E66E010EADEC73F000C0C5F19EEC1DF00A
:106A200089EC23F09DEC23F018EC0CF0139C010191
:106A30003CB1138C139E3CB3138ECBEC60F01398D7
:106A400001013CB91388E7EC1EF02CB602D001011D
:106A5000CC9F12900101CCBF12801292CCAF128257
:106A600027EC08F0A7EC4BF062EC4BF00A6A01014E
:106A700038A702D0C1EC45F0ABEC76F0C1EC76F073
:106A80008BDD0101256B1EBC04D00701C86B20EC17
:106A900076F0010EA6EC79F002E2E16AE552E16ED1
:106AA0004B502AEF73F0D6EC79F00B0E01012C5D00
:106AB0000FE2C1C1E6FFC0C1E6FF2CEC7CF0005044
:106AC00001012C5D05E00701020E58EC7AF07DD043
:106AD0002CC161F10A0E2C5D02E249C18DF127EC57
:106AE00074F0DFEC1EF00101CC9F12B0CC8F39A303
:106AF0000DD0F80ECD17CD9120B2CD81CD9313B628
:106B0000CD83CD9513B4CD8573EC3EF02CC1CFF180
:106B10007AEC7BF0050E64EC79F09BEC7CF043ECB6
:106B200073F00A0EDF24016E0101D139F00BD01190
:106B30006DEC78F0050EE66ECB0EE66E010EE66E9D
:106B40000B0EDF2497EC7AF02CC161F1050E5FEC9F
:106B500079F0E66E050EDF2497EC7AF01DBA28D0A6
:106B600027EC74F001015751080B03E12C5109087F
:106B700002E249C19DF23BECD9F00101CC51800BFE
:106B800001E0010EF7EC77F0CEEC79F003E1AAC258
:106B90000AF002D0100EDF26100EE66E9A0EE66E98
:106BA000020E9BEC7CF043EC73F00A6AA3EC12F04B
:106BB000010138A705D0010EE66EE2EC45F0E55282
:106BC0000A6ADCEC7BF002011F6BE5522AEF73F0DE
:106BD000D6EC79F00F0EDF6E53EC76F008E02D5016
:106BE000400B05E12D50800B02E11F0EDF6EF40E0D
:106BF00006010017F00E0517DF500617E5522AEFC1
:106C000073F006010691009501910299019914997A
:106C1000139904990391120080EC7CF0DBCFE6FF1E
:106C200062EC10F0E552E71803E00601058502D09A
:106C30000601058701013DA502D006010689010173
:106C40008BA102D00601068D2AEF73F01A9E005028
:106C5000050A01E173D0010A5BE0070A2AE0010A94
:106C600023E0030A1FE0010A01E012000601058388
:106C7000C6EC79F002E0000E01D0010E4B6E01016E
:106C8000CC51400B01E0010E4B1802E006010581DA
:106C90000601EA5101E0068B01018FAD60D00601CB
:106CA000068D1200E66A02D0010EE66EB5DFE552EF
:106CB000120006010081C6EC79F002E0000E01D05E
:106CC000010E10EC77F002E0060105810B5003E0A5
:106CD000030E0B5C02E106010571BAEC79F002E0EB
:106CE0000601068B33A00ED0C6EC79F002E0000E50
:106CF00001D0010E10EC77F003E00601058702D009
:106D00000601058501013DA72AD00601068912006A
:106D1000060100830101CEA722D0CEA303D0060135
:106D2000058702D00601058501018F51080B03E19B
:106D300002013E5114E00601068B12000601008795
:106D400002019CA502D00601068B02019CA102D083
:106D50000601068D02019CA302D00601068F1200D7
:106D6000800E081406E02150010B03E1D0C100F0B1
:106D700003D0A0EC1EF0006E2BDF26EF36F01200E1
:106D800025EC73F04DEC75F00DE10B0403E0020E01
:106D90000B5C04E1CC51040B1CE10ED0CB51040B75
:106DA0000BE017D0D0050AE128EC7CF002E6B7EC46
:106DB00077F002E2420E24D0450E22D0020ED05DC2
:106DC0000AE128EC7CF002E6B7EC77F002E2400E34
:106DD00017D0440E15D0050ED05D07E1E151800BB0
:106DE00002E0480E0DD0470E0BD0040ED05D02E13C
:106DF000460E06D0CC51400B02E1430E01D0410EAD
:106E000055EC73F01CEC76F0030E005C12E10B0401
:106E100003E0020E0B5C05E10101CC51040B05E11E
:106E200006D00101CB51040B02E0540E1CD0550ECC
:106E30001AD0000402E1520E16D0020E005C02E1EC
:106E4000500E11D0050E005C02E1570E0CD0040E5E
:106E5000005C02E1560E07D00101CC51400B02E16B
:106E6000530E01D0510E55EC73F02AEF73F039EC4C
:106E70007BF0E9EC73F011E12B50020B01E0010E05
:106E8000E66ED950010FE96EDACFEAFFE552E7501E
:106E9000EE6EED6A2B922DEC15F034BA4BD0075004
:106EA00002E134EC0EF02150800B15E11550100B6F
:106EB00012E01550200B0FE10101D05109E0030E43
:106EC000D05D06E0050ED05D03E053EC76F003E004
:106ED0001598D3EC4CF02150800B0AE11550200B93
:106EE00007E0E9EC73F004E1159A1598D3EC4CF047
:106EF0004DEC75F003E0050ED05D01E1CE9D1490E0
:106F0000D05103E114908BB51480030ED05D05E1E0
:106F10000B5003E014908FB51480149A14A0148AB7
:106F200026EC0BF0075004E1CBEC60F063EC17F0BB
:106F30009DEC23F026820FEC30F0010EE66E20DF90
:106F4000E5527DEC15F05FEC1CF034BA6ED0D5CA7A
:106F5000E6FFAB0E4FEC73F075EC17F0D3EC4CF092
:106F600068EC0EF0EDEC1DF02EEC1DF029B25DD0BA
:106F70001D9835922550010B05E12850200B02E0A9
:106F80009FEC07F00F6A106AE9EC73F003E0040E5F
:106F9000D05D04E1100E0F6E270E05D0CEA104D0F7
:106FA000400E0F6E1F0E106ED1EC74F0A40E38EC74
:106FB00073F001013951040B05E1050ED05D02E0CB
:106FC000000E01D0010E000902E0840E01D0820EF5
:106FD00055EC73F0E9EC73F003E0050ED15D02E1CE
:106FE000F0EC0AF01FEC1DF06F0E55EC73F02FEC77
:106FF00050F007501AE1A0EC1DF0DCEC1BF082EC25
:1070000017F037EC14F097EC73F002E071EC1CF021
:1070100047EC14F0050E005C02E1D5EC07F00BEC38
:1070200022F02CEC61F084ECF1F0E9EC73F00AE171
:10703000010EDB502B92E8B02B822BB203D02B82B7
:1070400034EC15F0349A030EE15C02E2E16AE55299
:10705000E16E2AEF73F08C9800000000030EE66EDC
:1070600041EC59F0E552040E0A5CE66E41EC59F031
:10707000E5520150E66E41EC59F0E552D5ECF9F0DD
:10708000006E00008C881200D9CFE6FFE1CFD9FF57
:107090008C9800000000060EE66E41EC59F0E552B7
:1070A0008C880000000000008C9800000000020E98
:1070B000E66E41EC59F0E552040E0A5CE66E41ECD6
:1070C00059F0E5520150E66E41EC59F0E552FE0EE2
:1070D000DBCFE6FF41EC59F0E5528C88040EE66EFA
:1070E000A7ECF9F0E552E552E7CFD9FF1200E0EC4A
:1070F00079F00050DF6E010EDB6A3ED8DF50005C95
:1071000033E0680E0A5C02E1012A0106040E0A5C03
:1071100018E2F29EA6980A50636E0150626EDF502C
:10712000616E7F9E7F9C7F84550E7E6EAA0E7E6E62
:107130007F82F28E040EE66EA7ECF9F0E5527F94A2
:1071400013D0010EDB2ADFCFE6FF9EDFE55283DF9F
:10715000DF50005C02E005EC0CF0DF50005C04E066
:10716000050ECDEC74F0EDE3020EE15C02E2E16AA3
:10717000E552E16E2AEF73F0E0EC79F0010EDB6A84
:10718000040E0A5C0AE20A50636E0150626E7F9E32
:107190007F9C7F806150006E12D0010EDB2A5BDF86
:1071A0000050DF6E58DF0050DF5C02E005EC0CF0B1
:1071B0000050DF5C04E0050ECDEC74F0EEE3020E4F
:1071C000E15C02E2E16AE552E16E2AEF73F025EC40
:1071D00073F0CDEC78F013E0FC0EDBCFF3FFDB2A8D
:1071E000F350D6EC74F0FD0EDBCFE9FFDB2AFE0E88
:1071F000DBCFEAFF01E3DB2A00C0EFFFEAD72AEF8B
:1072000073F025EC73F0CDEC78F01BE09FEC77F099
:1072100018E38FEC7BF005E24B50A408000E4C54B1
:1072200010E36BEC77F0016EFC0EDBCFE9FFDB2A9D
:10723000FD0EDBCFEAFF01E3DB2AEF506DEC78F0C7
:10724000E2D72AEF73F025EC73F01F0E0501235DE2
:107250000DE2232B2551EA6A270FE96E050E10EC8B
:107260007CF0252B25511F0801E2256B2AEF73F0D6
:1072700025EC73F0030E0B5C5BE10F6A106AFE0EE7
:10728000DB500D0803E11F0E0F6E106AFE0EDB507F
:107290000A0803E11D0E0F6E106AFE0EDB5009088E
:1072A00003E1EF0E0F6E106AFE0EDB50080803E1DB
:1072B0000F68020E106EFE0EDB507F0804E1B50E63
:1072C0000F6E030E106EFE0EDB501F0827E27F0EBE
:1072D00058EC73F023E2410E58EC73F00EE3FE0E0F
:1072E000DB505A080AE3200E4B6EFE0EDBCFE7FFA1
:1072F0004B50E726FE0EE7CFDBFFF80E4B6E850EF8
:107300004C6E010E4D6EFE0EDB50E00F73EC7CF008
:107310000900F5CF0FF00A00F5CF10F00F50101054
:1073200049E010C0E6FF8FDFE5520FC0E6FF3DD019
:10733000FE0EDB50090803E1200E46EC76F0016AF0
:10734000400E015C37E20D0E4C6EAF0E4D6E010E1D
:107350004E6E015086EC73F0FE0EDB504B5C28E164
:10736000030E066E01B0068C01B2068A01B40688CF
:1073700001B6068601B806842450040B09E1200EEC
:10738000011406E06F0EE66E5EDFE55224840BD03A
:107390002450040B08E0200E011405E17F0EE66E78
:1073A00052DFE55224940650E66E4DDFE55202D0DE
:1073B000012AC6D72AEF73F0D6EC79F0800E58EC8C
:1073C00073F003E3200E46EC76F00201050E2C6FFD
:1073D000FE0EDB50740810E1010E2C6F030E0B5CE7
:1073E00007E10501235153EC7CF0020F02012C6FE1
:1073F0000501106B1E822BD0FE0EDB5028E0DF6AE9
:10740000150EDF5C11E2E2EC7BF00BE1DF2A7DEC94
:1074100075F069EC79F0DF2A7DEC75F069EC79F0B4
:1074200003D0030EDF26ECD7150EDF5C04E115EC6C
:107430007AF01EDFE552200E58EC73F003E2200EC6
:1074400046EC76F015EC7AF048EC6BF0E552E5523C
:107450002AEF73F0E0EC79F024A012D01EB009D02E
:107460000201565D1CE30701016B026B56C257F225
:1074700016D00201562B565180081BE2800E18D000
:107480001EA010D0070E0701015D09E2012B029139
:107490000243020E0201565D02E30701028F020160
:1074A000010E06D00201562B5651800802E2800ED2
:1074B000566F1E9024B01E802450010B03E1020E73
:1074C000565D04E01E50020B01E188D01EA204D0DC
:1074D0000701CC0E026F0FD0070102910243028F09
:1074E000070ED8800155016E01500106000903E026
:1074F00002910243F9D700C70AF002015751070869
:107500001DE257513F0802E23F0E576FC1EC77F082
:1075100006E0200E48EC75F0200E69EC79F03BECAB
:1075200077F00CE00701035109E0800E02015725B6
:10753000006E03C701F007010307D9DD780E0701CC
:10754000025D18E22A8A02C7E6FF40EC04F0E55229
:10755000DF6EDF500EE0C1EC77F00BE02C5104E061
:10756000DFCFE6FF29DF04D0DFCFE6FF48EC6BF08A
:10757000E5522A9A0101B1A731D00701035105E074
:1075800002C700F003C701F0B2DD0701035106E0B6
:107590001E50020B03E11C0E025D1DE103510AE0C7
:1075A0001C0E025D07E1CC0E006E030703C701F05D
:1075B0009EDD1E820101B197E6EC61F0230E165CA0
:1075C00003E1410ED5EC73F0259224BC2582020123
:1075D000010E2C6F01D003070701026B0A6A020E2D
:1075E000E15C02E2E16AE552E16E2AEF73F0E5EC5C
:1075F00075F00CE11A0E0101B55D08E11950400B60
:1076000005E084848C808D8A8D8C12000601505197
:10761000040B02E08D8C01D08D9C5051080B02E0D0
:107620008D8A01D08D9A5051010B02E08C8001D0DF
:107630008C905051020B02E084841200849412005A
:10764000000012000601D99D8850800B01E0D98D01
:10765000D99F8850400B01E0D98FD9918850100BE9
:1076600001E0D981D9938850200B01E0D983D999C1
:107670008850080B01E0D989D99B8850040B01E0A0
:10768000D98B120025EC73F0FD0EDB5058EC73F033
:1076900008E3FE0EDBCFE6FFFD0E27EC78F00AE2F2
:1076A00007D0FD0EDBCFE6FFFE0E27EC78F002E2FE
:1076B000010E01D0000E2AEF73F039EC7BF02FB2EF
:1076C00054D082B003D00701290E76D082B203D005
:1076D00007012C0E71D0DF6A060EDF5C43E2DF503B
:1076E000040DF35083093AEC79F0050EDF5C03E1F9
:1076F000DE52BB0EDD6E31EC7CF000C068F700504E
:107700001A082EE2F00E005C2BE2FE0EDB5002E1C6
:10771000010E56D031EC7CF000C069F700501A0819
:107720001FE2F00E005C1CE231EC7CF000C06AF756
:1077300000501A0815E2F00E005C12E2080EE66E28
:1077400069C7E6FF68C7E6FFCAEC75F009E0080EF6
:10775000E66E6AC7E6FF69C7E6FFCAEC75F002E1AC
:10776000DF2ABAD7060EDF5C02E1000E29D0010E37
:1077700091EC75F02FEC78F010E20C0EE66E020E34
:10778000DB50350FE0EC75F0E66E69C7E6FFCAEC3A
:1077900075F003E1020EDB2AEDD72FEC78F00FE253
:1077A00068C76BF769C76CF76AC76DF7020EDB50E5
:1077B000080DF350DF1007016E6F6E5101D0800E7F
:1077C0004B6E030EE15C02E2E16AE552E16E4B5062
:1077D0002AEF73F0E4EC77F08EEC79F006E102EC3E
:1077E00077F003E001011E0EA86F01012D0E186F46
:1077F00020A402D02B0E186F0201435107E1425121
:1078000005E1415103E10101200E186F61EC7AF0AE
:1078100043C240F095EC7BF0300F0101196F300E40
:107820003C241A6F300E0201422501011B6F070133
:10783000E3AB05D0300E0201412501011C6F0101AF
:107840001A8F12009FEC7CF0EFCFDFFF01019F6BDE
:10785000A06BA16BA26BA36B1EAE03D0050EA16F34
:107860003BD087EC77F0400B03E12850040B1DE080
:1078700015EC7AF01FEC0CF0E55200C0A1F10050BD
:10788000630825E20101A16BA02B7D0E005C02E1E3
:10789000190EA16FB4EC7AF0FA0E4B1818E14C50A7
:1078A00016E1A02B320EA16F12D087EC77F0200BDF
:1078B00002E0A32B0CD087EC77F0100B07E0020E50
:1078C000A26F58A704D0050EA26F01D0A22B2BAE39
:1078D00003D0020E64EC73F0E5522AEF73F0A90EA8
:1078E000006E005056EC78F036C100F0D2EC79F022
:1078F00001011B5D05E13EEC7BF002E1200E1C6FF7
:107900000201060E3F6F9DEF23F025EC73F0CC0EC5
:107910004B6EB10E4C6E010E4D6E050E516E51C088
:1079200045F0FE0EDBCF40F05CECFAF040C04EF0CC
:1079300063EC7CF0006EADECE0F00101020E006F34
:1079400090ECE6F00101138F0C0E58EC73F003E29B
:107950000E0E106F0ED00E0E116FFE0EDB50630870
:1079600002E2100E116F0F0E58EC73F002E2090ED6
:10797000126F140E156F120E166F2AEF73F025ECAE
:1079800073F0BDECE0F00101012BFE0EDB50006E48
:10799000ADECE6F02C50100B07E1640E58EC73F0E0
:1079A00003E20101200E186F2CA807D001014D0E33
:1079B0001C6F570E1D6F198F16D0FD0EDB5003E1A3
:1079C00001011A8F07D0640E58EC73F003E2010135
:1079D000200E196F0101570E1C6F34B802D02A0E09
:1079E0001D6F60B31D8F2AEF73F025EC73F09DECD3
:1079F00023F0FE0EDB5003E08BEC79F003D000683F
:107A000007EC25F0B8EC1FF0000907E0010EE66E68
:107A100083EC05F0940FE66E03D0E66A49C1E6FFF9
:107A2000AEDFE552E5522CA807D00068FBEC24F04D
:107A300049C1E6FF6ADFE5522AEF73F0D6EC79F030
:107A40009DEC23F0B10E006EF0EC24F035C1DFFFA9
:107A500059EC78F003E092EC79F001E1DF6ADF5055
:107A6000006EADECE6F0640EDF5C03E20101200E77
:107A70001B6F0A0EDF5C03E20101200E1C6FE55252
:107A80002AEF73F0E4EC77F08EEC79F006E102EC8B
:107A900077F003E001011E0EA86F4AC100F0ADECC3
:107AA000E6F0640E01014A5D02E2200E176F0A0E35
:107AB0004A5D02E2200E186F8C0E006E48EF24F033
:107AC000270ED5EC73F00101500EA86F3C51200B2E
:107AD00006E102EC77F003E001011E0EA86F120030
:107AE000EF0E006E97EC73F002E0F20E006EF0EC19
:107AF00024F033C100F097EC73F002E054C100F0C1
:107B00000101040E016FADECE6F001011C8F1200C3
:107B100025EC73F097EC73F003E071EC74F003E084
:107B200029C100F008D0B6EC79F003E059C100F0AB
:107B300002D055C100F02AEF73F0CA0E006EF0ECCF
:107B400024F0010EE66EE4DFE552D2EC79F001019B
:107B50001B5D05E13EEC7BF002E1200E1C6F120084
:107B600025EC73F057EC7CF0400B03E12850040B3C
:107B700005E001018F51020B01E18BD057EC7CF045
:107B8000200B03E02850040B02E001019E6B57EC30
:107B90007CF0400B03E12850040B57E00101A05199
:107BA0000EE0A1510CE1FE0EDB5005E19C5102E11B
:107BB0009D5101E0A06B9C6B9CC19DF16AD05A0E57
:107BC000A15D13E161EC7AF09CC140F0D4EC78F057
:107BD00007E1005003E101019D5102E00101A16BA9
:107BE00001019D6B00509C5F54D09C5102E19D515E
:107BF00050E09D514B6E4C6A9C510A0DE9EC7BF0B4
:107C0000A1510A0D3FEC79F00AEC75F0D4C144F0B3
:107C1000D5C145F002ECFAF03BC0D2F13CC0D3F143
:107C20000101D251D31135E0D2510F5ED351105A18
:107C3000FE0EDB5001E1A16B4AEC78F0AAEC7CF07F
:107C40003FC09CF13BC09DF124D057EC7CF0100B61
:107C500020E057EC7CF0200B1CE1020E016E0101CC
:107C600058A702D0050E016E01C0A2F101C045F077
:107C70009DC140F0D4EC78F004E1005002E000C077
:107C8000A2F1FE0EDB5005E0005003E000500101C0
:107C9000A25F2AEF73F025EC73F015EC7AF0E66A38
:107CA0005FDFE552E5529AC1B7F29BC1B8F29CC1C1
:107CB000B9F29DC1BAF29EC1BBF2EBEC2FF001010B
:107CC0009A510DE11F0E9B5D0AE2B7C29AF1B8C24C
:107CD0009BF1B9C29CF1BAC29DF1BBC29EF10201F7
:107CE000722B2AEF73F001012C51615D06E1DA93EA
:107CF000CDB3DA83DA95CDB5DA851200010139A367
:107D000006D0CD9313B6CD83CD9513B4CD85EBDFDF
:107D100004B060DD1BECA5F0A0EF2CF00A0E020110
:107D20004203F3504D6E4E6A4351640DB9EC78F046
:107D3000415101014B24D66F000E4C20D76F0A0E23
:107D4000006E0701E3AB02D0010E08D0E3A907D013
:107D5000140E006E010158A702D0320E006E20B43E
:107D600005D00101D66DD71F000ED72329AA1AD03E
:107D7000B4EC7AF0100ED8804B56270E4C56010109
:107D8000D7514C18E8AE02D04C3404D04B50D65DDD
:107D90004C50D7591FE2B4EC7AF04B50D6274C50D8
:107DA000D72318D000504C6AF00F4B6ED80E4C22DF
:107DB00001014C50D719E8AE02D0D73504D0D651C6
:107DC0004B5CD7514C5806E2B4EC7AF04B50D65F7E
:107DD0004C50D75B2084800ED71505E02094D66DDB
:107DE000D71F000ED723B4EC7AF0D6C13FF0D7C12D
:107DF00040F0A8EC78F04CAE04D03B6C3C1E000E7A
:107E00003C223B500101D65F3C50D75B640E4B6E69
:107E10004C6AF0EC7BF03FC043F23B500101D66F5F
:107E2000D76B4AEC78F0F0EC7BF03FC042F23BC0FD
:107E300041F21BEF3FF0308E04807EEF3EF00A01EE
:107E4000DA9F26EC0BF0016A0101D05112E14BECF4
:107E500076F02AE10701E3BF12D00A0E016E050E8B
:107E6000C2EC74F04050006E0150005C1DE2005006
:107E70001AD0030ED05D11E10701E3AF02D0160E58
:107E800012D0030E0B5C02E1140E0DD00B5002E178
:107E90001E0E09D00DEC7BF006D053EC76F002E01C
:107EA000010E01D0160E016E0150160802E2160EE8
:107EB000016E1200000CFEDF000903E00101500E0C
:107EC000496F120025EC73F000AE14D0FF0E0002D3
:107ED000F3CF72F2720EE96E020EEA6EEFCF40F04F
:107EE000FE0EDBCF45F05CECFAF040C0EFFF020184
:107EF000726D09D000C040F0FE0EDBCF45F05CECA7
:107F0000FAF040C072F22AEF73F0D6EC79F03050FC
:107F1000200B5AE12450800B57E13150400B54E1C3
:107F20002550010B51E120A61BD033EC78F0010164
:107F300027990201725102E0010127890101279B63
:107F4000020172AF02D00101278B010127A93CD0A9
:107F50001EAC02D0C3EC0AF00201640E3D6F34D0B7
:107F600025C100F001012799005001E02789279BD6
:107F700000BE278B27BB006CE5EC75F017E12F5096
:107F8000100B0DE01F50040B0AE11C50080B07E119
:107F9000005002E0B7EC07F0006A0101256B210EEA
:107FA0000101B55D06E0410EB55D03E000380F0B41
:107FB000006E005007E00101278D279F27BB278F08
:107FC000256B02D001012799010127A902D0A2EC5B
:107FD00004F001012751100B06E02C50200B40E06B
:107FE0001E50400B3DE12050080B16E03C51200B89
:107FF00013E13CB332D03BEC78F001012899020147
:10800000725102E0010128890101289B020172AF2F
:1080100027D00101288B24D026C100F028990050D8
:1080200001E02889289B00BE288B289928BB006C7A
:1080300033A005D00038E8461F0B006E04D0D8905E
:108040000032D890003200500AE00701460ECD6F92
:108050000101288D289F28BB288F266B01D02899E5
:108060002C50200B03E01E50400B10E00101275163
:10807000100B02E065EF44F02851100B02E065EFB1
:1080800044F02150200B02E165EF44F0D7CADCFA3E
:10809000D6CADDFA0601D551D595010B01E0D5858B
:1080A000D551D597020B01E0D587D5918650040BA9
:1080B00001E0D581D5938650020B01E0D5830F0EE8
:1080C000D515B2EC74F000A019D0A2EC04F00601B2
:1080D0005051040B0CE03350010B09E13150040BFB
:1080E00006E100AE02D0DA0709D0DA2B07D000AEE5
:1080F00003D00101260702D00101262BDAC600F0C9
:108100000601D599005001E0D589D59B00BED58BDD
:10811000D5A930D0D5BB006C0090004200502AE0B9
:10812000DA6B0201640E3D6F060150A523D00101F8
:108130003851010B06E01350080B03E11350040BF8
:108140000DE0298A0601D5BB299AE8DD1FAC03D0D2
:10815000020109870FD0020106810CD0C8C225F1A7
:108160000601D5AB04D0C8C225F10101256D01017E
:10817000278928840601D651D695010B01E0D685C2
:10818000D651D697020B01E0D687D951D691020B72
:1081900001E0D681D951D693010B01E0D6830F0EB1
:1081A000D615B2EC74F000A009D08DEC77F000AEDB
:1081B00003D00601DB0702D00601DB2BDBC600F093
:1081C000D699005001E0D689D69B00BED68BD6A9A1
:1081D000CCD0D6BB006C31BC02D000900042005025
:1081E00001E1C3D0DB6B010E0E6ED6BB0E68FEEC58
:1081F00076F001E1B3D00201780E2B6FE9EC73F059
:1082000003E1ABEC0AF0AAD032BCA8D031AC0ED05E
:10821000D00EE66E0F0EE66EA50EE66E070E80EC33
:1082200073F008EC05F00DEC4DF098D0D0510BE058
:10823000030ED05D08E0CE51800B42E0020ED05D0F
:1082400002E0D0053DE115BC1CD03586BAEC0EF03D
:1082500045EC7AF007E24B501408000E4C5402E251
:10826000BAEC0EF045EC7AF009E24B503D08000EF6
:108270004C5404E2BAEC0EF0BAEC0EF0C3EC0EF083
:108280006DD03586D8EC77F008E0C80EE66E280E83
:10829000E66ED00EE66E030E0AD0D1DD190E012473
:1082A000E66E9EEC79F0E66ED70EE66E0A0E80EC76
:1082B00073F00A01030ED46F348A8AEC19F04BD0A4
:1082C00015BC25D03586BBDD0E040BE1DBEC78F068
:1082D00008E2190E0124D75D04E2020ED65FD72B07
:1082E00011D0800E0E140EE0AAEC0EF0FF0F0A0162
:1082F000D65D08E29EEC79F0D880D75503E2020EF5
:10830000D627D7070A01010ED46F348A25D03586C7
:1083100096DD800E0E140CE0DBEC78F009E29EECAA
:1083200079F0D880D75504E2020ED65FD7070FD078
:108330000E040DE1AAEC0EF0FF0F0A01D65D07E274
:10834000190E0124D75D03E2020ED627D72B0A01AE
:10835000020ED46F348A010E86EC78F01FAC03D085
:108360000201098902D00201068B0601D751D79577
:10837000010B01E0D785D751D797020B01E0D787D2
:10838000D951D791200B01E0D781D951D793100B48
:1083900001E0D7830F0ED715B2EC74F000A009D01E
:1083A0008DEC77F000AE03D00601DD0702D00601A8
:1083B000DD2BDDC600F0D799005001E0D789D79BAF
:1083C00000BED78BD7A996D1D7BB006C00900042D6
:1083D000005001E18FD1DD6B010E0E6ED7BB0E6830
:1083E0001AA8B7D001018EB568D134B831D021BEFA
:1083F00004D0850E006EFBEC24F0FF0E0E5C0CE149
:108400000201050ED8800155000E02551EE2060E2F
:10841000015F000E025B19D074C201F02C50100BEA
:1084200007E102017451780803E26C0E015C016EF1
:1084300001500C5C0AE20201880E015D130E025924
:1084400004E2060E0127000E0223BCEC0AF04ED116
:1084500002011C6B780E016E026AA6EC1FF0000987
:1084600002E0DA0E016E2CA804D0960E016E0A0E00
:10847000026E780EE66E490EE66E010E69EC73F040
:10848000010149510A0808E2010E491505E00E04F0
:1084900002E1492B01D049072B84FCEC04F00BECE2
:1084A00022F0010EE66EF5EC3CF0E5520101E383AB
:1084B000E395E39749C1E6FF70EC78F0780E016E22
:1084C0002C50100B12E10E0404E1790E0101495DFC
:1084D00007E0800E0E1409E001500101495D05E13D
:1084E000328EFEEC76F001E01D941CEC76F03250FA
:1084F000800B0EE1020120510BE000500EE0050E52
:10850000005C0BE0030E005C03E1020E0B5C05E077
:108510000E50E66E32EC1BF0E55232AE17D0329EB2
:1085200004981AA006D004880CEC0AF0050E64EC3E
:1085300073F0C1EC1FF084ECF1F004A802D007EC5A
:108540000AF00E50E66E32EC1BF0E5520201078B8A
:10855000CDD00101E2AF28D08EB5AFD035C1C6F283
:1085600078EC17F01E0EE66E350EE66E010E69EC25
:1085700073F01EEC3DF06EEC79F035C1E6FF70EC67
:1085800078F0DCEC1BF00201C65103E0010135512B
:1085900006E00201C65105E10101355102E0B1ECEE
:1085A00016F002010885A1D02DA426D0E385E3931F
:1085B000E39797EC73F00EE1C80EE66E330EE66EAD
:1085C000010E69EC73F033C1E6FF70EC78F0CBEC90
:1085D00060F00FD0C80EE66E010EE66E540EE66E29
:1085E000010E80EC73F054C1E6FF70EC78F063ECA0
:1085F00017F070EC3DF07AD025A033D0D05111E1C6
:10860000460EE66E280EE66E2A0EE66E010E80EC31
:1086100073F001012A51E8240301D06F43EC76F096
:1086200016D018EC76F007E0E66A2F0EE66E010E23
:1086300069EC73F00ED0E9EC73F00BE1320EE66EEC
:10864000010EE66E9A0EE66E020E80EC73F008ECF8
:1086500005F05AEC4CF0E66A4EEC74F0B1EC16F012
:1086600045D097EC73F003E071EC74F021E0320E2A
:10867000006E01018FAD02D0640E006E0050E66EF8
:10868000080EE66E4A0EE66E010E80EC73F042ECC8
:108690003DF00101E393E395E3874AC1E6FF70EC07
:1086A00078F04AC113F575EC61F0020106871ED01F
:1086B0001CEC76F001018EA503D0B0EC07F016D0CB
:1086C00078EC17F0280EE66E360EE66E010E69ECB9
:1086D00073F037EC14F06FEC3CF06EEC79F036C1CF
:1086E000E6FF70EC78F0020108832B842E8E0201E5
:1086F0001E0E1F6F0601D851D895010B01E0D885D9
:10870000D851D897020B01E0D887D951D891800B66
:1087100001E0D881D951D893400B01E0D8830F0EE6
:10872000D815B2EC74F000A009D08DEC77F000AE53
:1087300003D00601DC0702D00601DC2BDCC600F00A
:10874000D899005001E0D889D89B00BED88BD8A911
:10875000BCD0D8BB006C00900042005001E1B5D005
:10876000DC6B010E0E6ED8BB0E682DA631D097ECD7
:1087700073F003E071EC74F00AE0280EE66E290E47
:10878000E66E010E69EC73F077EC75F01ED059ECD3
:1087900078F00BE11E0EE66E590EE66E010EE66EE7
:1087A00068EC7FF0E552E5520DD01E0EE66E550ED8
:1087B000E66E010E69EC73F06EEC79F055C1E6FFE0
:1087C0000DEC09F0E55282EC17F09DEC3DF079D00C
:1087D00024AE37D022B675D0016A0101D05102E033
:1087E000010E016E015085EC7AF0EF50006EB4EC92
:1087F0007AF0190E48EC73F0190E4C02F3CF4CF0DE
:108800004B02F3CF4BF0F4504C264B50006E0E044D
:108810000AE1DDEC7AF004E6E20E4B5C000E4C5807
:1088200002E2190E0026FF0E0E5C05E1005018084A
:1088300002E2190E005E015085EC7AF000C0EFFFF5
:108840000BD030AA0DD022B63CD00E0EE66EA60E8E
:10885000E66E020E69EC73F008EC05F0248A31D064
:1088600022B00ED022B62DD03C0EE66E670EE66E1C
:10887000010E69EC73F014EC50F02FEC05F021D0F0
:1088800022B61FD0E9EC73F00CE1280EE66E690EFB
:10889000E66E010E69EC73F0F0EC0AF06DEC05F099
:1088A00010D0800E0E1404E03C0E685D01E2682BCF
:1088B0000E0403E1685101E068072FEC50F049EC29
:1088C00005F02E8E02011E0E1F6F1EAC66D0070132
:1088D000E38346EC08F001013C91139C3C51010BF1
:1088E00001E0138CE66A60EC2AF0E552006E00505D
:1088F0000F0802E20F0E006E100E0002F3CF0EF210
:1089000093EC25F01E9A050E0701C8250201D880B8
:108910000E5501E21E8A2B50800B13E10D5111E020
:10892000050E0701C85D02010E5D03E29FEC07F032
:108930001E881E50100B31E01E50200B2EE002014D
:1089400009D02B50800B0AE11E50800B07E11E500E
:10895000200B04E0FA0E0D6F1E981FD02BBE02D024
:108960009CEC07F02CBA17D01E0EE66E050E64ECD8
:1089700079F0E66E37EC76F00AE019C5C0F11AC559
:10898000C1F11BC5C2F11CC5C3F11DC5C4F1C8C2EC
:1089900025F10101279B010127891E50800B0DE164
:1089A00001012751100B01E17CD02050080B01E19F
:1089B00078D02150200B01E174D002011E0E1F6FF0
:1089C0001EAC02D0140E1F6F2CAA2FD01EBC16D0C6
:1089D00001014551630801E2456B800E251506E053
:1089E000FB0E255D03E2256B000E12D0800E2515CF
:1089F00057E12551030854E2256B09D00101256B8D
:108A00002BAE09D0050116514BE1320E166F010E47
:108A1000E2EC78F045D0A951030842E3010EE2EC04
:108A200078F00101140EA96F3BD01F50400B03E0FA
:108A30000951010B35E11FAC02D0098101D0068339
:108A40002C8C2D8A27EC75F0D0C1E6FF22EC3CF08F
:108A5000E55233EC78F01E50800B06E00101255101
:108A600003E1C7EC2FF016D0020172AF0AD0E3C7C2
:108A7000E6FF4BEC3EF0E5520201C851010125270B
:108A800009D0725107E0E3C7E6FFD7EC76F0C85192
:108A90000101255F02017251DCE12E8288EC04F0B5
:108AA0001E9E01012851100B51E02050080B4EE092
:108AB0002150200B4BE002011E0E1F6F1EAC02D096
:108AC000140E1F6F1FAC02D0098301D006832C8CBB
:108AD000D1C1DFFF2D9AB6EC76F0DFCFE6FF22ECB6
:108AE0003CF0E5523BEC78F0020172AF0DD0DF5064
:108AF000F2EC73F0EF50E66E4BEC3EF0E552020103
:108B0000C951010126270CD072510AE0DF50F2EC66
:108B100073F0EF50E66ED7EC76F0C9510101265F95
:108B200002017251DFE12E829AC1C5F19BC1C6F1EB
:108B30009CC1C7F19DC1C8F19EC1C9F125A606D04F
:108B40000101010EA86F0701140E766F2CAC08D03E
:108B500029EC2DF00FEC30F02C9C26822DAA248AD3
:108B60000101289927992894E5522AEF73F0770E8E
:108B700044EC75F00101320EA86F308834C118F250
:108B80001200010138A70AD04D0E0A6E0F0EE66ED4
:108B9000100E0D03F350CBEC77F010D0030E0A6EDD
:108BA0000F0EE66E140ECBEC77F03DEC73F0030E77
:108BB000E66E230EE66E230EE66E0A0E3DEC73F0B3
:108BC0000A6A120025EC73F0030E0A6E140EE66EAC
:108BD000000EE66E0A0E0CEC7CF0040EE66E260E1D
:108BE000E66E0A0EE66E260E97EC7AF0FE0EDB506D
:108BF0001EE0010138A70AD04D0E0A6E0F0ECBEC15
:108C000077F0E66E100E0D03F3500ED00F0ECBEC86
:108C100077F0E66E140E97EC7AF0030EE66E230EF4
:108C2000E66E0A0EE66E230EE66E43EC73F00A6AF9
:108C30002AEF73F0030E0A6EAA0EE66E2A0EE66E97
:108C40000A0EE66E300EAEEF7CF06AEF7CF00101AA
:108C500022A184EF4AF0229102010F070F5101E097
:108C600032D1640E0F6FE9EC73F016E12150400B26
:108C700013E1080E9BEC74F0046E04AC0DD00101FE
:108C8000E1BF02D0E18F02D0E1BFE19FE66AC0EC14
:108C900036F0E5520FEC30F002013F510CE03F514D
:108CA000010803E3FEEC76F006E002013F073F51C6
:108CB00002E19DEC23F03296150E0101565D0BE0AA
:108CC00002011551161103E01507000E165B155130
:108CD000161101E1308C01018C5104E08C078C519C
:108CE00001E1329602011F510CE02050080B09E00F
:108CF0001F071F5106E11EAC02D01E8E02D02EBEF1
:108D00002E9E300E0401F75D06E10201066B076B33
:108D1000086B096B05D0340EF75D02E2B5ECA8F0E4
:108D2000020118511CE00501105119E12850400BB7
:108D300016E102013851391112E1180718510FE1FB
:108D40000D50006E585106E07F0E5815006E199AAE
:108D500058BF198A010EE66E00500FEC78F0020140
:108D60005B075B510BE10101525102010B5D06E211
:108D70007D0E44EC75F00101A869268EFEEC76F0BC
:108D800008E00101845105E0775103E105ECEEF0C4
:108D900002D0CEECEEF096EC79F009E0E5EC75F05F
:108DA00006E1280E0101B55D02E106011D79010110
:108DB0003C51100B11E01C50100B0EE12250020B25
:108DC00009E0050ED05D06E0040ED05D03E01F5003
:108DD000200B02E10601047901013951100B06E173
:108DE0001450020B05E01A50200B02E106010D752C
:108DF0002950400B01E0010E020F016E2950400B7B
:108E000001E0010E050F026E03681EAC08D099EC5C
:108E10007BF0EF7E99EC7BF0EF50800B036E53EC10
:108E200076F00EE02D50400B0BE12D50800B08E149
:108E30000101E0B703D00601067902D006010689D8
:108E40000201315105E01450080B02E006011073D5
:108E5000010184512BE076ECEEF0000903E12F5084
:108E6000200B24E02F9A2DEC15F0016A030E015C13
:108E700012E2026A040E025C08E2020E94EC7AF03E
:108E8000320E64EC73F0022AF5D7E66808EC20F0A5
:108E9000E552012AEBD734EC15F0010160992682E6
:108EA000F9EC7DF060ECEEF005ECEEF002012C51F7
:108EB00001E02C077E5104E02350100B01E17E07F6
:108EC000335101E033071FAC08D0F307F35105E13C
:108ED000B5ECA8F00201030EF36F3851391141E0EF
:108EE0002150400B3EE01A50400B3BE03BEC77F04A
:108EF00003E11A50200B35E002013807000E395B00
:108F00001A50200B0AE0D4EC77F009E183EC75F0FD
:108F100004E10101E051100B02E1000E01D0010E4D
:108F20000490E8B0048002013851391103E0045084
:108F3000010B17E0386B396B0101E09904A006D0F2
:108F40000201186B18C258F2E6EC61F0D6EC09F099
:108F50000101B1A705D0259224BC25821AEC77F037
:108F6000219402013D5101E03D073E5101E03E07E1
:108F70003C5101E03C07345101E03407305101E03D
:108F800030072F510AE02F072F5107E17FEC76F0D1
:108F900001E14C5002E018EC0CF00201175109E01D
:108FA0001707175106E1FAEC76F00201F25101E1E0
:108FB0001294100710513CE1280E106F1BAC0FD01B
:108FC000E8EC35F0D0C100F026EC36F0060101796E
:108FD00001A92ED0D1C100F026EC36F029D01CA872
:108FE00003D00601047924D01DA203D00601147118
:108FF0001FD01A50200B06E001013951100B02E17D
:1090000006010D752550020B03E1D0EC77F010E05E
:1090100002012F510DE17FEC76F001E14C5008E0A8
:109020002D50800B05E12D50400B02E1060101712E
:1090300002012A5101E02A070701CD5105E0CD07C1
:10904000CD5102E11CEC79F00201295116E029070B
:10905000295113E197EC73F003E1ABECE7F00DD08D
:109060000701CA51CB1109E0CA5101E0CA07CB512F
:1090700001E0CB070201020E296F020128510CE02A
:109080002807285109E1188E18901888080E166EC6
:109090002DAC02D0290E166E0101AA516DE0AA076F
:1090A000AA516AE1AEC1F6FFAFC1F7FFB0C1F8FF48
:1090B0000800F550006E0201C75107E0830E0A6EEA
:1090C000C7C201F0BCEC38F00A6AFF0E0201975DDE
:1090D00022E0130E4E6E920E4F6E010E506EB5C111
:1090E00051F0526A536A640EFCEC73F097C254F06C
:1090F000556A566A75EC74F00800F550006E02016E
:10910000972B005008E197690101020EAE6F8D0E9A
:10911000AF6F010EB06F005011E00101190EAA6F80
:10912000005048EC75F00201C75102E0C72B24D073
:109130000101AE2B000EAF23B0231ED02950080B27
:1091400003E13150080B02E0299616D00201C75105
:1091500005E0C76B0101FA0EA86F05D00101D89098
:10916000A833D890A83324A607D01F0EE66E8D0E24
:10917000E66E010E74EC78F00201275104E0270737
:10918000275101E1269E265107E02607265104E1DA
:109190000601416941C640F60101A6510DE0A6074E
:1091A000A6510AE1090E165C07E1E5EC75F004E151
:1091B0000101FA0EA76F1B8A0101A75101E0A70761
:1091C0000701765101E0760702012E5123E02E07B8
:1091D0002E5120E1000E0601E76EBE19E8AE02D066
:1091E000BE3503D0E750D880BE5502E2BE0701D09D
:1091F000BE2B000EE76EBF19E8AE02D0BF3503D01C
:10920000E750D880BF5502E2BF0701D0BF2B020153
:10921000050E2E6F145105E01407145102E19DEC68
:1092200065F00201205121E0200728AA1ED021BCB0
:1092300018D01B50800B15E0800E081412E021504E
:10924000010B0FE1206B1B9E0A01DA8F26EC0BF05D
:109250007BEC77F01FAC03D00201098902D0020138
:10926000068B205102E1248A26820D5107E01E5010
:10927000400B04E00D070D5101E11E8E0501165152
:1092800001E016070201365105E03607365102E1CA
:109290008FEC09F00201D25101E0D207F2510DE04A
:1092A000F207F2510AE107010A8355ECF1F02FECC5
:1092B00050F00201175101E112942B5101E02B07EC
:1092C0000101A8515CE0A807A85159E1B19DB19FE7
:1092D0003098E0951D921C9831BCC0DB30BAA4DAFE
:1092E00024BE32DA25B0FCDA2682248A289821BAF4
:1092F00002D03DEC25F0218A0C0E165C29E12250AB
:10930000200B26E00101A65123E11668E5EC75F07B
:1093100002E11F8417D001013C71139C3C51010BE9
:1093200001E0138C75EC9DF0540ED5EC73F0010147
:109330003CA108D04B0EE66ECC0EE66EEEEC08F0CB
:10934000E55204D0550EE66E1DEC25F0E5521B8665
:109350001E50400B14E02B50800B11E12250200BCB
:109360000EE02B8E130E56EC78F0460EE66E410E94
:10937000E66ED6EC08F0E552E5529FEC07F00201EC
:109380001C5101E01C071D5101E01D071E5101E0A9
:109390001E07355101E03507315101E031073251E7
:1093A00001E032070101A95101E0A90702013A5188
:1093B00001E03A07060143510AE04307435102E145
:1093C0005A0E436F26860F0E435D01E22696020178
:1093D000215108E02107215102E153EC65F002011F
:1093E0001E0E206F3B5111E001012751400B0DE192
:1093F00002013B073B5109E145C100F01986358464
:1094000075EC9AF00201010E236F0201235147E02F
:109410002307235144E1780E2B6F0101E38FFAEC0F
:10942000F1F00201176BF25101E11294FAEC76F0BF
:1094300021A204D02192A0EC2CF022D096EC79F05D
:1094400007E03C51100B04E03C991F9A35EC7BF08F
:109450003CEC12F0B1EC16F0259C076A34EC15F0E8
:10946000640E64EC73F005ECEEF037EC77F008E096
:109470002150200B05E0010EE66E15EC9EF0E55242
:1094800019B006D00BEC22F05BEC3FF0F0EC76F07C
:109490001990020106891FAC02D00987098537514E
:1094A00004E03707375101E12682245101E0240707
:1094B000F45109E00501105106E10201F407F451ED
:1094C00002E11AEC09F00201225101E022071A51CF
:1094D00006E01A071A5103E1630E55EC73F002011E
:1094E0001B5106E01B071B5103E1B10E55EC73F055
:1094F0000201195105E01907190502E10AEC0FF004
:1095000002012D5101E02D07120006014F6B4FC6DD
:109510004EF64FC64DF64FC64CF64FC64BF61200F0
:10952000E0EC79F0DE52010EDD6EFE0EDB501AE14A
:10953000C5EC7BF0050EE66E200EDF24E66E4B0ECA
:10954000E66E060E3DEC73F0050E9BEC7CF0B60E5D
:10955000E66E010E3DEC73F00F0EE0EC7AF0005079
:10956000DF6E0A6A0101B651630805E3B6510EE1E8
:109570001F0EB75D0BE2360E006EE5EC24F0FE0E1A
:10958000DB5001E1C2DF010EDB6A23D0FE0EDB50AF
:1095900020E12D50800B07E0DF500A0804E20701AC
:1095A000E39B46EC08F0DFCFE6FF3CEC31F0E55200
:1095B00001018B51100B0DE00A0E455D0AE2ADEC86
:1095C000E0F00101050E006FDFCFE6FFBEEC85F095
:1095D000E5520201285116E1640E0101455D0CE2DD
:1095E00061EC7AF045C140F095EC7BF0300F010161
:1095F000176F300E3C2405D04D0E176F030E451526
:10960000310F186F016A050E015C2EE2850E4B6E5C
:10961000AF0E4C6E010E4D6E0150EA6A4B0FE96EB3
:10962000060EEA22EFCF4EF063EC7CF0026E2D0EB8
:10963000025C05E10101B25102E1200E026E02015D
:10964000285110E1020E012471EC77F002C0EFFF07
:10965000015008E12C9A2A0E025C04E12D50800B87
:1096600001E02C8A012ACFD70201285102E1010131
:10967000198F010EDB50A6EC79F002E2E16AE552A7
:10968000E16E4B502AEF73F04CEC79F0016E4551CE
:10969000D7EC75F0050EE66E4B0EE66E060EE66E26
:1096A000200E0124AEEF7CF00201050EDA6FF00E01
:1096B000DB6FFA0EDC6F140EDD6FF00EDE6FFA0E4C
:1096C000DF6F1200016A0101D05102E0010E016E4C
:1096D000015078EC73F0EF50006ECEAD006A01508F
:1096E00085EC7AF0EF50E66E015078EC73F0010EE5
:1096F00097EC7CF0E66E0050E66E250EBCEC74F044
:1097000001011596CE51400B01E015861200026A48
:109710000101D05102E0010E026E025085EC7AF098
:10972000EFCF4BF0190EA2EC73F001EC76F002E1F2
:10973000200E1C6F4E0E196F520E1A6F62EF4BF017
:10974000248E209687EF4BF0249E43EF78F0020E94
:10975000E66EBD0E4FEC73F00101CCBB0FD0BB0E1B
:1097600055EC73F0010EE66E200EE66EE66A2F0EE3
:10977000E66EF7EC14F05FEC7CF03DD0070E0201D2
:10978000A65D1BE2A651E8244B6E4C6AFF0ED88002
:109790004B56000E4C564B50E66E060ED880A65522
:1097A000070DF3500A0FE66EBC0E38EC73F0010E95
:1097B000E66E200EE66EE66A17D0F30EE66E0A0E2F
:1097C000E66EBC0E38EC73F00201A6510A0802E204
:1097D000030E01D0010EE66E0F0ED880A6550C0DBB
:1097E000F350E66E800EE66E2F0EBCEC74F0B90EF0
:1097F000E66EBBEC14F0E55201011594CC51200B40
:1098000001E0158412000201A62901EC76F002E1C4
:10981000200E1C6F4E0E196F420E1A6FA7EF4BF001
:10982000308A209603EF4CF0309A43EF78F0BDEC8D
:10983000E0F0E9EC73F01AE1020E016F0D0E020187
:109840009A2508EC79F0DFEC73F071EC75F0030EFB
:10985000E66E020EE66EFAEC07F0E552E552010103
:109860001D8F500E176F4C0E186F1200030ED05D37
:1098700010E118EC76F006E0290EE66EE60EE66ED4
:10988000010E05D0210EE66EE60EE66E010E9CEF8F
:109890007BF0016B2AC100F0D2EC79F00101175D79
:1098A00002E1200E176F300E1A6F480E1C6F5A0E11
:1098B0001D6F12002550010B09E1E9EC73F006E081
:1098C0002DEC15F0030E006ED6EC70F02580E9EC5F
:1098D00073F003E00068F0EC24F0209617EF4CF0F2
:1098E000E9EC73F003E1A0EC1DF004D08FEC09F07B
:1098F00034EC15F025901B940101A86BB19F2498BE
:10990000D7EC0BF0FEEF0CF0BDECE0F0F60E4B6E7A
:10991000860E4C6E010E4D6E0B5057EC76F0F9EC46
:1099200079F0F8EC73F018C1E6FF17C1E6FFD6EC4A
:1099300008F0E552E552010137AD02D0AEECE4F09B
:10994000120033808BEC79F02096DEDFB0EF36F03A
:109950003390D7EC0BF0FFD93098120027EC7AF057
:10996000140DDFEC73F0AEEC79F005E0D1EC74F09F
:10997000230E38EC73F0F1EC13F0140E64EC73F07A
:109980002AEF73F025EC73F0D8C200F0FE0EDB5026
:1099900001E1006AD9C2E6FF0050E66E240E38EC01
:1099A00073F02AEF73F04FEC7AF00701B051A55D28
:1099B00016E11550100B01E0010E4B6E3450020BF6
:1099C00001E0010E4B5C0BE11550200B01E0010E94
:1099D0004C6E3450040B01E0010E4C5C1CE0076A35
:1099E000A5C7B0F7349215B83482349415BA3484CC
:1099F00015A80BD015AA03D0A5C7E6FF07D0E66AC5
:109A0000ADDFE552010EE66E04D0E66AA7DFE5524F
:109A1000E66AB8DFE55253EF7AF00701A551140D5D
:109A2000DFEC73F071EC75F01AC117F11BC118F17E
:109A30001CC119F11DC11AF10101200E1B6F480E46
:109A40001C6F5A0E1D6F300E175D02E1200E176F4E
:109A5000D3EF4CF0318C20960DEF4DF0319C01018D
:109A6000A86B2498B19FD7EF0BF00101A85103E038
:109A70002550080B03E0B151200B01E03088005065
:109A800048EC75F00101A85106E03050100B03E1DD
:109A9000FA0EA86F25861200010E0701D8907737BD
:109AA0007837E806FBE122AC02D0070177810D0E82
:109AB0000701795D01E2792B1200229C8450020B90
:109AC00001E0228C07016F5111E122AC78D06F2B9D
:109AD000010E776F786B796F31987A6F7251FE0B48
:109AE000E8427225716F010122931200010122A345
:109AF00066D0229307016F0562E122BC52D031A8E3
:109B00004DD00C0E795D47E2D89078337733006AF8
:109B10005F0E005C1BE2F80E4D6E850E4E6E010E60
:109B20004F6E0050506E5AEC74F077514B180CE1A8
:109B300078514C1809E1200E0026610E005C02E30A
:109B4000200E005E92DF02D0002AE2D75F0E005C9A
:109B500022E107011F0E771901E178510AE01D0E7D
:109B6000771901E1785105E0EF0E771905E1785199
:109B700003E1200E006E79DFFF0E0701771902E185
:109B8000020E781906E0B50E771905E1030E781973
:109B900002E120EC6BF007016F6B120031884CEF93
:109BA0004DF07ADF31A804D00701010E7A6F06D09C
:109BB00007017A2B7A510C0801E26F6B3198120081
:109BC00008AE06D08450020B02E0229C01D0228C09
:109BD00007016F5110E122BC75D0010122930701EA
:109BE000706B08AE6FD0020E6F277251FE0BE84209
:109BF0007225716F12006F050BE16F2B72C771F741
:109C00000101229322AC5ED00701080E6F6F120093
:109C1000010122A357D02293070E07016F5D46E191
:109C20006F6B22AC40D00101A85103E02550080B16
:109C300003E0B151200B01E030880D0E4B6EAF0EEA
:109C40004C6E010E4D6E0701705173250FEC7AF0CA
:109C5000006E810E005C02E1736B1BD0800E005C15
:109C600003E1200E736F15D00D0E005C03E00A0EA9
:109C7000005C02E1200E0BD00B0E005C02E12A0E0C
:109C800006D00A0E005C05E0005003E0005048ECEE
:109C900075F00101A85109E03050100B06E1FA0EF1
:109CA000A86F25861200080E6F6F1200080E6F5DF8
:109CB00004E122AC07D06F6B12007091704322BC9C
:109CC00070896F2B1200BDECE0F04DEC75F014E1E3
:109CD000BAEC79F006E01A0E4B6EE60E4C6E010EF1
:109CE00005D0E60E4B6EE60E4C6E010E4D6E5CEC32
:109CF0007AF04DC0E6FF0CD0B60E4B6E860E4C6E61
:109D0000010E4D6EEAC64EF04F6A506AF9EC79F0DA
:109D1000F8EC73F0EDEC1DF092EC0EF0006E0050DC
:109D20000A01D65D05E200C0D6FAE66A4EEC74F090
:109D300012000101D05105E131848BEC79F02096BD
:109D400003D0006807EC25F063EF4EF03194D7ECB8
:109D50000BF0ABEF4EF0040EE66EEA0EE66E060E6A
:109D6000E66EA00E97EC7AF0140E016E3DC100F085
:109D700077EF38F0D6EC79F0E0C64BF0E1C64CF066
:109D8000D8904B364C36060173EC79F00CE3DEC606
:109D90004DF0DFC64EF0D8904D364E36E0514D5C5A
:109DA000E1514E5820E2DE51E0250F6EDF51E121F6
:109DB000106E5DEC78F0E2C64BF0E3C64CF0030E9B
:109DC000A9EC77F0FDE14B500601E25F4C50E35BFC
:109DD000AAEC7AF0030EA9EC77F0FDE14B500601F6
:109DE000E2274C50E323DEC6E0F6DFC6E1F693EC53
:109DF00077F04B364C36D8904B364C3673EC79F0C6
:109E00000BE393EC77F04C324B325BEC7CF04B5035
:109E1000DE5D4C50DF5902E2DF6A09D0E251DE5DBF
:109E2000E351DF5902E2010E01D0020EDF6E93EC26
:109E300077F04B364C364B50E225E46F4C50E32123
:109E4000E56FDF50E5522AEF73F01EBC1200229C32
:109E50008450020B01E0228C22AC03D002016F2B54
:109E600002D00201702B209E0601E65109E122ACCE
:109E70004BD0010EE66FDE6BDF6BE76BE86B44D017
:109E8000E60515E122BC40D0020EE66F73DF006EDE
:109E900000500BE0070E0601E85D07E2E82BE791B2
:109EA000E7430050010801E2E78F06011FD0020ED0
:109EB000E65D2AE122AC1DD0E2C64DF0E3C64EF0CD
:109EC000030E0F0B05E0D8904E324D32E806FBE151
:109ED00006014D50E25D4B6E4E50E3594C6E4B50B7
:109EE000DE5D4C50DF590EE2010EE66FDE6BDF6B7C
:109EF0000BD0E451E4254B6EE551E5214C6E73EC3B
:109F000079F002E2030EE66F030EE65D43E1E791AE
:109F1000E743E78F070ED880E855016E0150010630
:109F2000000903E0E791E743F9D7780EE75D30E2F7
:109F30000101A85103E02550080B03E0B151200BAB
:109F400001E03088E7C6E6FF40EC04F0E552006E21
:109F5000200E005C03E300506E0802E22A0E0BD0D4
:109F60002A8A005048EC75F00601DE51E45DDF51AD
:109F7000E55903E2200E48EC75F02A9A0101A85138
:109F800007E03050100B04E12586FA0EA86F3186E9
:109F90000601E66B208E12000101E183D05102E13F
:109FA00054DF07D0209EE0EC77F002E086DD01D0A0
:109FB00007DE0101E1931200800E081420E02B500F
:109FC000020B1DE12150200B1AE00201C75117E1DD
:109FD0000101D05104E10601EA51010806E34DEC0C
:109FE00075F00DE1BAEC79F00AE02A0E0101B11525
:109FF00006E10C0E165C10E12250200B0DE0800EE5
:10A00000081409E171EC74F006E00601EC5103E07C
:10A0100002012C5101E0000C010C02013A5103E154
:10A02000120ED5EC73F01200D6EC79F0076A67C116
:10A03000DFFF22A205D00101675153EC7CF0DF5E07
:10A040001FBCDF6ADFCFE6FF720E4FEC73F031808A
:10A050000201078335B2E1DFE5522AEF73F0D6EC57
:10A0600079F0076A68C1DFFFE9EC73F002E1DF6AAB
:10A0700005D007010AB302D00F0EDF5EDFCFE6FF87
:10A08000710E4FEC73F002010787E5522AEF73F06F
:10A0900025EC73F0040EE126C40EDE6E090EDD6EB3
:10A0A000080E91EC75F0070E78EC79F065EC78F01D
:10A0B00003E06051020B06E1FC0E91EC75F0080E16
:10A0C00078EC79F023A806D0B80E91EC75F00B0E61
:10A0D00078EC79F002010B517D0808E20101605132
:10A0E000020B04E1B80EDE6E0B0EDD6EE7EC77F0CE
:10A0F00003E2C1EC73F011E3E7EC77F00CE3020E3E
:10A10000DBCF4DF0030EDBCF4EF00201EF514D5C83
:10A11000F0514E5802E3000E01D0010E4B6E040EBA
:10A12000E15C02E2E16AE552E16E4B502AEF73F026
:10A13000E0EC79F008EC10F027EC46F002EC77F058
:10A1400002E02ADF02D020BE209E2550200B06E030
:10A150000201235103E184ECF1F0259A02012A5116
:10A1600002E022EC3BF00101B35111E1E66A60EC40
:10A170002AF0E552006E1EAC39EF57F00701C851C6
:10A18000F00BE83AC85D0024C86F39EF57F0B3050B
:10A190000DE18CEC6CF093EC25F026EC17F01F929F
:10A1A000E8A039EF57F01F8239EF57F0020EB35D88
:10A1B00004E1E3ECE0F039EF57F0030EB35D07E1A3
:10A1C0002FB439EF57F0FFECE5F039EF57F0040EFC
:10A1D000B35D01E0B2D00201245102E039EF57F043
:10A1E0001850100B06E11850010B03E11850200B1A
:10A1F00002E0000E01D0010E2390E8B0238022AAD5
:10A2000044D0E9EC78F023A036D00101A6512AE130
:10A21000090E165C17E1E5EC75F014E10101A75198
:10A220000BE1A00E186E61EC08F000093CE037EC81
:10A2300077F039E11B8637D0175035E1A76B900EC8
:10A24000186E1FD0175002E1010E01D0100E8009C8
:10A25000186E61EC08F0000926E037EC77F023E196
:10A260001B8421D017501FE1A76BA7C1A6F1810E57
:10A27000186E229A06D0175016E12350010B13E1F5
:10A28000229A0201020E246F0ED032B40CD0E66A7C
:10A290005DEC3BF0E552000906E032840201020E5B
:10A2A000246F08AE246B3250040B02E139EF57F0F3
:10A2B0000201245102E039EF57F03294E9EC78F0D2
:10A2C000175002E139EF57F0A2EC04F00201C76B1E
:10A2D0000101280EA66F150E175C05E12150400BF9
:10A2E00002E01E0EA66F080E175C06E0290E175C32
:10A2F00003E0100E175C02E12D0EA66F0201020EA4
:10A30000246F228A186A1750166E61EC08F0000953
:10A310000BE001013751800B07E00201365104E1E7
:10A32000040E006ED6EC70F029B602D00101AA6BC3
:10A330007CEC0BF02B8439EF57F0050EB35D21E177
:10A34000FEEC76F00FE01C50080B0CE10CEC76F004
:10A3500009E20CEC76F006E202011E0E176FFAEC31
:10A3600076F0128401012751100B02E039EF57F00B
:10A370002851100B02E039EF57F022EC3BF039EF97
:10A3800057F0060EB35D07E121AA39EF57F0BDEC97
:10A3900006F039EF57F0070EB35D02E139EF57F0E1
:10A3A000080EB35D01E05ED32650800B0AE0020187
:10A3B000275107E1020E94EC7AF002011E0E276F7E
:10A3C000269E26AC03D043EC76F0269C26AA03D02A
:10A3D0008FEC09F0269A01013751800B1BE0020136
:10A3E000365118E11BA404D0040E94EC7AF01B94AF
:10A3F0001BA604D0070E94EC7AF01B961BA804D081
:10A40000060E94EC7AF01B981BAA04D0050E94EC6F
:10A410007AF01B9A0101B1BD93D0B1A959D021AEF8
:10A420000ED0A9516EE12CA805D00C50E66E85EC3B
:10A430003CF003D0E66AA5ECDAF0E55262D025A044
:10A4400003D05AEC4CF05DD02D50400B03E12D5061
:10A45000800B37E027AD55D090EC07F00101B251E9
:10A460001CE1630EE66E450EE66E010EF0EC78F030
:10A4700045C10CF202013B6BE66A90EC4AF0E552F2
:10A4800000091CE02D50800B19E001018F51100BC9
:10A4900015E10201100E3B6F11D0290EE66EB205D8
:10A4A0004C6A4B0F4B6E060E4C225CEC7AF068EC5B
:10A4B0007FF05FEC7CF07DEC79F0E5520101A96B57
:10A4C00020D022B61ED05CC200F0E5EC24F019D0FA
:10A4D000B1A305D026A215D02692238212D0B1A115
:10A4E00010D026A206D026922CC1E6FF3CEC31F01B
:10A4F000E5520201205105E11B50400B02E1B0EC96
:10A5000036F08BEC13F0006EFF081AE0540E005C7E
:10A5100007E1ADECE0F0220E006EE5EC24F010D087
:10A52000FF0E015C0DE0ADECE0F00101140E126FC6
:10A530000D0E136F050E006F0150006E90ECE6F0EB
:10A540000101B1BF77D2B1AB04D12DA603D09DECF0
:10A550003DF05AD231AC03D00DEC4DF055D230AABB
:10A5600005D024AA51D203EC4CF006D024AE06D07C
:10A5700024AA4AD287EC4BF0249AB5D025A003D068
:10A5800017EC4CF041D22DA403D070EC3DF03CD23E
:10A59000E2AF03D01EEC3DF037D21AA805D0010E71
:10A5A000E66EF5EC3CF0BDD03150040B1CE0D05110
:10A5B0001AE128AD0ED0010E0E6E28BF0E680A0EED
:10A5C000E66EEA0EE66E060E69EC73F0E66A4EEC95
:10A5D00074F02450200B04E101012851400B49E0A4
:10A5E00063EC4EF046D033A048D028AD1CD0010E0D
:10A5F0000E6E28BF0E680BC006F1030EE66E060E47
:10A60000E66E010EF0EC78F006C10BF07AEC7BF010
:10A610002C51615D06E10B5038EC74F0D815F31045
:10A62000D86FABEC4EF02450200B03E037EC77F002
:10A6300004E001012851400B1CE07CEC0BF0A0EC85
:10A640001DF0E66A4EEC74F0B1EC16F084EC4CF0C0
:10A65000020108811FBC09852050020B08E0E0ECD4
:10A6600077F005E02092E3EC0CF0A0EC2CF037EC56
:10A6700037F00101289D249A37D02D50400B03E17B
:10A680002D50800B33E024AA04D0249A7DEC79F07D
:10A6900048D028ADB9D1289D010E0E6E28BF0E6896
:10A6A000006A050EE66E0050E66EB20EE66E010E12
:10A6B00080EC73F00601030E426F0101B2510EE00F
:10A6C000B2294B6E010E4B5204E0E846FE0B4B06DE
:10A6D000FCE10601426F1E0E436F02D044EC4BF0CA
:10A6E0007DEC79F0E5520101A96B8ED121AE1BD032
:10A6F000A95101E089D10C50016E23A802D0DFECF2
:10A7000063F0006A2C50100B06E1010149517808F2
:10A7100002E2010E006E00504FEC76F0BFEC3CF010
:10A72000E552E55271D122B66FD15DC200F0F0EC76
:10A7300024F0A00E02015D5D01E066D197EC73F09C
:10A7400001E162D171EC74F001E05ED10101320EE1
:10A7500020D0B1B359D1B1A71ED01A50400B04E09C
:10A760001A50040B01E050D1BDECE0F00A0E006E6F
:10A7700048EC24F00101040E016F03C700F01AAC8D
:10A7800002D0AAEC04F0ADECE6F01AAC3DD1010128
:10A79000200E1B6F39D13CAB21D1070E006E00504B
:10A7A000D880775501E2776B28AD10D0289D010E37
:10A7B0000E6E28BF0E680050E66E770EE66E010E34
:10A7C00069EC73F00601426B0101A96BA95101E02C
:10A7D0001BD12150200B01E117D10201C75101E02B
:10A7E00013D1070E0101775D46E1BDECE0F026ECE8
:10A7F00015F001012B0E176F000110AE0BD00101F7
:10A800002D0E176FFF0ED8800F561056010E0F2613
:10A81000000E1022E70E30EC79F004E2E70E0F6E26
:10A82000030E106E0F50101003E10101200E176F80
:10A83000AAEC7AF0640E446E456A7BEC7CF002EC84
:10A84000FAF03BC04BF03CC04CF04B50006E0101A5
:10A85000012BADECE6F097EC04F0300F0101186F1E
:10A86000300E185D02E1200E186F1A8F640E1B6FF8
:10A87000420E1C6FA5D0060E775D1EE1BDECE0F028
:10A8800023EC15F071EC75F00101410E176F460EC7
:10A89000186F560E196F300E1A5D01E0B5D0200EFC
:10A8A0001A6F300E1B5D01E0AFD03EEC7BF001E093
:10A8B000ABD0200E1C6FA8D0040E775D03E0050E10
:10A8C000775D3DE1BDECE0F00101500E176F410EE8
:10A8D000186F4AEC78F0D0C73FF0D1C740F027ECB2
:10A8E0007BF0050E0101775D0EE14F0E176F530EE1
:10A8F000186F430E196F4AEC78F0CEC73FF0CFC700
:10A9000040F027EC7BF0049000AE02D0006C048095
:10A910000101030E016F73EC76F004A002D02D0E3E
:10A920001A6F430E1D6F050E775D6EE15851100BC7
:10A930006BE05851200B68E02A0E1A6F65D077053E
:10A9400014E1BDECE0F0160EE66EE60EE66E010ECA
:10A950009CEC7BF00BC200F0D2EC79F001011A5DA7
:10A9600002E1200E1A6F1C8F2BD0020E775D2BE1B7
:10A97000BDECE0F00E0EE66EE60EE66E010E9CEC0F
:10A980007BF00101845140E034AE02D02A0E196FF1
:10A99000060EE66E820EE66E17ECEFF0E552E5521B
:10A9A000006E005002010B5D006E0101030E016F8D
:10A9B000D2EC79F001011A5D02E1200E1A6F1C8FB2
:10A9C000560E1D6F21D0030E775D03E17FEC0FF073
:10A9D0001BD0775119E1A2ECEEF016D0020118510C
:10A9E0000BE02850400B10E1140E0101A85D0CE2B1
:10A9F000770E44EC75F008D00101B1A105D024AA6E
:10AA000003D0249AE9EC31F08BEC13F0006EFF08D0
:10AA100011E0540E005C0AE18BEC79F0060EE66E54
:10AA2000E60EE66E010E9CEC7BF004D00050006E4A
:10AA3000F0EC24F00101A95101E01BD2140EA96F22
:10AA40000201595101E05907020E6B5D01E011D27C
:10AA5000300E0101B55D04E00C0EB55D01E009D2D8
:10AA6000268207D2090EB35D0AE106015051515DFD
:10AA700001E1FFD150C651F6F7EC3AF0FAD10A0ED7
:10AA8000B35D05E1E7ECE4F0B2ECE4F0F2D10B0EDB
:10AA9000B35D01E0EED1B45103E1B8EC10F0E3D1C5
:10AAA000B4054DE160EC77F001E3DDD135EC0FF05A
:10AAB00060EC77F001E3D7D11C50080B01E0D3D153
:10AAC000E7EC77F015E2D10E44EC75F0AEECE4F073
:10AAD000320EE66E20EC0DF0E552FA0EE66EE50E53
:10AAE000E66E010EE66E37EC13F0E552E552BAD190
:10AAF000C80E3AEC7CF012EC12F00701A80E35EC0F
:10AB00007CF00DE2E90EE66EE50EE66E010ED0EC8D
:10AB100073F0E10EE66EE50EE66E010E98D0760E4D
:10AB200035EC7CF001E39FD1D00EE66EE50EE66ECB
:10AB3000010ED0EC73F0D10E44EC75F0CDD0020EC6
:10AB4000B45D01E0CDD035EC0FF0FEEC76F001E124
:10AB50008AD02150040B01E086D02150400B01E047
:10AB600082D05E0EDE6E010EDD6E65EC78F004E3E1
:10AB7000900EDE6E010EDD6EC1EC73F001E373D159
:10AB80001C50080B01E06FD135EC0FF0020E64ECA5
:10AB900073F0C1EC73F001E366D135EC0FF0050EF4
:10ABA00064EC73F0C1EC73F001E35DD12DA609D024
:10ABB00097EC73F003E071EC74F00AE082EC7BF048
:10ABC00007D00101675181EC79F0675F14EC50F018
:10ABD000460E3AEC7CF0C1EC73F001E344D1170E61
:10ABE000D5EC73F02DA609D097EC73F003E071EC6F
:10ABF00074F011E082EC7BF00ED0B80EE66EE50E3C
:10AC0000E66E010ED0EC73F00101675153EC7CF05D
:10AC1000675F14EC50F0960E3AEC7CF03EEC7CF062
:10AC2000320E4B26000E4C220201EF514B5CF051CC
:10AC30004C5801E318D1A50EE66EE50EE66E010E46
:10AC4000D0EC73F09D0EE66EE50EE66E010E8AEC1A
:10AC500078F0A7EC0FF0010EE66EB6EC0FF0E552BF
:10AC6000E1EC0FF000D148EC50F0000901E1FBD01D
:10AC70001C50080B01E0F7D035EC0FF048EC50F019
:10AC8000000901E1F0D0170ED5EC73F0AEECE4F062
:10AC9000E7EC77F009E28F0EE66EE50EE66E010E48
:10ACA000D0EC73F0320E0BD049511E080EE2810E2B
:10ACB000E66EE50EE66E010ED0EC73F01E0EE66E4B
:10ACC00020EC0DF0E552640E8AD06E0EE66EE50EB5
:10ACD000E66E010ED0EC73F0219451EC79F0C3D004
:10ACE000030EB45D36E1060150932550020B14E1CA
:10ACF0002050020B04E03AEC28F000090BE013505E
:10AD0000080B03E11350040B07E002014351421109
:10AD1000411102E0060150832550020B01E0A3D04F
:10AD2000D0EC77F001E09FD002012F5101E09BD0E1
:10AD30007FEC76F001E14C5001E195D02D50800B75
:10AD400001E091D02D50400B01E08DD00601018132
:10AD50008AD0040EB45D4FE15751040B4AE02050F5
:10AD6000080B47E0FEEC76F044E0B6EC79F041E108
:10AD70003BEC77F03EE1D70E96EC75F02BBC25D07E
:10AD8000DDEC7AF004E68F0E4B5C000E4C586BE263
:10AD9000140E64EC73F0D70E96EC75F00050016E53
:10ADA000050E64EC73F0D70E96EC75F0040E4FECC4
:10ADB00076F00050E66ECAEC75F055E02B8CDAECBC
:10ADC0000AF00201090E346F4ED08FEC7BF00BE2DB
:10ADD0004B508F08000E4C5406E22B9C140EE66E6E
:10ADE00008EC20F03FD0020134513DE1DAEC0AF0EA
:10ADF0003AD02B9C38D0050EB45D35E1A30E96EC0D
:10AE000075F00101E1A105D00050E66E2EEC71F065
:10AE1000E55204902250020B01E00480C00E005C59
:10AE200002E2229204D00050F00801E22282225075
:10AE3000020B02E08F9001D08F800450010B4B6E0B
:10AE40002250020B01E0010E4B5C0DE0A2EC04F07D
:10AE50007DEC15F014EC50F035EC7BF0010EE66E55
:10AE600019EC1CF0E5520101B42BB451050801E2C4
:10AE7000B46B0101B32BB3510B0801E2B36B020EAB
:10AE8000E15C02E2E16AE552E16E2AEF73F0016AE9
:10AE9000700E015C0DE2CF0E4B6EAD0E4C6E010ECE
:10AEA0004D6E01500FEC7AF06DEC78F0012AF0D77E
:10AEB0001200026A400E025C08E2B00E0224016E2B
:10AEC000320E6DEC78F0022AF5D7120043EC7BF0DD
:10AED000060F016E040E4FEC76F0A00EE66E020E29
:10AEE0003DEC73F00A6A2AEF73F043EC7BF0060F37
:10AEF000016E040EE66EA00EE66E020EFCEC7AF019
:10AF00002AEF73F043EC7BF00A0F016E020E4FEC58
:10AF100076F0A40EE66E020E3DEC73F00A6A2AEF9C
:10AF200073F043EC7BF00A0F016E020EE66EA40E86
:10AF3000E66E020EFCEC7AF02AEF73F0D6EC79F0B4
:10AF4000700EF4EC78F0010E0A6EDF6A100EDF5C12
:10AF500042E2026A100E025C3CE26FEC7AF003E01F
:10AF6000050E025C06E1DF50E824800FE0EC75F08E
:10AF7000006E020403E0060E025C07E1DF50E824E5
:10AF8000800F010FE0EC75F0006E020EDF5C03E352
:10AF9000030EDF5C0AE10A0E025C02E1110E006E94
:10AFA0000B0E025C02E1240E006E0C0E025C05E149
:10AFB0000A0EDF5C02E11B0E006E0D0E025C05E165
:10AFC0000A0EDF5C02E1200E006E77EC38F0022AF8
:10AFD000C1D7DF2ABBD7020E0A6EDF6A090EDF5C1B
:10AFE00012E2026A100E025C0CE26FEC7AF003E0EF
:10AFF000050E025C02E11C0E006E77EC38F0022AAE
:10B00000F1D7DF2AEBD70A6A42DFDF6A200EDF5C66
:10B0100009E2100E006E800EDF24016E77EC38F02E
:10B02000DF2AF4D7DF6A0B0EDF5C03E242DFDF2AA0
:10B03000FAD7DF6A090EDF5C37E2DF28006E0038DE
:10B04000F00B006E090E0012DFCFE6FF80EC7AF005
:10B0500000C0EFFF73EC73F0EE52090EEF6E73EC6D
:10B0600073F0020E0FEC75F02C0EEF6E73EC73F0B4
:10B07000030E0FEC75F0010EEF6E73EC73F0040E1F
:10B0800040EC7AF0050E40EC7AF0070E40EC7AF0D6
:10B09000080E40EC7AF0060E40EC7AF0090E0FEC48
:10B0A00075F0EF6ADF2AC6D720D82AD8DF6A060EE5
:10B0B000DF5C0EE2DF5002E1030E01D0010EE66E0E
:10B0C000DF50F2EC73F0E552E750EF6EDF2AEFD776
:10B0D0006AEC7CF0FD0E016EDB0E6DEC78F0010188
:10B0E000010EB16FE5522AEF73F0020E0A6E5A0E8E
:10B0F000E66E000EE66E030EE66EA20EAEEF7CF07C
:10B10000D6EC79F0DF6A030E0A6EFE0ED6EC74F010
:10B110000A6A850E005C02E0010EDF6E690EF4EC37
:10B1200078F0140EEBEC77F0000EE66E0A0EADEC44
:10B1300073F00A0EEBEC77F0CA0EE66E0A0EADEC79
:10B1400073F0040EEBEC77F0260EE66E0A0EADEC13
:10B1500073F0DF501DE00F0EEBEC77F0140EE66E8F
:10B160000A0EADEC73F0030EEBEC77F0230EE66EF7
:10B170000A0EADEC73F00A012D0E1B6F1BCA1AFAF2
:10B180001BCA19FA410E206F20CA1FFA20CA1EFAE4
:10B190000A01D46BDA6BDA81D56B380ED66F040EE8
:10B1A000D86F3C0ED96F190ED76F016A020E015C81
:10B1B0000CE20150050D47EC7BF0000EE9260A0E6B
:10B1C000EA22360EEF6E012AF1D70101D06B050E8F
:10B1D000D05D18E20701010ED66FFF0ED65D0FE0BD
:10B1E000A3EC12F064EC7AF056EC79F00701D6513A
:10B1F000EDEC73F03DEC75F00701D607EED70101D9
:10B20000D02BE5D70701D66B0101D06BDFCFE6FF6E
:10B21000E2EC45F0E5521AEC46F0030E0A6EFE0E23
:10B22000016E850E6DEC78F00A6AE5522AEF73F034
:10B230000490049201013FB104803FB304820450A2
:10B24000010B02E08E8E01D08E9E0450020B02E0B4
:10B250008F8801D08F984151E8240A0FE66EE66A84
:10B2600060ECF8F0E552E5520C0EBB6E006A01018D
:10B270003F5104E1100E4003F350006E0050BC6ECD
:10B28000120025EC73F015EC7AF055ECF9F0E5526C
:10B29000000902E0C69EF7D72AEF73F0C79EC69852
:10B2A000C78C1200C78EC688C78C1200F29E080E8B
:10B2B000E66E0A0E4CEC7BF0E66AE66A480E43EC5A
:10B2C00074F0E66A010E4CEC7BF00701146BF90E8A
:10B2D000156F14C7E6FF120E4CEC7BF015C7E6FFA6
:10B2E000130E4CEC7BF0F28E1200D9CFE6FFE1CFCB
:10B2F000D9FF030EE126EBEC0EF0E668930EE66E46
:10B30000B9ECF8F0E552E552AA9EC26A00000000CE
:10B310000000000000008A8A219A3488288ABAEC4A
:10B3200012F00601B66BB76B05EC0CF0F1ECF0F027
:10B3300084ECF1F089888F0EE66EE668DAECF6F0C0
:10B34000E552E552CF0EE66EE6682BECF8F0E552DA
:10B35000E552050EE66E73ECF9F0E5520101010EBF
:10B360003F6F0101030E406F0101020E416F60DF6C
:10B37000E668870EE66E8FECF8F0E552E552B09E77
:10B380000201320E116F000EA56EA26E9F6EA28298
:10B39000D08E010EC26EC16A0A0EC06E0F01DF0EA2
:10B3A000256F0F01F70E246F0F01E00E236FDB0EE8
:10B3B000006E02EC24F000C04EF5010EDB6A100EA8
:10B3C000F36E010EDBCFF4FFF350F45C28E2B00E15
:10B3D0004B6EAF0E4C6E010E4D6E010EDBCF4EF07C
:10B3E0004F6A506A4B504E24F36E4C504F20F46E0F
:10B3F0004D505020F86EF4CFF7FFF3CFF6FF080062
:10B40000F550E66E010EDB50EA6AC50FE96E060ED6
:10B41000EA22E552E750EF6E010EDB2AD0D7010198
:10B42000276B010127918850010B01E02781010161
:10B4300027938850020B01E02783F28E06015069A2
:10B44000F7EC3AF05FECE6F00101020EAE6F8D0E04
:10B45000AF6F010EB06F020197690601506BF7ECF8
:10B460003AF00101010EB16FADECE0F0BDECE0F09F
:10B4700005EC6BF0060117810601416941C640F6F3
:10B480000601426B148A1380128812821486148873
:10B490000A01380ED66F0A01010ED76FCFEC17F0F4
:10B4A000B2ECE4F07CEC1EF0010EE66E5DEC3BF0DD
:10B4B000E552176E200E175C0AE101013989010E71
:10B4C000E66E5DEC3BF0E552000901E0F8D7640E52
:10B4D000E66EA7ECF9F0E5521D9E84ECF1F00A6AE5
:10B4E000FC0E016EBCEC38F0001CDF6EFC0E016E31
:10B4F000DF50006E77EC38F0FC0E016EBCEC38F0DB
:10B50000DF50005C06E01E0EE66E4CEC13F0E552D8
:10B510004ED0830E0A6EFC0E016EBCEC38F0001C9F
:10B52000DF6EFC0E016EDF50006E77EC38F0FC0E23
:10B53000016EBCEC38F00A6ADF50005C06E0210EB8
:10B54000E66E4CEC13F0E55232D0FD0E016EBCEC11
:10B5500038F0DB0E005C03E1210E175C02E1EEDC4B
:10B560001ED0020E016EBCEC38F000C02BF1370E7D
:10B57000016EBCEC38F000C060F1110E016EBCEC45
:10B5800038F000C03AF1120E016EBCEC38F000C089
:10B590003BF10F0E016EBCEC38F000C038F1E00E4C
:10B5A000016EBCEC38F00050800801E282DC328889
:10B5B0000701580E836F020E846F0701B0697CEC9F
:10B5C0000BF0BBEC1CF084ECF1F02A9E22EC3BF07B
:10B5D00020860001126A136A146A156A800E086ECA
:10B5E000186A229A700EE66EE66A290EE66E010E61
:10B5F000E66EE7EC38F0E552E552E552E552020E10
:10B600000A6E5A0EE66EA20EE66E000EE66E030E8F
:10B61000E66EE7EC38F0E552E552E552E552030EEE
:10B620000A6E2A0EE66EE66A000EE66E0A0EE66EF8
:10B63000E7EC38F0E552E552E552E552AA0EE66E27
:10B64000300EE66E2A0EE66E0A0EE66EE7EC38F075
:10B65000E552E552E552E552FE0E016EBCEC38F0C3
:10B660000A6A850E005C01E04BDD060EE66EF00E08
:10B67000E66EDD0EE66E070EE66EE7EC38F0E5529C
:10B68000E552E552E552040EE66EA00EE66EEA0EB5
:10B69000E66E060EE66EE7EC38F0E552E552E5524E
:10B6A000E5520601EA510A0802E20601EA6B0601C8
:10B6B000EC51010802E20601EC6B200EE66E800EF2
:10B6C000E66E850EE66E070EE66EE7EC38F0E552A4
:10B6D000E552E552E552060EE66EF60EE66E470EB0
:10B6E000E66E050EE66EE7EC38F0E552E552E552FF
:10B6F000E552830E0A6EF90E016EBCEC38F000C004
:10B7000074F202017451DA0803E20201DA0E746F76
:10B71000F80E016EBCEC38F0349C6E0E005C01E15A
:10B72000348CDF0E016EBCEC38F00101DF91720E3B
:10B73000005C02E10101DF817E0E0A6E080EE66EFA
:10B74000E66AD80EE66E020EE66EE7EC38F0E552D9
:10B75000E552E552E5520A6A1C0E175C10E1010140
:10B76000378F0101378D0101379137833795010EEE
:10B77000E66E5DEC3BF0E552000901E0F8D7090EFA
:10B78000175C09E11C86010EE66E5DEC3BF0E552AC
:10B79000000901E0F8D701018151060802E2010128
:10B7A000816BE2EC04F0A9EC0BF001018EAB06D04A
:10B7B00001013D9F01013D9D01013C9F01010101EE
:10B7C0005851200B07E0010101015851100B02E113
:10B7D0000101589BD8C201F0DFC202F0FF0E015CEC
:10B7E00007E0015005E0FF0E025C02E0025008E1B4
:10B7F00002017C0ED86F0201FA0ED96F54EC4BF0A7
:10B8000001018451050802E20101846B01018551A7
:10B81000020802E20101856B0101435104E00101CC
:10B820004351020803E20101020E436F01016E5110
:10B83000230803E201010A0E6E6F0101608D010110
:10B84000515104E0010151510D0803E20101010EC3
:10B85000516F0601EA510A0804E20601EA6B06018B
:10B86000EB6B0101CB970101588301012F6B460E51
:10B870000101535D04E301015351730803E2010127
:10B88000640E536F01015651150804E3030E0101C4
:10B89000565D03E20101150E566F040E0101485D6D
:10B8A00004E301014851080803E20101050E486F55
:10B8B00001017E514B6E4C6AD8904C5004E6C80E84
:10B8C0004B5C000E4C5803E20101D70E7E6F010164
:10B8D0004E514B6E4C6A4C3404E24B509608000EAD
:10B8E0004C5403E201018C0E4E6F01014D513208A0
:10B8F00003E20101280E4D6F01014C514B6E4C6A61
:10B900004C3404E24B50C808000E4C5402E20101D2
:10B910004C6B0A0E0101425D04E3010142510F0824
:10B9200003E201010F0E426F01013651280803E2C4
:10B930000101010E366F01012951280803E20101BE
:10B94000280E296F550E01014F5D07E0680E0101B9
:10B950004F5D03E00101680E4F6FFF0E01016A5D4C
:10B9600003E001016A5109E10101C80E6A6FD90EB5
:10B970006B6FCF0E6C6F060E6D6F01017851010871
:10B9800002E20101786B010167513C0802E201010A
:10B99000676B010168513C0802E20101686B01011B
:10B9A0006951280802E20101696B010101018E5110
:10B9B000020B05E101013B5102E001018E8301010F
:10B9C0006251030802E20101626B2CC161F10101C5
:10B9D0006151180803E20101030E616FFF0E0101BE
:10B9E000605D02E10101606B010172514B6E4C6AB6
:10B9F0004C3404E24B50C808000E4C5403E20101E1
:10BA0000C80E726F010174514B6E4C6A4C3404E2E3
:10BA10004B50C808000E4C5403E20101280E746F0D
:10BA2000010173514B6E4C6A4C3404E24B50C80810
:10BA3000000E4C5403E201010C0E736F01017651AC
:10BA40004B6E4C6A4C3404E24B50C808000E4C5408
:10BA500003E201011E0E766F01013251020803E27A
:10BA60000101010E326F3C0E0101E76E7D19E8AE57
:10BA700002D07D3503D0E750D8807D550BE3C40E4E
:10BA80000101E76E7D19E8AE02D0E73402D0E7503D
:10BA90007D5D02E201017D6B01017C513C0802E207
:10BAA00001017C6B01016F513C0802E201016F6BE7
:10BAB000010170513C0802E20101706B0601EB517B
:10BAC0001E0802E20601EB6B0601ED511E0802E2C0
:10BAD0000601ED6B01018051640803E201011E0EB5
:10BAE000806F01012A514B6E4C6AD8904C5004E68D
:10BAF000280E4B5C000E4C580BE301012A514D6E91
:10BB00004E6A4E3404E24D504608000E4E5403E295
:10BB10000101370E2A6F01018651DA0802E20101A4
:10BB2000866B2A50800B07E101018651780803E2F9
:10BB30000101780E866F02019A5104E002019A51C8
:10BB4000320803E202010D0E9A6F010187510C08C1
:10BB500002E20101876B01018851640803E20101DF
:10BB6000460E886F01019451140803E201010C0E86
:10BB7000946F01019651140803E201010C0E966FB7
:10BB80000501475150080EE20501280E4A6F4AC5CB
:10BB900047F50501050E4B6F4BC548F505014C6B8C
:10BBA0004CC549F5010189511E0802E20101896B6A
:10BBB00001018BAF02D001018B6B01018EAF02D06E
:10BBC00001018E6B01018FAF03D001010A0E8F6F4F
:10BBD000010197AF03D00101600E976F1E0E0101A6
:10BBE0008A5D04E301018A51280805E201011E0E65
:10BBF0008A6F01018B9101018C510A0802E2010157
:10BC00008C6B01017B51190804E201017B6B01017E
:10BC10008B930101715104E0010171511E0803E28F
:10BC200001011E0E716F01013F51010803E2010184
:10BC3000010E3F6F1E0EE66EC7EC12F0E5520009D2
:10BC400009E00101010E3F6F0101030E406F010188
:10BC5000020E416F18EC59F005014F698FEC09F0A5
:10BC60000101DF8301012A51E8240301D06FDAECDE
:10BC70001FF0300E010185250401F76F020E01014E
:10BC8000855D03E10401340EF76FE4ECAEF00401CE
:10BC90003B0EFE6F0501106B10C512F510C511F5B6
:10BCA0000501800E156F27ECEAF041ECEAF04DEC4F
:10BCB000EAF0000905E12A0EE66E4CEC13F0E552BD
:10BCC00007013C0EA56F0101D16BD1C1D0F1070175
:10BCD000D66B010EE66EA3EC70F0E5520701E3812E
:10BCE000076A7CEC0BF0BCEC1CF014EC50F02FEC71
:10BCF00050F00101010139510701099F040B01E0D6
:10BD0000098FE7EC1EF0A7ECF0F0A6DA84ECF1F076
:10BD1000B8EC10F0F3CF0FF0F4CF10F0430E0F5C3F
:10BD2000010E105806E3D30ED8800F54020E1054A3
:10BD300011E20FC04BF010C04CF0040ED8904C3202
:10BD40004B32E804FBE14BC026F7570EE66E4CEC95
:10BD500013F0E55212EC12F0F3CF0FF0F4CF10F025
:10BD60001F0E0F5C010E105806E3D30ED8800F543F
:10BD7000020E105411E20FC04BF010C04CF0040E34
:10BD8000D8904C324B32E804FBE14BC026F75A0EF8
:10BD9000E66E4CEC13F0E552550EE66E020EE66EC2
:10BDA000400EE66EC7ECF0F0E552E552E552AA0E01
:10BDB000E66E020EE66E420EE66EC7ECF0F0E5525D
:10BDC000E552E552020EE66E400EE66E13ECF1F01F
:10BDD000E552E552550802E1000E01D0010E006E59
:10BDE000005007E000C026F75D0EE66E4CEC13F045
:10BDF000E552020EE66E420EE66E13ECF1F0E552ED
:10BE0000E552AA0802E1000E01D0010E006E0050BA
:10BE100007E000C026F7600EE66E4CEC13F0E5522A
:10BE20000101845116E016ECEFF000090AE0A6ECDF
:10BE3000EDF005ECEEF001018451010801E2348ED1
:10BE400008D00701050E266F1B0EE66E4CEC13F0B2
:10BE5000E5524DECDAF02C9601013B515CE0150EF9
:10BE6000E66E020EE66E440EE66EC7ECF0F0E552AA
:10BE7000E552E5522A0EE66E020EE66E460EE66EBC
:10BE8000C7ECF0F0E552E552E552020EE66E440EC4
:10BE9000E66E13ECF1F0E552E552150802E1000EF2
:10BEA00001D0010E006E005008E000C026F7630EBE
:10BEB000E66E4CEC13F0E5522ED0020EE66E460E06
:10BEC000E66E13ECF1F0E552E5522A0802E1000EAD
:10BED00001D0010E006E005008E000C026F7660E8B
:10BEE000E66E4CEC13F0E55216D0120EE66E440EE0
:10BEF000E66E13ECF1F0E552E552006EC00E00164E
:10BF0000005008E000C026F7810EE66E4CEC13F0FE
:10BF1000E55201D02C8656EC59F01C920101955146
:10BF20001FE0370EE66E020EE66E480EE66EC7ECB8
:10BF3000F0F0E552E552E552020EE66E480EE66E6E
:10BF400013ECF1F0E552E552370809E00701010E64
:10BF5000266F180EE66E4CEC13F0E55201D01C82F1
:10BF60002680E6685FEC33F0E552C1EC1FF001017A
:10BF7000B181229401013CBB06D006015095060117
:10BF80005087F7EC3AF00101D05104E0030E0101B3
:10BF9000D05D04E10A01D46B159C04D00A01020EA5
:10BFA000D46F158CA2D901012BBD0CD054ECEBF051
:10BFB000E8C26AF1E9C26BF1EAC26CF1EBC26DF161
:10BFC00001012B8DA0EC2CF00201320E236F010138
:10BFD0000E0EB56F0501010E176F0901020EBC6F41
:10BFE00002015B2B0201320E216F55EC9AF0A2EC9C
:10BFF00004F00201F15108080AE2BAEC12F0F1C2B1
:10C0000026F7270EE66E4CEC13F0E5521C860D0E5B
:10C01000E66EC3EC13F0E552870B006E005008E0AB
:10C0200000C026F7390EE66E4CEC13F0E55214D042
:10C03000A8EC1EF03B0E0F5C000E105806E3E60E57
:10C04000D8800F54030E105407E20FC026F7540E89
:10C05000E66E4CEC13F0E552030EE15C02E2E16A9D
:10C06000E552E16EE552E7CFD9FF1200400E010123
:10C07000B55D03E3B551450801E2000C010C010177
:10C080003C7B289D266B1DD8248A268201013CBB5F
:10C0900013D009014F0EBD6F460EBE6F060150A7AB
:10C0A00007D00901560EBD6F420EBE6F01013789E0
:10C0B0000601436B43C642F601013CBB048099EF85
:10C0C00008F006015097509501013CBB07D022B4FF
:10C0D00003D00601508512000601508712000A01A4
:10C0E000D6514DEF7CF0D0C100F0005003E0030EBC
:10C0F000005C35E100500EE10101CC7D0901430EE9
:10C10000BD6F0101CCAD02D099EC77F00101CCAD4F
:10C1100020D010D018EC76F00FE00101CC750901A9
:10C12000440EBD6F0101CCA502D099EC77F001015E
:10C13000CCA50FD004800DD00101CB750901440EB0
:10C14000BD6F0101CBA502D099EC77F00101CBB511
:10C15000048099EC08F037EC37F0B1EF16F00004EA
:10C1600003E0020E005C16E1A3EC12F0000402E111
:10C17000020E01D0010E006E09014C0EBD6F020EC1
:10C18000005C03E10480550EBD6F99EC08F000C01F
:10C19000D0F16BD812000101335103E197EC73F039
:10C1A00002E0000E01D0010E1592E8B0158297EC66
:10C1B00073F004E101013D51800B0CE197EC73F049
:10C1C00007E071EC74F004E101013C51800B02E1E5
:10C1D000000E01D0010E1590E8B01580120097EC0A
:10C1E00073F007E0CAEC79F004E192EC79F001E039
:10C1F000000C010CC2EC79F003E001018251120045
:10C20000010179511200C2EC79F003E00101835180
:10C21000120001017A51120025EC73F0C2EC79F0A2
:10C2200005E0FE0EDB500101826F04D0FE0EDB50F4
:10C230000101796F2AEF73F025EC73F0C2EC79F00D
:10C2400005E0FE0EDB500101836F04D0FE0EDB50D3
:10C2500001017A6F2AEF73F0D6DFE66ECBDFE66E70
:10C26000AFECF0F0E552E55212002290D0C100F0A0
:10C270000050800802E2050E006E060E005C01E32D
:10C28000006A000402E10101CB91020E005C02E1B0
:10C290000101CB8100C0D0F1258A21BE0AD03CEC3F
:10C2A00012F04BEC76F002E086EC05F0B1EC16F003
:10C2B00002D037EC37F09DEF23F0D6EC79F0030E87
:10C2C000DF6E01018FBDDF6A4A514B6E4C6AB00EC2
:10C2D0003F6E040E406E5CEC73F03F50D880DF542C
:10C2E0000201536FE5522AEF73F0D6EC79F027B0D4
:10C2F00012D0320EDF6E01018FAD02D0640EDF6E00
:10C30000080E4A5D02E2080E4A6FDF50D8804A5597
:10C3100002E2DFCF4AF1D1DFE5522AEF73F053C2D8
:10C32000ACF123AE44D0006A01013E510C0803E396
:10C33000070E3E5D02E20C0E3E6F070E3E5D4F6E35
:10C34000506A020153514D6E4E6A4DC03FF04EC0CF
:10C3500040F04FC044F050C045F093EC78F0140E1C
:10C36000446E456A33EC7AF04B50006EB4EC7AF0D0
:10C370000101AC514D6E4E6AFF0ED8804D56000E35
:10C380004E564C504E18E8AE02D04E3404D04D50AC
:10C390004B5C4E504C580BE20050D880AC5507E235
:10C3A00024A003D00050AC2702D00050AC5F3BEC7F
:10C3B00077F008E102012C510601EA1106E028504D
:10C3C000400B03E11E922AEC3AF01200050E56ECE7
:10C3D00078F0580EC6EF77F0F9DF268E1200180EAF
:10C3E000D5EC73F0010137AD03D0580EC6EF77F0EE
:10C3F000268E120025EC73F0050EE12620A20FD048
:10C40000BBC1DFFF010EBCC1DBFF020EBDC1DBFF04
:10C41000030EBEC1DBFF040EBFC1DBFF0ED0B6C1F1
:10C42000DFFF010EB7C1DBFF020EB8C1DBFF030E59
:10C43000B9C1DBFF040EBAC1DBFFDF5042E0DF040D
:10C4400004E1460ECDEC74F03CE30101E1BD07D000
:10C45000DF50180815E21C0EDF5C12E232D0190E14
:10C46000DF5C2FE01A0EDF5C04E1010EDB505F0899
:10C4700028E31B0EDF5C04E1290ECDEC74F021E310
:10C480002C50100B06E12F50800B03E02C510A08B2
:10C4900002E2F36A1BD0660EE66E020EE66ED9CF9C
:10C4A000E6FFDACFE6FF37EC76F00BE1D9CFE6FF17
:10C4B000DACFE6FF610EE66E020EE66E37EC76F03E
:10C4C00004E08DDF010EF36E01D0F36AF46A050E0D
:10C4D000E15C02E2E16AE552E16E2AEF73F065C3C6
:10C4E00001F023A802D078C301F00E0E015C01E236
:10C4F000010C100E015C01E2020C120E015C01E263
:10C50000030C140E015C01E2040C160E015C01E246
:10C51000050C1B0E015C01E2060C220E015C01E21F
:10C52000070C080C27EC7AF096EC75F00050F00838
:10C5300001E2006ADDEC7AF004E6BE0E4B5C000E10
:10C540004C580AE2960E4B6E8E0E4C6E010E4D6EDE
:10C5500000500FEC7AF001D0B00E0F6E106ADDECD7
:10C560007AF004E6AA0E4B5C000E4C580CE2EC0E7E
:10C570004B6E8D0E4C6E010E4D6E00500FEC7AF02E
:10C580000101D46F02D00101D469D56B2AEF73F099
:10C59000049035BA0480B30E43EC7CF0D4C161F34F
:10C5A000D5C162F335BA120014A634D00C50016E16
:10C5B00023B805D9050E01244B6E0A0EA2EC73F0C8
:10C5C000016E015005E12350400B02E0010E016EA7
:10C5D00097EC73F003E03550800B05E001C0CAF71B
:10C5E00002010A0E08D00701CA51015C05E301C02F
:10C5F000CAF702010C0E296F72DF0701CB6F2C50B6
:10C60000100B03E1040E0C5C01E2CB6BE9EC76F05D
:10C61000DCEC75F01CEC76F00480005009E035503D
:10C62000800B06E1030E005C04E1020E0B5C01E1ED
:10C630000490070E016E3250010B03E10450010B10
:10C6400004E0090E9BEC74F0016E0F0E0114020160
:10C65000766F32B002D0070E761701380F0B016EDD
:10C6600004A0016A14A408D0020EE66E76C2E6FFAA
:10C670000150E66EDCEC75F0010153514B6E4C6AD3
:10C680000AEC75F0AFEC7AF0A3EC7AF0640ED6EC1D
:10C690007BF00F500C6E1CEC76F0040E005C22E177
:10C6A000100E016E01504B6E4C6ACEC23FF0CFC2ED
:10C6B00040F05CEC73F03FC0D0F20C5093EC7CF097
:10C6C0000201CE274C50CF23D0514B6E4C6ACE5135
:10C6D0004B5CCF514C5806E2D05193EC7CF0CE5FCE
:10C6E0004C50CF5B000409E0020E005C06E0030E34
:10C6F000005C0AE1020E0B5C07E00201D151D88018
:10C700000C5402E20CC0D1F2B70E43EC7CF0D4C161
:10C7100063F3D5C164F303016151635D62516459F0
:10C7200006E3010E6325616F000E6421626F6151A3
:10C730006325676F62516421686F675167254B6E8F
:10C74000685168214C6E67C34DF068C34EF0030E0C
:10C75000D8904D364E36E804FBE14B504D24030192
:10C76000676F4C504E20686F6351615D4B6E625134
:10C7700064554C6EAFEC7AF067C33FF068C340F08D
:10C7800002ECFAF03FC067F340C068F367C365F39B
:10C7900067C34BF068C34CF04D6A4E6A4E34000ECE
:10C7A0004E1809E6D880FF0E4B54000E4C54000E74
:10C7B0004D54000E4E5402E203016569120049C156
:10C7C00001F02C50100B07E101014951780803E2F8
:10C7D0006C0E015C016E12001CEC76F000500DE056
:10C7E0003550800B0AE1050E005C07E0030E005C8B
:10C7F00003E1020E0B5C01E0000C010C0482ECDF93
:10C80000000901E00492358804A23598359AC0DE0B
:10C8100035BA12001CEC76F004980496030E005C06
:10C8200001E10486000403E0020E005C01E10488DB
:10C830002350400B01E1DBD02350100B01E0D7D097
:10C840003450100B01E1D3D002011C5101E0CFD0D4
:10C850001A50010B01E1CBD004820494BDDF000922
:10C8600001E00492040E005C01E10484A8DF0150A1
:10C8700053EC7CF0026E32A01CD002017651070806
:10C880000AE20150E840E840E8401F0B015C405DCF
:10C8900009E2402B07D0325105E1405103E0400747
:10C8A000040E326F4051D880015405E24051015EC0
:10C8B00002D00201406B04900450040B03E00250CC
:10C8C000D05D06E30450040B49E101500C5C46E2E4
:10C8D000880E015D130E025901E37AD003016C0E3C
:10C8E000635D000E645901E373D004B209D00C50AB
:10C8F000015C0F6E106A0F5002010127105005D025
:10C9000004A405D00201012B000E022360D0020115
:10C910001D515EE10A0E1D6F0150D15D1DE2D15126
:10C920001BE004A802D0020E1D6F0450080B0FE09C
:10C93000030E0B5C03E07651010809E20A0E0127A1
:10C94000000E02231E5107E01D911D4304D0020E6C
:10C950000127000E02230480D16B3AD00450040B4F
:10C9600004E00250D880D05507E30450040B30E1B6
:10C970000150D8800C542CE2010E036E04B407D091
:10C9800004A206D00A0E036E04A802D01E0E036E87
:10C9900003500F6E106A0450020B05E00450080BA0
:10C9A0000CE01E510AE001500C5C4B6E4C6AAFEC7F
:10C9B0007AF00AEC75F0A3EC7AF0020101510F5CF9
:10C9C0000251105805E20F50015F1050025B0480C5
:10C9D00004A00DD002010351011902E10451021912
:10C9E00006E0BCEC0AF001C203F202C204F202014A
:10C9F0001F5102E00F0E1F6F1200D6EC79F0DF6AB4
:10CA00001850100B0CE0200E165C47E0210E165C4F
:10CA100044E0150E165C03E192EC79F03EE018500C
:10CA2000010B09E0150E165C38E0220E165C35E0AD
:10CA30001D0E165C32E01A50200B12E10201185153
:10CA40000FE1230E165C29E00B0E165C26E0090EA2
:10CA5000165C23E0090E165C20E0220E165C1DE039
:10CA60006DEC07F0000904E061EC9AF0000915E1B3
:10CA70001D0E165C07E11850100B04E057EC17F080
:10CA800000090BE12150800B06E102016B5103E02C
:10CA90003350400B02E0000E01D0010EDF6EDF507C
:10CAA000E5522AEF73F0030E47EC79F08A8607010E
:10CAB0000B9154ECF1F075EC17F032EC0AF0000930
:10CAC00003E042EC15F002D034EC15F00601509171
:10CAD000F7EF3AF05EC249F15FC201F260C202F2C2
:10CAE000BCEC0AF00BEC22F0C1EF1FF00101AC51DD
:10CAF00003E12C820950086E2150010B12E097ECE3
:10CB000073F00FE11850800B03E0BEEC79F006E003
:10CB10002150040B06E183EC75F003E06ED943EC81
:10CB20006DF012000101050EAB6F2150010B04E006
:10CB30001A50020B01E0AB6B120025EC73F0040EEF
:10CB4000E12605C2DFFF22ECDBF0DF500201055DCC
:10CB500023E0010E69C3DBFF020E6AC3DBFF030E95
:10CB60006BC3DBFF010EE66EE3ECDBF0E552010E7A
:10CB7000DB500301695D08E1020EDB506A5D04E1F0
:10CB8000030EDB506B5D08E078ECDAF084ECF1F03A
:10CB90001D820101960EA86F040EE15C02E2E16ABB
:10CBA000E552E16E2AEF73F00201175107E0176BAF
:10CBB000FAEC76F00201F25101E112940101E199DF
:10CBC0004BEC76F002E00101E18997EC73F00AE1A9
:10CBD0002150010B07E101013D51800B03E1215080
:10CBE000800B0DE03BEC77F00AE11F50400B07E1B2
:10CBF000E5EC75F003E10101B50501E0238C23BCF0
:10CC000006D0E66AE66A740E38EC73F014D092EC43
:10CC100079F00FE101C24BF002C24CF0030E0F0B92
:10CC200003E044EC79F0FDE14B500201015F4C5010
:10CC3000025BBCEC0AF002010A0E1D6FD16B21AE43
:10CC40001D84C80E1E6F32EC0AF0000903E03BECB5
:10CC500015F002D02DEC15F0960E006E0050F5EC9C
:10CC600076F023EC17F00201216B8A96320EF5EC78
:10CC700076F0359023EC0EF0000901E03580A6EC4B
:10CC800073F01FE12C50080B11E02350100B0EE144
:10CC900001013B050BE097EC73F007E12150800B9D
:10CCA00004E102011E0E146F01D047DF3550010B65
:10CCB00008E0D0EC77F005E1A6EC73F002E107ECB8
:10CCC0000AF02150800B0EE12150010B0BE197EC93
:10CCD00073F008E03550800B05E102012C5102E0B1
:10CCE000050110511EAC02D0C3EC0AF0218C328237
:10CCF00035A002D08A964AD0D5CA98F21CEC76F0BC
:10CD0000360E026E380E036E0101E1B91AD0B6C1BB
:10CD100081F266EC77F040C082F229EC2DF0B6C1CA
:10CD20007FF266EC77F040C080F220A20AD0BBC14F
:10CD30007FF261EC7AF0BCC140F05CECFAF040C0EC
:10CD400080F223AC10D007010B8F0B8154ECF1F073
:10CD500065EC78F008E15851010B05E00701088FF8
:10CD6000089D88EC7BF00101E1B910D020A203D02E
:10CD70000701506B516B020181517F5D04E18251CB
:10CD8000805D01E12A84308E0FEC30F00201FA0E52
:10CD9000226F248A2682329223AC04D0060150816D
:10CDA000F7EC3AF0B0EC36F022AE11D0229EE3EC74
:10CDB00009F0D4EC7AF0E7EC79F009E0E7EC79F0EF
:10CDC00006E0E7EC79F003E0D6EC09F016D81200A3
:10CDD000D6EC79F0050123072451EA6A270FE96EA2
:10CDE000050EEA22EFCFDFFF242B24511F0801E2BA
:10CDF000246BDF50E5522AEF73F03AEC20F0020189
:10CE0000186B18C258F2C1EC77F007E0200E010150
:10CE10001D5D03E0200E48EC75F00101AC6B006A6B
:10CE2000D6EF70F0320E026E140E0301655D07E35B
:10CE300065EC78F019E11E0E0301655D15E22C50DA
:10CE4000100B04E0640E0101495D0FE02C50100B43
:10CE50000BE1280E0101495D08E03C0E495D05E04B
:10CE60006C0E0224495D01E0000C010CD6EC79F057
:10CE7000DF6A1C50080B0AE1E5EC75F009E1380E99
:10CE80000101B55D03E03F0EB55D02E1000E36D055
:10CE90000101825102E0835104E1450E51EC74F02E
:10CEA000DF2A0101795102E07A5104E1480E51EC88
:10CEB00074F0DF2AB7DF00091CE1AAEC32F00009A8
:10CEC00006E03C0E51EC74F006EC77F0DF2ABFEC84
:10CED00032F0000907E03F0E51EC74F00201A46B40
:10CEE000A56BDF2A0701E55104E1420E51EC74F015
:10CEF000DF2ADF5002E081DF2194DF50E5522AEF84
:10CF000073F0D6EC79F00850DF6E28AA03D0020146
:10CF10001E0E206F050110510201181103E1385156
:10CF2000391109E01E50040B0FE01E50080B0CE0F5
:10CF30001F50010B09E01850800B08E02850200B0F
:10CF400005E10501105102E058DF48D308501FE108
:10CF500028BA04D043EC76F0020E58D087DF0009DF
:10CF600001E03CD30201235101E038D321B002D0CB
:10CF70001BDE0AD02C5108E00501105105E1D0EC70
:10CF800077F002E143EC76F00101AB6BEAD00804E4
:10CF90001BE10101AB5101E01DD3209CA6EC73F015
:10CFA00002E0208C08D03550010B05E1D0EC77F081
:10CFB00002E107EC0AF00101280EAB6F21AE02D0AE
:10CFC000050EAC6F082A17D0020E085C16E10201AC
:10CFD000145102E01E0E146F28BA06D00101AC51A4
:10CFE00001E0F8D20950F5D20101AB5102E1FEECAB
:10CFF00063F011EC0AF07ADDEDD2030E085C36E145
:10D0000028BA06D0006AD6EC70F0070E086EE6D299
:10D010002CA212D05CC1ABF10101AB6B2C92215060
:10D02000010B04E01A50020B01E0AB6B02012C5122
:10D0300003E0006AD6EC70F00101AB5106E097EC1A
:10D0400073F00FE03550800B0CE12050400B05E1F0
:10D0500002012C5102E10CEC0AF00101280EAB6F29
:10D0600006D127B8B7D2FEEC63F0B4D2050E085C47
:10D070004AE10101AB5101E0ADD2082A279821B065
:10D08000A9D21C0E016EE1A902D0140E016E8751C7
:10D09000E8240124006E02017A5107E000507A5D15
:10D0A00004E2090E086E278895D2328207010B9F91
:10D0B00054ECF1F065EC78F008E15851010B05E013
:10D0C0000701089F088D88EC7BF0219C35B010D0BB
:10D0D00098C2D5FA3FECF1F00101E1B909D029EC91
:10D0E0002DF020A203D00701506B516B0FEC30F0F4
:10D0F00097EC73F003E03550800B03E00101050E5F
:10D10000AB6F329267D2060E085C2DE10101AB5184
:10D1100001E060D221B023D02750100B0EE1335133
:10D120000AE097EC73F003E03550800B04E0010156
:10D130003D51800B02E1B7DC12D033C121F227A8A8
:10D140000ED0050EB4EC7CF087C140F095EC7BF07E
:10D15000006E00500201215D02E200C021F20201D6
:10D16000596B082A37D2070E085C24E10101AC5143
:10D170000FE118AE0BD0BEEC79F003E01AEC9BF097
:10D1800005D065EC0AF0000901E0189E0950086E10
:10D1900002012C5101E01ED2295106E03550800BCE
:10D1A00003E1E9EC76F003D0E66AE66AE66AFDECB4
:10D1B00026F047D0080E085C4BE10101AC5106E0B7
:10D1C0001E50040B03E01E50080B02E10950086ECC
:10D1D00002012C5101E1FED1FEEC63F011EC0AF0EA
:10D1E00002012D5101E0F6D12EEC0DF0000901E114
:10D1F000F1D10501020E266F235111E0E9DD006E29
:10D20000020E0B5C02E1005010D0016A05012351AF
:10D2100002E0DEDD016E00504FEC76F00ED01051D2
:10D2200014E1020E0B5C07E1030EE66E150EE66ECE
:10D23000E8EC14F007D0E66AE66A160EE66EEEEC4D
:10D2400014F0E552E552E552C5D102012C6BC2D172
:10D25000090E085C2EE102017A417F0B7A2501015B
:10D26000D880AD5506E202017A6B7AC2ADF1050EA7
:10D27000B0D11FB0AFD1010EAD6F320EAB6FE1A9CF
:10D2800002D0280EAB6F010E086E97EC73F006E02B
:10D2900002012C5103E13550800B08E0D0EC77F00F
:10D2A00005E12850200B02E143EC76F00B0E096EED
:10D2B00091D10A0E085C06E122BA9FD0189E0B0E8F
:10D2C000086E9DD00B0E085C01E09CD01850800BBE
:10D2D00039E12150010B06E02150040B03E183ECFE
:10D2E00075F030E197EC73F003E03550800B0CE003
:10D2F0002150800B09E11F50010B06E01E50040B6A
:10D3000003E01E50080B1EE197EC73F00CE0355063
:10D31000800B09E12150040B06E183EC75F003E07A
:10D32000D4EC77F00FE02150800B09E01E50040B85
:10D3300009E01E50080B06E083EC75F003E0A6EC54
:10D3400073F051E018AE0ED0BEEC79F005E01AECA7
:10D350009BF0000907E142D165EC0AF0000902E008
:10D36000189E3CD197EC73F023E03550800B20E100
:10D3700071EC74F01DE11AAA06D0D6EC09F078EC35
:10D3800007F0DCEC1BF03BEC77F00AE01A50400BA6
:10D3900007E0259224BC2582D6EC09F01AEC77F040
:10D3A0000101895105E089C1E6FF08EC20F0E55252
:10D3B000ADC17AF20101AD5102E0010EAD6F27A8B7
:10D3C00002D0FEEC63F00701C86B030E086E800EFE
:10D3D000096E2150800B03E11850800B08E0219466
:10D3E0000C0E096E04D023A802D0A1ECDCF00101E0
:10D3F000AB5105E12750100B02E1FEEC63F011EC9C
:10D400000AF0E8D00C0E085C01E0E4D022BAE2D0C9
:10D41000D3EC9CF021AEDCD01E50040BFDE01E507E
:10D42000080BFAE02B840101B19B248AB199268272
:10D4300099510BE020A203D099C1D1F102D099C13A
:10D44000D0F129EC2DF035EC61F023A803D06AEC83
:10D4500065F097D0E7DC000901E18ED031EC12F0E5
:10D4600001C20FF002C210F00FC04FF010C050F018
:10D470000FEC74F039C035F73AC036F73BC037F7D8
:10D480003CC038F761EC7AF00BC240F095EC7BF0D1
:10D49000006E0050536E546A556A566A00504F6EC3
:10D4A000506A516A526A4FC03DF050C03EF051C0C0
:10D4B0003FF052C040F053C042F054C043F055C05A
:10D4C00044F056C045F0F3ECF7F039C04BF03AC0E9
:10D4D0004CF03BC04DF03CC04EF0EBEC74F0F3EC84
:10D4E000F7F03CC0EDFF3BC0EDFF3AC0EDFF39C0A7
:10D4F000EFFFC40E426E160E436E020E446E456A76
:10D5000035C73DF036C73EF037C73FF038C740F06B
:10D5100031ECF9F03DC035F73EC036F73FC037F784
:10D5200040C038F749C14BF04C6A4D6A4E6AEBEC8B
:10D5300074F031ECF9F040C0EDFF3FC0EDFF3EC0AC
:10D54000EDFF3DC0EFFF070135513611371138119E
:10D550000EE0C80E355D000E3659000E3759000E2C
:10D56000385905E235C700F077EC38F005D035C7FB
:10D5700026F74B0E51EC74F019A803D06AEC65F055
:10D580001998219E4BEC76F003E13450080B03E030
:10D5900037EC37F005D0010EE66EC0EC36F0E55200
:10D5A000239877EC75F0010137BF04D0050E94EC99
:10D5B0007AF00ED037AD0CD0DF85E383E395E397A7
:10D5C0000601FB29FC6F65C3E6FF0DEC09F0E5528F
:10D5D000800E086EDF50085C01E01D8CE5522AEFDA
:10D5E00073F03050100B0FE1070176510CE101018F
:10D5F000B151200B08E13C51200B06E0E5EC75F041
:10D6000003E0C75101E1000C010C070EE66EE66A6B
:10D61000200EE66E440EE66E060EE66EC0ECF6F0E8
:10D62000050EE15E120045C644F646C645F647C6FD
:10D6300046F648C647F649C648F64AC649F61200B5
:10D6400049C64AF648C649F647C648F646C647F6AA
:10D6500045C646F644C645F60601200E446F120044
:10D6600025EC73F032AA02D08EEC78F00101E15182
:10D67000020B0CE0280E0901BB5D08E2BB51BB2B7D
:10D68000EA6A930FE96E090E10EC7CF02AEF73F052
:10D69000E0EC79F0010EDB6A1B50010B0AE0800E12
:10D6A00058EC73F004E2FE0EDB50200802E11B9000
:10D6B0005CD0B9DFFE0EDBCF4AF6DB50800804E019
:10D6C000850E58EC73F003E30601200E21D0FE0E08
:10D6D000DB50300803E10601630E1AD02A50200BFC
:10D6E0001CE02950080B19E1DF6A150EDF5C15E21A
:10D6F000E2EC7BF00FE1DE52010EDD6EDF2A7DEC05
:10D7000075F006014A6F8FDFDF2A7DEC75F00601A8
:10D710004A6F03D0030EDF26E8D7E5EC75F012E080
:10D72000010EDB5004E049C6E6FF9ADFE5524AC627
:10D7300000F0630E005C02E1300E006E0050E66EF9
:10D740008FDFE5524EDF000910E0E4EC77F044C6CD
:10D7500017F145C618F146C619F147C61AF148C671
:10D760001BF149C61CF14AC61DF1020EE15C02E242
:10D77000E16AE552E16E2AEF73F0D6EC79F00850D9
:10D78000DF6E2492100E085C13E11C0E086E02017D
:10D790005451010B03E11E50040B02E1110E92D013
:10D7A0005451040B27E11E50080B01E0AAD022D0EF
:10D7B000110E085C09E12480238E0201080E546FCB
:10D7C0002482086A120E9CD0120E085C06E1249096
:10D7D0002482030E086E130E93D0130E085C0CE126
:10D7E0001C0E086E02015451040B04E11E50080B7C
:10D7F00001E087D0140E66D0140E085C10E124807E
:10D80000238E180E086E1E50040B01E07AD01E50B5
:10D81000080B01E076D02482086A150E71D0150E2F
:10D82000085C0CE101012BAF03D00201020E546F22
:10D83000239E2482020E086E160E62D0160E085C1D
:10D8400005E12482020E086E170E5AD0180E085CED
:10D8500007E10201020E546F2482086A190E50D0AB
:10D86000190E085C06E1239E2482020E086E1A0E31
:10D8700047D01A0E085C05E12482020E086E1B0ECA
:10D880003FD0170E085C08E101012BBF03D0020155
:10D89000020E546F1B0E16D01B0E085C05E124907F
:10D8A000238E2482030E2AD01C0E085C2AE12490C9
:10D8B000800E086E02015451010B03E11E50040B4F
:10D8C00003E1110E086E1DD035AE02D0359E19D081
:10D8D0001850800B16E13BEC77F004E0090E0201D2
:10D8E000565D0AE30601EA5104E0080E0201565DA6
:10D8F00003E302012C5105E02482080E086E100E8D
:10D90000096E24A202D08FEC61F0DF50085C01E0C8
:10D910001D8CE5522AEF73F04FEC7AF01D961D50E6
:10D92000080B01E0010E076E01015751400B18E092
:10D930003EEC08F0050814E00201215111E12251EA
:10D940000FE123510DE1800E08140AE02D50080B61
:10D9500007E11E50400B04E12550010B01E102D804
:10D9600053EF7AF039EC7BF0C9C7DFFF020EDB6AB8
:10D9700035A203D0010E91EC75F0010E69C1DBFFF9
:10D98000DB50DF5C0DE3020EDB5002E09FEC07F0A2
:10D99000020EDB6A0201FA0E226F28A80CD009D011
:10D9A000020EDB5002E19CEC07F0010E91EC75F0E9
:10D9B00002010A0E226F3592020EDB5001E0358221
:10D9C000030EE15C02E2E16AE552E16E2AEF73F0D8
:10D9D0000201596BE66AE66AE66ADCEC75F0020160
:10D9E000296B0701CA6B0C6A21B003D02180D4ECEB
:10D9F00065F01200D6EC79F00201050E2C6F280EAE
:10DA00002D6FE6DF020E0B5C05E181EC77F0140E62
:10DA100038EC73F00501040E266FE5522AEF73F01F
:10DA2000358E12000101DF51020B18E03D51800BD1
:10DA300015E12150010B12E12650040B0FE1255096
:10DA4000020B0CE1DF9330886E0EE66EE60EE66E9A
:10DA5000010EC8EC74F00101AA0EA86F12000101BA
:10DA60003D51800B04E12150010B01E1000C010C40
:10DA700001015751800B05E0020E005C03E0000439
:10DA800001E0000C010CD6EC79F0CAEC79F005E06D
:10DA900081EC77F0140E38EC73F02190219407019B
:10DAA000C86B51EC79F0E5522AEF73F050EC7BF043
:10DAB000800E4B1837E14C5035E10101DF9BFF0E22
:10DAC00005014F5D04E04FC508F04F6912000101E8
:10DAD000E1A503D0E19582EC17F00101E151080BBB
:10DAE00008E02150400B05E1120EE4EC73F0010157
:10DAF000E19735BE359E21B013D0CAEC79F002E033
:10DB0000006A54DB229602016B510AE13350010B8B
:10DB100007E12D50800B04E12D50400B01E12086E0
:10DB2000082A120077EC77F001E0F0D14C5001E0C8
:10DB3000EDD121A0239C8BEC13F0FF0801E0EFD086
:10DB40002150200B01E1EBD01950800B01E0E7D010
:10DB500002017A6B7AC2ADF11A921CEC76F0359E16
:10DB60001D901F50010B18E1005006E02050020BE1
:10DB700013E17EDF000910E00101010EAD6F1A8292
:10DB8000086A0B0E096E005003E169DF000901E02D
:10DB90001D8000502CE12DD01E50040B03E01E50C0
:10DBA000080B29E100500CE0CAEC79F009E12050A3
:10DBB000020B21E171EC74F003E15ADF00091BE074
:10DBC0001EB402D0110E05D01EB604D00201546B53
:10DBD000140E086E005003E142DF000901E01D80D1
:10DBE000005007E04DEC75F002E104DF98D018DF3B
:10DBF00096D018DF94D0050110511EE028AA12D04B
:10DC0000005003E071EC74F010E0005003E127DFF6
:10DC1000000901E01D80005001E104DF71EC74F0A7
:10DC200001E0E8DE1E0E086E7AD0268E870E56ECD6
:10DC300078F01DEC20F073D021AE05D0086A0A0EF2
:10DC4000096E1D806CD0005051E083EC75F006E049
:10DC50002150040B03E11F50020B48E00201185150
:10DC600014E01F50020B07E1A2EC07F000090DE1E0
:10DC700083EC75F00AE10201386B396B186B18C23E
:10DC800058F2D6EC09F0E6EC61F0A6EC73F00AE08D
:10DC900083EC75F0FDE0D4EC77F0FAE121941F926B
:10DCA000A2EF04F01D803BEC77F013E01A50400B1C
:10DCB00010E01A50040B0DE021A40AD01A94050EAE
:10DCC000E66ED00EE66EE80E0D2438EC73F001D04F
:10DCD0001D901DA024D0000E0201296F0701CA6FFC
:10DCE0000C6E1F92086A0B0E096E19D0005017E1D6
:10DCF0002150010B14E183EC75F003E02150040B7B
:10DD00000EE00101DF93A2EC04F0A6EC73F005E055
:10DD100083EC75F0FDE0219412001D8059DE215046
:10DD2000200B04E182EC0AF0000903E10201355105
:10DD30004EE0E5EC75F04BE00501106B219021946D
:10DD4000810E086E0EEC05F0000906E1660EE66E27
:10DD5000E50EE66E010E0DD083EC75F002E11B0EB0
:10DD600013D0D4EC77F00BE05E0EE66EE50EE66EB7
:10DD7000010EE66E13EC25F0E552E55208D082EC78
:10DD80000AF0000905E01A0EE66E1DEC25F0E552DA
:10DD900082EC0AF0000919E0A8C135F20EEC05F09A
:10DDA000000905E10101816BE2EC04F00ED0D4EC36
:10DDB00077F00BE0B6EC79F003E001013D9D02D075
:10DDC00001013C9F63EC17F01590BDEC06F077EC79
:10DDD00077F001E14C5038E0A2EC04F028AA28D0FA
:10DDE000ABECE7F00201296B30AA02D014EC4CF046
:10DDF00031A402D0A6EC4EF031AC02D02EEC4DF0A6
:10DE000025A002D070EC4CF033A002D0A8EC4CF06E
:10DE100024AE02D0A4EC4BF020A802D00AEC0FF004
:10DE20002D50800B03E12D50400B02E039EC0DF03A
:10DE3000269A1BAC02D08EEC08F029A203D02992BE
:10DE400037EC37F01D8C12002150010B14E0020159
:10DE50002C5111E11850800B06E0BEEC79F009E07E
:10DE60000B0E165C06E02150040B05E183EC75F007
:10DE700002E043EF6DF00201295104E0E9EC76F095
:10DE8000DCEC75F018AE5BD01AEC9BF0FEEC76F093
:10DE900017E03050200B14E13150040B11E12450F5
:10DEA000800B0EE13150400B0BE12550010B08E1D6
:10DEB0003350010B05E13350020B02E1A0EC2CF0D2
:10DEC000339220AA3CD0209A01013CAB38D0E4EC3C
:10DED00077F00201305110E1E9EC31F0190E165CD7
:10DEE00014E11850010B11E00101D051D15D0DE199
:10DEF0000201C80E306F1200306B1C0EE66E61EC32
:10DF0000E7F0E5520101960EA86F12007FEC76F063
:10DF100016E14C5014E122BA12D0A6EC06F000092A
:10DF200002E131EC29F018EC0CF0248A810E086E25
:10DF3000A6EC06F0000903E0A0EC2CF0268212000B
:10DF40000D04040F0701006F12000101B19B1AAC10
:10DF500026D0D6EC09F0148226A41BD0BDECE0F04C
:10DF6000560EE66EE50EE66E010E9CEC7BF0AEEC16
:10DF7000E4F0E30E0D2499DBE3EC09F0BDECE0F0F6
:10DF80004E0EE66EE50EE66E010E9CEC7BF0AEECFE
:10DF9000E4F002010E0E386F060E396F1200D0DF6A
:10DFA0000701FA0E036F016B026B0201566B576B90
:10DFB0001E90120000C70AF00201585104E0800EC2
:10DFC000DAEC73F01B800701035116E003510307DD
:10DFD000D6EC74F0CC0E005C0FE0FF0E005C0CE0A1
:10DFE000800E005C06E20050E66E40EC04F0E55264
:10DFF000006E0050DFDBE7D70A6A120080EC7CF08D
:10E00000DBCF58F23088006A248807EC25F0010144
:10E01000320EA86F19AA02D00201588F02011851BE
:10E0200002E0010E186F189E15D319AA02D0B7ECA2
:10E0300045F01AAC24D0D6EC09F01492D4EC7AF066
:10E04000D00ED8800F54050E105405E2ECEC61F0B0
:10E050000201186B120014820101E283228EB8ECD7
:10E0600009F01A8AA2EC07F000090FE121840101EE
:10E07000E09983EC75F009E00101E0891200288A3B
:10E0800002012C5102E0010E2C6F1200DEDA1A8C14
:10E090004EDB03E071EC74F001E01A9C26A410D072
:10E0A000FE0EDB500D6E51DF26940101B187249CDA
:10E0B00025B2248C25821AAC31D01A8429802ED026
:10E0C0001A50400B0FE0A2EC07F000090BE083ECC4
:10E0D00075F008E02150040B05E11D0EE66E1DEC05
:10E0E00025F00CD0FD0EDB500BE10201185103E1CD
:10E0F0002850400B05E015EC7AF080DFE5520ED099
:10E10000FE0EDB500D6E21DF1ABC07D053DF050178
:10E11000105103E1ECEC61F001D087DF9BD20601E6
:10E12000060E406F0701E3A902D006014007010176
:10E130002C510A0804E2A45102E00601402B02011E
:10E140001E0E266F120081DA01012A51E824030114
:10E15000D06F0A01190ED76F360ED66F0101D0515C
:10E1600003E0030ED05D03E10A01080ED66F4EEC0A
:10E1700078F003E10A013C0ED66F0A01DA8FD46B06
:10E18000358615EC7AF08ADB65D25FDABFEC36F0C3
:10E19000CFEC17F0348AE66A15EC7AF048EC7CF0A4
:10E1A00059D2010EE66EF1DFE5521200000403E1E0
:10E1B00012EC7BF019D0005042E0030E005C16E137
:10E1C00012EC7BF0E0EC77F004E0E80E0F6E030E4B
:10E1D000106E18EC76F003E074EC04F0F0DAF9DA83
:10E1E00003E1640E0F6E106AF6EF7BF0F1EC13F0B2
:10E1F000930E0F6E020E106E0050030819E2700E9F
:10E200000F6E030E106E050E005C04E1930E0F6E90
:10E21000020E106E060E005C04E1970E0F6E040EE7
:10E22000106E070E005C04E1200E0F6E060E106EDD
:10E23000F6EC7BF0020E005C04E1500E45DA8FEF45
:10E2400009F00050030803E20201040E366F070EC6
:10E25000005C03E10201080E366F1200F6D9280EA9
:10E2600019EC7AF0290EB0DAF5D1D9CFE6FFE1CF7B
:10E27000D9FFE6528C9E00000000000000008C9642
:10E2800000000000060EE66E41EC59F0E5528C8667
:10E290000000000000008C9600000000D80EE66E22
:10E2A00041EC59F0E552CCC7E6FF41EC59F0E5529C
:10E2B000E66A41EC59F0E552E66A41EC59F0E55264
:10E2C0008C868C8EDF6A1E0EDF5C07E2640EE66EC3
:10E2D00008EC20F0E552DF2AF6D7E552E552E7CF09
:10E2E000D9FF1200D9CFE6FFE1CFD9FF8C9E000005
:10E2F0000000000000008C9600000000030EE66E97
:10E3000041EC59F0E552CCC7E6FF41EC59F0E5523B
:10E31000FC0EDBCFE6FF41EC59F0E552FB0EDBCF04
:10E32000E6FF41EC59F0E552FA0EDBCFF3FFDB06D6
:10E33000F35000090FE0D5ECF9F0006EFD0EDBCFD5
:10E34000E9FFDB2AFE0EDBCFEAFF01E3DB2A00C098
:10E35000EFFFEAD700008C86C69E8C8EE552E7CF91
:10E36000D9FF1200E0EC79F0DF6ADF2A2DEC77F0BC
:10E37000FD0EDBCFE6FF15EC7AF0FAEC78F02DEC31
:10E3800077F0AA0EE66E030EE66EFAEC78F0010E58
:10E39000DB6AFA0EDB5001DB1AE2010EDB50E76E9E
:10E3A000FD0EDBCFE9FFFE0EDBCFEAFFE75037DBE8
:10E3B000EFCF4BF0010EDB50EA6AAA0FE96E030EB5
:10E3C000EA22EF504B5C03E1010EDB2AE2D701ECBD
:10E3D00079F002E005EC0CF001EC79F003E00A0EB4
:10E3E000DF5CC3E30A0EDF5C02E3000E01D0010E26
:10E3F000A6EC79F002E2E16AE552E16E4B502AD1D7
:10E40000D9CFE6FFE1CFD9FF8C9E000000000000CD
:10E4100000008C9600000000060EE66E41EC59F0FC
:10E42000E5528C860000000000008C960000000081
:10E43000020EE66E41EC59F0E552CCC7E6FF41EC26
:10E4400059F0E552FE0EDBCFE6FF41EC59F0E55204
:10E45000FD0EDBCFE6FF41EC59F0E552FA0EDBCFC3
:10E46000F3FFDB06F350000911E0FB0EDBCFE9FF01
:10E47000DB2AFC0EDBCFEAFF01E3DB2AEF50006E64
:10E480000050E66E41EC59F0E552E8D700008C866A
:10E49000C69E8C8E050EE66E08EC20F0E552E55225
:10E4A000E7CFD9FF1200D6EC79F075EC59F00101F5
:10E4B000640EA86F85EC3FF0020E07017B5D0EE055
:10E4C000BB5109E0E3EC05F00401FD6FFDC4E6FF7C
:10E4D000F4EC05F0E55213ECAFF05CD00701BB5152
:10E4E00059E0BB51E3D908E24B50C008000E4C5430
:10E4F00003E2040E58EC7AF0E3EC05F00401FD6F42
:10E500003B0EFD5D0CE13B0EFE6F0601C46B319AC4
:10E510000101389B076A7CEC0BF007017B6B610EF5
:10E520000401FD5D05E3FD51660802E3200EFD5F79
:10E53000300EFD5D1CE3FD51460819E30601C42BB6
:10E54000410E0401FD5D03E2300EFD5F04D0410E7B
:10E55000FD5D0A0FFD6F020E0601C45D06E1C339C1
:10E56000F00B0401FD25FD6F02D0FDC4C3F6020EC1
:10E570000601C45DB3E1FDC4E6FFDFEC0BF0E5523C
:10E58000006E010EA1D80601C46B0050E66E66DE77
:10E59000E552A4D702016B5102E048EC93F01D9CB8
:10E5A000100E085C03E281EC67F01ED01E0E085CC2
:10E5B00003E2BDEC6BF018D0085090D804E6800E52
:10E5C0004B5C000E4C5803E248EC20F00DD0085094
:10E5D00085D804E6920E4B5C000E4C5803E256ECD4
:10E5E0006DF002D096EC2BF01DBCD9D798EC50F012
:10E5F0000A5004E00701070E58EC7AF023A25AD71C
:10E6000023922F98339C10EC86F0DF682F50100B6C
:10E6100014E001012B51040B10E12A50020B0DE113
:10E62000DF500BE00E5002E1010E0E6E2F98F6EC5B
:10E6300092F010EC86F0DF06E9D7DF5001E03AD720
:10E640000701050E58EC7AF035D7D9CFE6FFE1CFB8
:10E65000D9FF1200E552E7CFD9FF12004B504E24EC
:10E66000F36E4C504F20F46E4D5050208AEF7AF0EC
:10E67000E66EEEEC14F0E5EF79F0E66EE7EC38F0DC
:10E68000E552E5EF79F001EC39F0E552E5EF79F08C
:10E69000446E456A33EC7AF040C04CF01200E66EEE
:10E6A000E8EC14F0E552E5521200E66E90EF7AF0D5
:10E6B000F36EFE0E1DEF7BF0AFEC7AF002EFFAF096
:10E6C000DBCFE6FF90EF7AF0E66E08EC20F0E55243
:10E6D0001200E66E68EC7FF0E5EF79F04B6E4C6A65
:10E6E000D8904C5012005AC3E9FF5BC3EAFF1200F6
:10E6F000030D47EC7BF0DA0EE926020EEA22120047
:10E70000E66E5AEC7FF0E552E5EF79F04F6E506A15
:10E71000516A4C504F24F36E4D505020F46E4E50C1
:10E7200051208AEC7AF00800F5CF4BF01200A0ECF3
:10E730001EF000091200D950FD0FE96EFF0EDA201D
:10E74000EA6E120017EC7BF095EF7BF0FAEC61F0CB
:10E7500022EC7BF04B504C101200E66EC0ECF6F051
:10E760004B6E050EE15E4B501200EECF3FF0EDCF49
:10E7700040F002ECFAF03BC0EEFF3CC0EDFF39EF99
:10E780007AF03EEC7CF00201EF514B5CF0514C58BA
:10E790001200DF50EA6A160FE96E070EEA22120035
:10E7A000E66E37EC13F0E5EF79F0E66E1DEC25F040
:10E7B000E5521200E66E8FEC0FF0E5521200F3CF37
:10E7C0000FF0F4CF10F01200E66E73EC06F0E55295
:10E7D0001200050E0101D05D12009FEC7BF04C6E23
:10E7E0005CEF7AF0EA6ADD0FE96E070EEA221200AA
:10E7F0005BECE7F0E5EF79F0436E446A456A51C09F
:10E800003EF052C03FF053C040F0AFECF5F03BC0DB
:10E8100051F03CC052F03DC053F0C1EF7AF0516A64
:10E82000526AAAEC7AF04D6A4E6A4BC03DF04CC079
:10E830003EF04DC03FF04EC040F04FC042F050C0DF
:10E8400043F051C044F052C045F0F3EFF7F02CC153
:10E85000E6FF15EC7AF020EC33F0E552E552DF6E7E
:10E860001200B4EC7CF0010EDBCF40F05CEFFAF06C
:10E87000070BF36EFCEF7BF0E00BE842E842E84266
:10E88000E842E8421200E66EC7ECF0F0E5EF79F0FE
:10E89000EA6A0F0FE96E010EEA221200E66A48EFFB
:10E8A0007CF0E66E4CEC13F0E55212004B6E4C6AB5
:10E8B0004C341200516A526AD89050365136523652
:10E8C0004D505024F36E4E505120F46E4F50522054
:10E8D0008AEC7AF00900F5CF4BF00800F5CF4CF048
:10E8E000120018EC0EF0000912004B505424F36E85
:10E8F0004C505520F46E4D5056208AEF7AF0446A01
:10E90000456AF3ECF7F039500701EC273A50ED2354
:10E910003B50EE233C50EF231200446A456AF3EC6F
:10E92000F7F039500701F0273A50F1233B50F2231A
:10E930003C50F3231200E66EC3EC13F0E5521200D4
:10E94000FC0EDBCFE6FFFD0EDBCFE6FFFE0EDBCFDE
:10E95000E6FF12000A0D47EC7BF0000EE926030EDD
:10E96000EA221200016E0150EA6AC50FE96E060E36
:10E97000EA22EF50006E1200E66EF7EC14F0E5525A
:10E98000E5EF79F0B4EC7CF02AC140F05CEFFAF0EE
:10E99000E66E13EC25F0E5EF79F0F36E010E1DEF56
:10E9A0007BF010C0E6FF0FC0E6FF1200016EBCEF67
:10E9B00038F0C3CF4BF0C4CF4CF05BEC7CF05BEC99
:10E9C0007CF04BC0DEFF4CC0DDFF63EC10F0B4EC1C
:10E9D0007AF04B501200350EE96E070EEA6E4BC00E
:10E9E00042F04CC043F019EC7CF0EECF3DF0EECF9E
:10E9F0003EF0EECF3FF0EFCF40F01200E66A90EC31
:10EA00007AF0E66A90EF7AF0E66E6CECE7F0E552A9
:10EA1000E55212000FC03FF010C040F01200E9268E
:10EA2000000EEA22120019EC7CF0A3EF7AF03EEC23
:10EA30007CF003EC7CF0020EE15C1200D151100D71
:10EA400022EC7BF07A0E4B260A0E4C221200C0C13B
:10EA50009AF1C1C19BF1C2C19CF1C3C19DF1C4C176
:10EA60009EF11200B6C19AF1B7C19BF1B8C19CF1F9
:10EA7000B9C19DF1BAC19EF1120095ECF6F04F6E4E
:10EA8000060EE15E4F501200006E248807EF25F05D
:10EA9000E66E48EC6BF0E5521200030E0101D05D0A
:10EAA00012000101A06BA0C19FF197EC04F00101DD
:10EAB000A16F3B500F6E106A93EC04F00101A26F3E
:10EAC0003BC0A3F11200E66E95ECF6F04B6E060E1D
:10EAD000E15E4B501200100DF3CF4DF0F4CF4EF02D
:10EAE0001200020EE66ED0EC24F0E5521200010E88
:10EAF000E66E19EC1CF0E5521200DFCFE6FF4BEC9E
:10EB000004F0E55212001DEC05F000091200020E9F
:10EB100094EC7AF002EF7BF0E66E19EC04F0E5522B
:10EB20001200F36E020EF3CFDBFF1200006E02EF55
:10EB300024F0D051100D22EC7BF02A0E4B260A0E49
:10EB40004C225CEF7AF0070BF36EF46EFCEC7BF07A
:10EB5000CB15F310CB6FF4500B6E120000C010F009
:10EB600050EC7CF000C00FF00A6A120093EC7CF0CD
:10EB70000F264C5010221200D051EA6ACA0FE96EDB
:10EB80000A0EEA221200DF50EA6A1E0FE96E070E33
:10EB9000EA22120042EC3BF05FEC7CF0000912002C
:10EBA000680E0A6EFE0EDB50100DF350120053EC8F
:10EBB0007CF00C0F0A6E1200FDEC26F0E5EF79F008
:10EBC000E66E24EC04F0E5521200020E02016B5DC9
:10EBD0001200ABECE7F0090E4B6EFD0EDBCFE7FF4A
:10EBE0004B50E726FD0EE7CFDBFFDF6A1200C15175
:10EBF0004B6E4C6AC051640DE9EC7BF0010E0F0BBB
:10EC00001200006EBDECE0F00101040E016FADECEE
:10EC1000E6F001013EEF7BF0B70E43EC7CF0010122
:10EC200051514B6E4C6A0F504B5C10504C581200B7
:10EC3000DDEC0DF000091200A0EC1EF0006E1200D9
:10EC4000030E016E2CC100F077EC38F0DCEF7BF0A6
:10EC50009BEC7CF06CECE7F0E552E5521200EA6ABE
:10EC6000CF0FE96E0A0EEA22EF50016E1200DFECC0
:10EC700023F05FEC7CF0E55200091200ABC2E9FF23
:10EC8000ACC2EAFF1200010E94EF7AF0F36EFE0EB2
:10EC9000F3CFDBFF1200B7EC05F000091200E66EBF
:10ECA0000150E66E1200B5EC06F0000912004E6E3F
:10ECB0004F6A506A1200FC0EDBCFF6FFFD0EDBCF71
:10ECC000F7FFFE0EDBCFF8FF0800F550120079ECDD
:10ECD00004F00701D951F3144B6EDA51F4144C6E61
:10ECE0004B504C101200ADECE6F00101200E1A6FF3
:10ECF0001200E66820EC33F0E552E552120050ECC9
:10ED00007BF0820E4B1812000150030D47EC7BF094
:10ED1000470EE926050EEA2212004B6E020E17EC92
:10ED20007BF051ECF5F040501200100E4B6EFE0ED1
:10ED3000DBCFE7FF4B50E75EFE0EE7CFDBFF1200B5
:10ED40009AC1B6F19BC1B7F19CC1B8F19DC1B9F1AF
:10ED50009EC1BAF11200C0C1B6F1C1C1B7F1C2C1C2
:10ED6000B8F1C3C1B9F1C4C1BAF11200C5C19AF179
:10ED7000C6C19BF1C7C19CF1C8C19DF1C9C19EF13B
:10ED80001200C5C1BBF1C6C1BCF1C7C1BDF1C8C14C
:10ED9000BEF1C9C1BFF11200BBC19AF1BCC19BF168
:10EDA000BDC19CF1BEC19DF1BFC19EF11200010E1B
:10EDB000E66EB0EC3DF0E552E552C7EC2FF00201F3
:10EDC0007207120002ECFAF03FC00FF040C010F0E2
:10EDD0001200010EE66ECAC7E6FFCBC7E6FF1200BF
:10EDE000E66A32EC1BF0E5521200E66E4EECFAF0E9
:10EDF000E552120009ECF2F084EFF1F0ACEC05F012
:10EE000000091200DCEC4FF00009120002018C0E28
:10EE1000A26F0A0EA36FA2C2A0F2A3C2A1F21200B7
:10EE20004B6E4BC0E6FF72EC0EF0E552E7CF4BF0B5
:10EE30004B181200010EE66EEFEC09F0E5520101ED
:10EE4000B197E6EF61F00900F5CFE6FF0900F5CFD5
:10EE5000E6FF0800F5CFE6FF1200FA0EDBCFE6FF73
:10EE6000FB0EDBCFE6FFFC0EDBCFE6FF120001015D
:10EE70003751400B12000101B151080B1200015033
:10EE80000224010FEA6A8D0FE96E030EEA221200D6
:10EE90001002F3CF10F00F02F3CF0FF0F450102652
:10EEA0001200DBCFE7FFD890E732D890E732E7CF08
:10EEB000DBFF12009BC1E6FF9AC1E6FF2CEF7CF05E
:10EEC00012EC12F00701620E35EF7CF0FADAB7C1EE
:10EED00040F05CEFFAF0FE0EDBCFF3FFDB2AF350DD
:10EEE0001200EA6A170FE96E010EEA221200D8DB5F
:10EEF000810E4B181200010EE66EA3EC70F0E55285
:10EF00001200010EDF6EE66ADFCFE6FF1200D9CFF6
:10EF1000E9FFDACFEAFFEF501200A2EC04F00201A1
:10EF2000140E2A6F1200E2C64BF0E3C64CF0D890E4
:10EF300012000901520EBD6F560EBE6F12007CEC1E
:10EF40001EF04B0E005C12004B509F08000E4C54FC
:10EF500012005BEC7CF0E8041200FE0EDB380F0BB5
:10EF6000E66E1200FE0EDB500F0BE66E1200300E46
:10EF70004B5C000E4C581200E66EBFEC1BF0E552E5
:10EF800012000601EA5102012C111200E66EC3ECD8
:10EF900008F0E5521200E66E140EE66E0A0E12003C
:10EFA0009AEC0BF00009120026EC17F00009120091
:10EFB00052EC0EF000091200FAEC0DF000091200FC
:10EFC000D5EC0DF000091200006807EF25F00101F3
:10EFD000495132081200E66EE66AE66A1200FE0E39
:10EFE000DBCF4BF0FD0EDB50D8804B541200EA6AA9
:10EFF0009E0FE96E020EEA223BC1EFFF1200E3C74B
:10F00000EFFFD0C1E6FF31EC08F0E552120001013C
:10F01000D56F050ED880D455000ED5551200E66E7A
:10F0200046EC70F0E552E5520201586B1200500EAA
:10F03000E66EE66A7A0EE66E0A0EE66E1200400E84
:10F04000426E420E436E0F0E446E456A1200DB5054
:10F05000E552E75C4B6EFC0EDB504B5C1200050E7C
:10F06000F36E020EEAD225C100F0C8C2E6FF62ECE0
:10F070003FF0E552120026C100F0C9C2E6FF62EC83
:10F080003FF0E5521200D7EC0BF024980101A86B79
:10F09000B19F12000A0E4B6E4C6A1200040E010161
:10F0A000D05D1200E6520750DF6E1200006E07EFCF
:10F0B00025F0A0EC1EF003081200D89010320F3299
:10F0C0001200190ED880D75512000A0E01012C5DCE
:10F0D00012003E6A3F6A406A1200006E77EF38F015
:10F0E0000DEC09F0E5521200E66E2BEC25F06DD127
:10F0F000FD0EDBCFE6FF8FEC0FF0E55212000201B0
:10F10000416B41C242F241C243F21200E66EE66E2A
:10F1100048EF7CF0E66E4CEC10F057D186D973ECDA
:10F1200006F0E552120091ECF5F03DC04BF03EC008
:10F130004CF012000750EA6AAD0FE96E020EEA22A7
:10F140001200E65297EC04F0DF6E3B50006E1200A6
:10F1500006DA6BEFF5F095ECF6F04D6E060EE15E1B
:10F160004D501200E66EE66A540EE66E060EE66E2E
:10F170001200F3504D244B6EF4504E204C6E120092
:10F1800000010F244B6E000E10204C6E1200E66A38
:10F19000E3ECDBF0E55278EFDAF0FB0EDBCFF3FFC8
:10F1A000DB06F350000912005CECFAF03C50006EF4
:10F1B000FE0EDB50120092EC0EF0010F0A01D88017
:10F1C000D6551200E66EE66A6AEC1FF0E552E5528B
:10F1D0001200010EE66E5DEC3BF0E552176E120078
:10F1E000E66E54EC7FF0F1D0006E248848EC24F0F9
:10F1F000AEEFE4F072EC71F04B6E050EE15E4B5039
:10F200001200FA0EDB50F36E010EDB50F35C1200BD
:10F21000E66E2FEC04F0E5521200A50E4B5C000EDA
:10F220004C5812000201586B58C218F21200E668DE
:10F230005FEC33F0E55212000101266B26C125F187
:10F240001200C3CF0FF0C4CF10F01200E66853ECE9
:10F2500035F0E55212007CEC1EF04C0E005C120002
:10F26000D8800F54030E105412002A0E4D260A0E99
:10F270004E221200E76E010EE7CFDBFF1200F3CF44
:10F28000D4F1F4CFD5F1120016DBE8061200E66ED9
:10F2900049EC15F0E5521200400E01014503F35010
:10F2A0001200030E086E0C0E096E12007A0E4D2627
:10F2B0000A0E4E221200FAECF1F009EFF2F0E66EBF
:10F2C000C50EE66E010E1200E66EC00EE66E010E71
:10F2D0001200E66E38EC39F0E55212000101E393BA
:10F2E000E395E3971200DE514B5CDF514C5812005E
:10F2F000F36E030EF3CFDBFF1200010EE66E90EF0C
:10F300004AF0F80BE842E842E8421200006E080EAC
:10F310000D24005C12000068F0EF24F001013C5164
:10F32000200B1200A0EC1EF0050812000101CE51C6
:10F33000010B120049EC0EF000091200190ED880E2
:10F34000015412000F5C000E105812004B6E020E9A
:10F35000E15C1200190E0A01D75D1200F1EC13F006
:10F360000009120000504D6E4E6A12000FEC0EF0B4
:10F370000009120004EC0EF000091200FDEC64F02C
:10F3800000091200EFEC60F00009120062EC10F0CE
:10F3900000091200E7EC0DF000091200FE0EDB5030
:10F3A000FF081200ADECE6F0300E120025EC73F011
:10F3B000E65212004D6EFE0EDBCF4EF063EF7CF096
:10F3C00025EC73F0020EE12612005FEF7CF0D1EC29
:10F3D00074F0E60E0D2438EC73F0010E64EC73F05B
:10F3E000E30E9BEC74F086EF79F08EDAFD0E60EFA1
:10F3F00073F0030E436E446A456A4EC03EF04FC040
:10F400003FF050C040F0AFECF5F03BC04EF03CC0D8
:10F410004FF03DC050F02EEC73F023EF77F047DC57
:10F420002EEC73F00800F5501200FE0EDBCFE6FF65
:10F430001200E4EC73F091DD2AEC14F0E552E4ECF8
:10F4400073F090DD2AEC14F0E552E4EF73F058DA33
:10F45000DB501200320E4B6E850E4C6E010E4D6E5F
:10F46000015073EF7CF047DA02ECFAF03FC04BF04A
:10F470001200FD0EDBCF4BF0FE0EDBCF4CF0120086
:10F480000FEC75F0EF6A73EF73F00A01B1EF7CF0E7
:10F4900056EC04F0E552E66E130E4FEF73F025ECD8
:10F4A00073F052EF78F0DF50076EE5522AEF73F0F9
:10F4B000266F240E51EF74F04BC0E6FF4CC0E6FF00
:10F4C00012000A0EB4EF7CF0080EE66EE66AD40E67
:10F4D000E66E0A0EE66E0101D0516BEF75F0100E6C
:10F4E000DF02F3500224016E700E0224E0EC75F08E
:10F4F000006E02501200E66AE66A120E38EF73F0F0
:10F50000CCEC0AF0E55273EF73F078EC73F0020E76
:10F510000FEF75F0F86EF4CFF7FFF3CFF6FF1200A0
:10F52000BBEC14F0E5521200006ED6EF70F0E66E00
:10F5300043EF73F00FDA3F501200300E4B24E4EC2F
:10F5400073F09BEF73F091ECF5F03DC00FF03EC00F
:10F5500010F012000FC04BF010C04CF012004BC066
:10F5600044F04CC045F0120000504B6E4C6A120043
:10F5700091EC08F01850010B030DF350840FDAEFF3
:10F5800073F04E5051244B6E4F5052204C6E5050E1
:10F5900053204D6E1200FE0EDB50400DF350DF6E17
:10F5A000FE0EDB50D7EF75F0A0EC6FF000C70AF04D
:10F5B000FC0ED6EC74F0AEEF75F000506EEF73F009
:10F5C000DF24D6EF74F04B6E4C6A95D913EF75F0CB
:10F5D000B2D9C00EE66E010E3DEF73F0CB513CEC9C
:10F5E00074F038EC74F0D815F310D86F1200FE0EDA
:10F5F000DB507F0BDAEF73F04FEC76F043EC73F0F7
:10F600000A6A1200FA0EE66EA7ECF9F0E552120053
:10F6100025EC73F00A0E58EF73F0230E01012F252D
:10F620008CEF75F001012A510A0DDFEF73F04C6E7B
:10F630004CC045F04BC040F01200DBCFF4FFF3505C
:10F64000F45C1200F3CF4BF0F4CF4CF012005CEC02
:10F6500073F03F50006E12000101D051F2EF73F0D1
:10F660000A0E48EC73F04B501200010EE66E4EEF9E
:10F6700074F025EC73F0030EE1261200200E1B6FD0
:10F68000300E1C5D120025EC73F0D0EF75F0F3CF57
:10F69000E9FFF4CFEAFF1200E66E480E43EF74F084
:10F6A00008504B6E4C6A1200318AFE0E60EC73F00B
:10F6B000FEEC74F0DF6E1200E66E0DEC15F0E55214
:10F6C0000C0E64EF73F071EC75F00101200E1A6FEF
:10F6D0001AC119F112009A0EE66E020E3DEC73F09B
:10F6E00043EF33F00A0EC2EC74F040C0A1F13CC00D
:10F6F000A2F112000B50010138EC74F0CB15F3109D
:10F70000CB6F120001012951FCDD295F77EF75F005
:10F7100008C7E6FF120EE66E400E43EF74F000508D
:10F7200056EF74F0D9516EEF73F05CECFAF0405084
:10F730001200015048EF74F0E66EF8EF73F0080D18
:10F740004D50F3244B6E4E50F42012004E6E00507C
:10F7500086EC73F00350EA6A120087DD0701D65188
:10F76000EDEF73F0C9EC73F0EF68C3EC75F0EF6880
:10F7700012000F6C101E000E1022D1EF74F0FC0E60
:10F7800060EC73F0FB0E60EF73F086DDDF6E4551C9
:10F79000D7EF75F04DC0E6FF4EC0E6FF3DEF75F0C8
:10F7A00098DC100E426E270E436E1200446E456ABE
:10F7B0000AEC75F0E2EF76F0380E016E61C100F0F0
:10F7C00077EF38F07DEC75F0F36EFE0EDB50F35CF6
:10F7D0001200F3504B240F6EF4504C20106E1200A8
:10F7E000D6C13FF0D7C140F05CEF73F0190EBCEC0E
:10F7F00077F0680E55EF73F0F346F346F346F346A1
:10F80000F3461F0E12004BC0F3FF4CC0F4FF120072
:10F8100055EC73F0CCEF07F0E66EE66A43EF73F059
:10F82000EA22FE0EDBCFEFFF12004B6E050EA2EFB9
:10F8300073F04DC044F04EC045F012008CEC75F0F2
:10F84000006E0050120073EC73F0010EEB501200CA
:10F850000701E9516EEF73F0C3EC1FF0E552E5527A
:10F860001200010EDB5096EF75F0D880D055020ED5
:10F87000D155120064EC73F035EF0FF0DECF4BF092
:10F88000DDCF4CF01200E66E92EC62F0E552120011
:10F89000D6EC19F0E552E5521200050DDFEF73F0DA
:10F8A000012ABCEF38F0FC0BE842E84212009BEC66
:10F8B00073F0EF501200D8904C324B321200E552E8
:10F8C000E552E55212004F6A506A2EEC73F00800C0
:10F8D000F5501200060EE66EDD0EE66E070EE66EC1
:10F8E000F00E97EF7AF057EC76F0D8904E364F3610
:10F8F00050362EEF73F04BC03FF04CC040F012007A
:10F9000025EC73F0FE0E120025EC73F0FE0E60EC99
:10F9100073F00101E3811200006E0050E66EF0DD2D
:10F92000EF50040B12004B6E4C6A4B5012000FEC60
:10F9300075F0EF501200E66EDFCFE6FF120036DD05
:10F94000FE0EDB50F2EF73F04D6EDF50DF2A67DD05
:10F95000016E12000AEC75F05CEF73F0E8DD0A6AE4
:10F960001200D65156EF74F04B6E4BC045F01200AA
:10F97000080E016E0101D05102E1180E016E340E25
:10F980000101B55D09E1016A5DEC0AF0000902E0E0
:10F99000100E016E78EC17F01200200EE66E850E48
:10F9A000E66E070EE66E800EE66E01EC39F0E5526B
:10F9B0009AEFA7F0C8ECA7F0FE0EDB507EECA6F0A5
:10F9C000EFCFDFFFFF0EDF5C02E1100EDF6EDF50D6
:10F9D000E55245EFA5F0CCDF03015E510126015051
:10F9E000E66EE8DFE552046E1200006807EC25F0D1
:10F9F0000101040E016F0450006E00500F0803E275
:10FA0000100E005E04D0100ED8800054006EADECD5
:10FA1000E6F00101200E1B6F050E006E300E1C5D1E
:10FA200002E0040E006E04500F0805E20050B5EC31
:10FA3000A5F02B0E04D00050B5ECA5F02D0EEF6E06
:10FA40000101010E016F200E4B6EEC0E4C6E010E8B
:10FA50004D6E5EC34EF04F6A506A030E436E446AA9
:10FA6000456A4EC03EF04FC03FF050C040F0AFEC92
:10FA7000F5F03BC04EF03CC04FF03DC050F09FEC65
:10FA8000A7F00900F5CFE6FF0900F5CFE6FF080073
:10FA9000F5CFE6FF5BECE7F03DECA8F00101198F34
:10FAA00012001B0E0101B55D01E1010C000CC8EC58
:10FAB000A7F00050EF0860E2F00E005CDF6EDF5050
:10FAC000080868E32A50010B06E10401F95103E13B
:10FAD0000401FA5109E00101E0910201236B0201E6
:10FAE0003C6B13ECAFF0EED7006807EC25F001019A
:10FAF000960EA86FDF50FE0BE842750F0A6E016A82
:10FB0000DFA002D0800E016E026A070E025C0CE2DA
:10FB1000BCEC38F0005008E0FF0E005C05E045EC5E
:10FB2000E7F0012A022AF1D7AEECE4F00101E0850A
:10FB3000080E016EDFA002D0800E0126026A780E48
:10FB4000025C10E2BCEC38F000500CE0FF0E005CF0
:10FB500009E00050036EE66EF4EC05F0E552012A70
:10FB6000022AEDD73B0E035C05E03B0EE66EF4EC9B
:10FB700005F0E5520A6A18D0E7ECA6F000504E6E88
:10FB80004F6A2EECA5F0056EFF0E055C05E1B60E82
:10FB9000BEECA5F0268E08D0B5C15AF205C0B5F16D
:10FBA0002A820201010E6B6FE55245EFA5F01B0E94
:10FBB0000101B55D04E1F00E03015D2515D000687B
:10FBC000016A0150DDECA5F004E6960E4B5C000ED8
:10FBD0004C580EE2E7ECA6F001504E6E4F6A2EEC48
:10FBE000A5F0B55D03E10150006E1200012AE9D7CE
:10FBF0001200020E016E2BC100F077EC38F02F0ED0
:10FC0000016E58C100F077EC38F0370E016E60C11C
:10FC100000F077EC38F00F0E016E38C100F077EC91
:10FC200038F0100E016E39C100F077EC38F02E0E6E
:10FC3000016E57C100F077EC38F0620E016E8BC197
:10FC400000F077EC38F0650E016E8EC100F077ECB5
:10FC500038F0660E016E8FC100F077EC38F06E0E52
:10FC6000016E97C100F077EF38F0130E016E3CC1C2
:10FC700000F077EF38F03B0E0101B55D04E11AB6F4
:10FC800002D00101CD7B150E0101B55D2FE11AB641
:10FC900002D001013C7901013C51100B0FE0BFEC97
:10FCA000A6F00CE0A30EE66EE80EE66E010E39EC4F
:10FCB000A5F02AB21BD001013C9918D02EEC1DF002
:10FCC000A0EC2CF001013C51100B0BE02250020B78
:10FCD00008E1BA0EE66E8D0EE66E010E84ECA6F01B
:10FCE000E55201013CB902D04BECA6F03A0E0101FD
:10FCF000B55D0AE11AB608D0020E0101435D02E1CA
:10FD0000010E01D0020E436F040E0101B55D03E048
:10FD1000050EB55D13E11AB608D0040EB55D03E11A
:10FD20000701E37102D00701E3739EEC1DF089EC3B
:10FD300023F046EC08F0020107812E84260E010113
:10FD4000B55D06E11AB602D001017871E7EC1EF04C
:10FD50001F0E0101B55D04E11AB602D00101CE7F8C
:10FD60000E0E0101B55D06E11AB602D001013F7128
:10FD700018EC59F0250E0101B55D0FE11AB602D05D
:10FD800001013975010139510701099F040B01E097
:10FD9000098F55ECF1F037EC37F00F0E0101B55D2E
:10FDA00004E11AB602D00101CE7B170E0101B55D48
:10FDB00004E11AB602D00101397F080E0101B55DD8
:10FDC00004E11AB602D00101977D0101B55104E1A9
:10FDD0001AA63476A0EC1DF02F0E0101B55D04E1EA
:10FDE0001AB602D001012B752A0E0101B55D04E19E
:10FDF0001AB602D001012B73190E0101B55D01E1A4
:10FE00002F742D0EB55D01E12F723C0EB55D04E13E
:10FE10001AB602D001013871110E0101B55D04E17D
:10FE20001AB602D001012B7F2C0E0101B55D0DE148
:10FE30001AB609D00101609F9F0EE66EE80EE66ECD
:10FE4000010E39ECA5F0E7EC1EF012002FECA8F043
:10FE5000FB0EDB50D880DF5403E2FB0EDB50DF6E7D
:10FE6000FC0EDB50DF5C03E2FC0EDB50DF6E0EAEFF
:10FE70000CD0FC0EDB50D880DF5402E2DF0605D048
:10FE800033B603D0FB0EDB50DF6E0E040BE1FB0E2E
:10FE9000DB50DF5C02E2DF2A05D033B603D0FC0E74
:10FEA000DB50DF6EF7EFA7F0FCECA7F0C5ECA5F098
:10FEB00045EFA5F040ECA5F03386FB0EDBCFE6FF67
:10FEC000FC0EDBCFE6FFC5ECA5F0339645EFA5F0C1
:10FED000FCECA7F002ECA8F0EDDF2CECA8F045EF6D
:10FEE000A5F02FECA8F0EEECA6F0E8AE02D04B3473
:10FEF00003D0E750D8804B5403E2FB0EDB50DF6E9B
:10FF0000F5ECA6F0E8AE02D0E73402D0E7504B5C47
:10FF100003E2FC0EDB50DF6E0EAE0BD0F5ECA6F06C
:10FF2000E8AE02D04B3403D0E750D8804B5401E206
:10FF3000DF060E040AE1EEECA6F0E8AE02D0E734EC
:10FF400002D0E7504B5C01E2DF2AF7EFA7F0960EF4
:10FF5000036E0450010B0BE0C5ECA7F008E1780E2E
:10FF6000036E17ECA8F00A0802E1500E036E1200AF
:10FF7000C8ECA7F080DE2E0E0101B55D2BE101017A
:10FF80003751070B006E0E040EE137BF02D0378FDA
:10FF90001AD037BD03D0378D006A15D0070E005C2C
:10FFA00012E2002A10D0FF0E0E5C0DE1005005E0B9
:10FFB000000600AE08D0006A02D037AD02D0379DEF
:10FFC00002D037BF379F0050070BF36EF80E37157E
:10FFD000F310376F1D0E0101B55D1FE10101D05116
:10FFE00004E00FEC0EF0000903E0ABEC0AF015D0D2
:10FFF0000E0409E1010157B102D057810ED057B567
:020000040001F9
:100000000CD057850AD0FF0E0E5C07E1010157A501
:1000100002D0579502D057B157910B0E0101B55D33
:100020000BE1150EE66E030EE66E560EE66E010E41
:1000300025ECA5F0A2EC04F00C0E0101B55D08E181
:10004000050EE66E840EE66E010E2AECA5F0349ED7
:100050000A0E0101B55D15E1020EE66E850EE66E33
:10006000010E2AECA5F0300E010185250401F76F81
:10007000020E0101855D03E10401340EF76FE4EC2B
:10008000AEF0200E0101B55D15E1030E0101CC15A6
:100090000101066F065102E1010E066F030ECBEC63
:1000A000A7F0FC0E0101CC17010106510101CC1390
:1000B000E7EC1EF0290E0101B55D12E11AB602D07F
:1000C0000101CE71BFECA6F007E001013C51100B1D
:1000D00003E03C992EEC1DF04BECA6F0A0EC2CF0CC
:1000E000100E0101B55D30E10E0412E1080E0101B0
:1000F000515D02E10D0E27D0050E515D1FE0030E8C
:10010000515D17E0510510E00D0E515D1DE007D067
:10011000FF0E0E5C19E1030E0101515D02E1010EBB
:1001200012D0050E515D02E1030E0DD0080E515D97
:1001300002E1050E08D00D0E515D02E1080E03D05C
:10014000510502E0010E516F82ECA7F02FE1010191
:10015000E3AB03D0ABEC0AF029D0640E006E0701CC
:10016000E3AB02D00A0E006E0E0409E1000100505C
:1001700001016A27000E6B236C236D2311D0FF0E43
:100180000E5C0EE100504B6E4C6A4D6A4E6A4B504D
:1001900001016A5F4C506B5B4D506C5B4E506D5B68
:1001A00027ECEAF02584348A37EC37F0120E01018F
:1001B000B55D0BE1030E010150150101066F020E42
:1001C0009CECA7F0FC0EFCECA6F0130E0101B55D53
:1001D00012E1300E010150150101066F06390F0BB7
:1001E000066F020E9CECA7F001010639F00B066FBA
:1001F000CF0EFCECA6F00D0E0101B55D09E1820EFB
:10020000E66E520EE66E520EE66E010E25ECA5F07D
:10021000390E0101B55D19E10701E351E840E840FD
:100220003F0B0101066F030E06179CECA7F00101BE
:10023000040E0603F3CF06F1F30E0701E3170101E5
:1002400006510701E31346EC08F03F0E0101B55DCE
:1002500009E1730EE66E460EE66E530EE66E010E73
:1002600025ECA5F0E3ECA6F033E12150040B30E0DF
:100270000E0414E12C50040B02E0140E01D0010E08
:100280004B6E4C6A4BBE4C682350040B01E0010ED0
:100290008BECA5F04B50EE264C50ED22FF0E0E5C81
:1002A00014E12C50040B02E0140E01D0010E4B6E31
:1002B0004C6A4BBE4C682350040B01E0010E8BECE2
:1002C000A5F04B50EE5E4C50ED5A7CEC14F01F88BC
:1002D000320E0101B55D08E17E0EE66E8D0EE66E12
:1002E000010E84ECA6F0E552360E0101B55D19E170
:1002F00034A808D0560EE66E8D0EE66E010E84EC24
:10030000A6F00ED031EC12F000C006F1C80ECBEC16
:10031000A7F006C100F077EC38F0E66A32EC1BF08B
:10032000E552160E0101B55D16E10101DFAD08D001
:10033000140EE66E050EE66E940EE66E010E07D004
:10034000640EE66E280EE66E880EE66E010E25EC53
:10035000A5F0D5EC07F0220E0101B55D07E1FA0E1C
:10036000E66E9B0EE66E020E2AECA5F0180E010159
:10037000B55D07E1010EE66E730EE66E020E2AEC25
:10038000A5F0090E0101B55D5FE11F862A50020B41
:100390000BE001013B5108E03B51010802E2010E74
:1003A00001D0020E3B6F07D0130EE66E3B0EE66ED9
:1003B000010E2AECA5F020EC08F001013B5103E00E
:1003C00001018E8304D03B5102E101018E93030EA3
:1003D00001013B5D37E33B51130834E3000E036E2C
:1003E000026E016E030E3B5D006E080E005C0BE2B8
:1003F000010E00C0E7FFE75204E0E846FE0BE70607
:10040000FCE1016E12D0100E005C0CE2080E005CE4
:100410004B6E010E4B5204E0E846FE0B4B06FCE12E
:10042000026E03D0100E005C036E010EE66E0350E8
:10043000E66E0250E66E0150E66E94ECD9F02CECBC
:10044000A8F002D078ECDAF0020E0101B55D0BE104
:100450001E0EE66E010EE66E710EE66E010E25ECC6
:10046000A5F09EEC1DF0060E0101B55D55E1010100
:10047000E45109E1080EE66E040EE66E480EE66EE3
:10048000010E25ECA5F00101E40508E1E668C80EBF
:10049000E66E7E0EE66E010E25ECA5F0020E010161
:1004A000E45D08E1C80EE66EE66A4C0EE66E010EEB
:1004B00025ECA5F0030E0101E45D14E10701E3A3BF
:1004C00008D0960EE66E780EE66E4E0EE66E010EC3
:1004D00007D0320EE66E0A0EE66E4D0EE66E010E87
:1004E00025ECA5F0040E0101E45D09E10F0EE66EB6
:1004F0000A0EE66E420EE66E010E25ECA5F0050E24
:100500000101E45D07E11AB602D001016373076AD5
:100510008FEC1CF09EEC1DF086ECA7F052E1016A16
:100520000101D05102E0010E016E020E0901BC5D15
:100530002FE19FECA5F0EF50006E00504B6E4C6A1F
:10054000190ECAECA5F0190E4C02F3CF4CF04B0279
:10055000F3CF4BF0F4504C264B50006E0E040BE1E1
:100560000050DDECA5F004E6E20E4B5C000E4C58AA
:1005700002E2190E0026FF0E0E5C05E1005018087D
:1005800002E2190E005E9FECA5F000C0EFFF17D04D
:10059000020EBC5D14E2FA0EE66E010EE66E01502C
:1005A000030DF3CF4DF0F4CF4EF0DA0E4D26020ED0
:1005B0004E22BC51ECECA5F07DDC2CECA8F062ECFA
:1005C0004BF0310E0101B55D0DE1DA0E006E2ABE71
:1005D00002D0780E006E0050E66E860EE66E010EBA
:1005E0002AECA5F0030E0101B55D09E1020EE66EED
:1005F000320EE66E010E2AECA5F02EEC1DF0370E41
:100600000101B55D0CE178EC17F0190EE66EE66AB3
:100610007B0EE66E010E25ECA5F047EC14F0350ECE
:100620000101B55D0FE1280EE66E1E0EE66E8A0E24
:10063000E66E010E25ECA5F037EC37F0A0EC2CF0BF
:10064000B1EC16F03D0E0101B55D09E13C0EE66E20
:100650006F0EE66E010E2AECA5F063EC17F03E0E6D
:100660000101B55D09E13C0EE66E700EE66E010E0D
:100670002AECA5F063EC17F0300E0101B55D28E11E
:1006800081C306F13B0E016E03017F5104E180C37B
:1006900006F1170E016E020E7F5D02E182C306F1C4
:1006A000015034ECA8F014ECA6F003017F5102E1F4
:1006B00006C180F37F0502E106C181F3020E7F5D72
:1006C00002E106C182F30101845102E03BECEEF04D
:1006D000070E0101B55D16E103017F5107E1170E19
:1006E000E66E830EE66E030E14ECA6F003017F05A2
:1006F00007E13B0EE66E840EE66E030E14ECA6F0E8
:1007000044ECEEF00101B5050EE11C50080B02E0CF
:10071000060E01D0050EE66E810EE66E010E2AEC85
:10072000A5F0E2EC04F0280E0101B55D31E1016AAB
:10073000D5CA03F0BFECA6F012E08AECA7F00FE0F8
:10074000040E036E1CA00BD0030E036E010E016E8F
:100750000A011C5104E1280E216F21CA1CFAFE0E69
:10076000E66E0150E66E05011751050DF3CF4DF011
:10077000F4CF4EF0140E4D260A0E4E220350ECEC30
:10078000A5F026EC7FF02CECA8F0258480EC0CF092
:10079000380E0101B55D16E1FA0EE66E2350040B2A
:1007A00001E0010E4C6AA40F4B6E020E4C224BC0AE
:1007B000E6FF4CC0E6FF68EC7FF03DECA8F07CEC77
:1007C00014F01F88240E0101B55D03E0340EB55D01
:1007D0001CE18EECA7F003E1ABEC0AF016D00201AD
:1007E000780E2B6FEBEC7CF004C006F1200E9CEC35
:1007F000A7F001507EECA6F006C1EFFF318E06C1D6
:1008000004F0F5EC7CF083EC1CF01C0E0101B55DEE
:100810000FE10101D05103E0030ED05D03E1ABEC29
:100820000AF006D01AB602D002017C7971EC14F0FD
:10083000230E0101B55D09E1030EE66E440EE66E7E
:10084000010E2AECA5F0DAEC1FF01A0E0101B55DDD
:1008500010E13FC1DFFF198C01013F6B070EE66E0F
:10086000400EE66E010E2AECA5F05CECA7F0DFCF9F
:100870003FF11E0E0101B55D03E10E500101342769
:10088000140E0101B55D09E10C0EE66E070EE66E71
:100890003E0EE66E010E25ECA5F05CC3E6FFCCEC47
:1008A0000AF0E552400E0101B55D14E11AB611D00F
:1008B000D0ECA7F0040A01E0010E4B6E20ECA5F08D
:1008C0004B50010BF36EF346F346FB0EEF14F3109F
:1008D000EF6E2F86410EB55D34E11BECA8F0016E82
:1008E0001FECA8F0026E0E50022602AE0FD0630E6F
:1008F000026E010601504B6E4C6A4C3407E24B50BD
:10090000F908000E4C5402E2F90E016E0250630821
:1009100002E2026A012A01504B6E4C6A4C3406E234
:100920004B50F908000E4C5401E2016A20ECA5F08E
:10093000030E01C0EBFF20ECA5F0020E02C0EBFF9E
:100940002F86420EB55D1BE117ECA8F0016E0E502C
:10095000E824012601500A0802E20A0E016E080E80
:10096000015C02E1090E016E030E015C02E2030E5E
:10097000016E20ECA5F0010E01C0EBFF2F86440EA6
:10098000B55D5BE120ECA5F0050EEB504B6E4C6ABB
:1009900020ECA5F0040EEB500A0DF3504B2401019E
:1009A000D66FF4504C20D76F20ECA5F0EF50010B20
:1009B00004E1D66DD71F000ED7230E040CE1D890AA
:1009C000D75104E6E70ED65D030ED75911E2D62BB8
:1009D000000ED7230DD0FF0E0E5C0AE1D73504E3DD
:1009E000D6511908FC0ED75503E2D607000ED75B87
:1009F0002988800ED71505E02998D66DD71F000EDF
:100A0000D723D6C14BF0D7C14CF00A0ECAECA5F0E3
:100A100020ECA5F0040E4BC0EBFF20ECA5F0050E7A
:100A20003BC0EBFF20ECA5F02950100B02E0EF805B
:100A300001D0EF902F86A0EC2CF0430E0101B55DA4
:100A40003FE120ECA5F0060EEB50006E20ECA5F087
:100A50000490EF50020B01E004800E50002600507D
:100A600006E104700480A7EC7FF00350006EA7EC51
:100A70007FF00350D880005404E204700480010E1B
:100A8000006EC5ECA7F001E00490048020ECA5F016
:100A90000450010B02E0EF8201D0EF9220ECA5F0B0
:100AA000060E00C0EBFF100E01012C5D03015C5D22
:100AB00006E100C049F160ECA7F05CC300F02F86AE
:100AC000450E0101B55D3EE10490C5ECA7F001E0E3
:100AD000048020ECA5F0EF50016E0F0E0114006EA3
:100AE00001380F0B016E0E50012604A00CD00150EE
:100AF000800803E2090E016E0490015009080CE21F
:100B0000090E016E09D0015002E1010E016E015083
:100B1000090802E2016A04800138F00B016E0150FD
:100B2000001220ECA5F000C0EFFF20ECA5F0090EAC
:100B3000E926000EEA220450010B02E0EF8E01D0FC
:100B4000EF9E2F86E55245EFA5F05C0E0024D7EC12
:100B5000A5F00101100E146F155102E1100E156F72
:100B600012001FECA8F0D4ECA7F01BECA8F0006E6C
:100B700028ECA8F090ECE6F054EFA6F040ECA5F0DD
:100B8000FE0EDB500A0809E2FE0EDB50F00F006E8D
:100B900000509CECA6F0E5DF26D0FE0EDB50006E88
:100BA000D4DF020EF36EFE0EA1ECA6F00DE2010101
:100BB000010E156F080E166FFE0EDB040DE1030E1D
:100BC000156F050E166F08D014C113F115C114F17D
:100BD00016C115F10101166BFE0EDB50080802E18B
:100BE000090E166F168F45EFA5F033EC24F02F8019
:100BF0001200140E006E04A002D0110E006EF5EF6C
:100C000085F00E0E006E04A002D0080E006EF5EF07
:100C100085F0B8EC10F0F4C7F3FFF5C7F4FF12004D
:100C200040ECA5F0040EE1260101B151800B04E077
:100C30003050100B01E1C4D0BDECE0F00CEC92F0B0
:100C4000060E0101B55D46E10101040E016F0101CF
:100C50002A0E1A6F0101E45107E19B0EE66EE80EC1
:100C6000E66E010E5DECA5F00101E40507E1970ECB
:100C7000E66EE80EE66E010E5DECA5F0020E0101D7
:100C8000E45D07E1930EE66EE80EE66E010E5DECA4
:100C9000A5F0030E0101E45D07E18F0EE66EE80E9C
:100CA000E66E010E5DECA5F0040E0101E45D07E1C6
:100CB0008B0EE66EE80EE66E010E5DECA5F0050EFD
:100CC0000101E45D07E1870EE66EE80EE66E010EB7
:100CD0005DECA5F086ECA7F010E10101420E1D6F5E
:100CE0000901BC0503E10101440E1D6F020E09015B
:100CF000BC5D03E101014D0E1D6F320E0101B55DBA
:100D000011E10201D2510EE0BDECE0F0800EE66E82
:100D1000E80EE66E010E5DECA5F02DA203D00101F8
:100D2000370E1C6F280E0101B55D08E18AECA7F0B3
:100D300005E001014C0E1C6F2A0E1D6F82ECA7F01E
:100D40000DE101015851100B09E001012A0E1A6F43
:100D5000010158BB03D001013F0E1A6F20A805D036
:100D6000BDECE0F0006A48EC24F036EC60F00009DD
:100D700005E0310E03015C250101196F1B0E010115
:100D8000B55D05E1310E03015D2501011D6F240EE6
:100D90000101B55D03E0340EB55D05E1310E0301DF
:100DA0005E2501011D6F160E0101B55D09E101010E
:100DB000DF51400B05E00101500E176F4C0E186F0C
:100DC000ADECE0F061ECA5F001010E0E146F156FB3
:100DD00051EC7DF0000907E00101006B280EE66E82
:100DE0003BECE7F0E552016A3D0E0101B55D08E11B
:100DF0006FC100F0016802016F0EC26F010EC36F78
:100E00003E0E0101B55D08E170C100F0016802010C
:100E1000700EC26F010EC36F1E0E0101B55D08E1B9
:100E20000201340EC26F010EC36F34C100F00168BD
:100E3000140E0101B55D0CE1050E01013E03F350F6
:100E4000410F006E016802013E0EC26F010EC36FBA
:100E50001A0E0101B55D09E101014029006E01682A
:100E60000201400EC26F010EC36F160E0101B55D87
:100E70001AE101018851FE0BE842006E0201880E62
:100E8000C26F010EC36F0101DFAD0BD094C100F042
:100E90000201940EC26F010EC36F030E0002F3CF66
:100EA00000F001682F88060E0101B55D69E10101BE
:100EB000E45106E10201480EC26F010E3DECA5F0BF
:100EC0000101E40506E102017E0EC26F010E3DEC58
:100ED000A5F0020E0101E45D06E102014C0EC26FB5
:100EE000010E3DECA5F0030E0101E45D1EE10101E0
:100EF000006B0701E3A30CD07C0EE66EE80EE66EF5
:100F0000010E1CECA5F002014E0EC26F010E0BD0BB
:100F1000780EE66EE80EE66E010E1CECA5F00201FE
:100F20004D0EC26F010E3DECA5F0040E0101E45D13
:100F300006E10201420EC26F010E3DECA5F0016810
:100F4000050E0101E45D19E1016A010163A306D008
:100F5000740EE66EE80EE66E010E05D0700EE66EBB
:100F6000E80EE66E010E1CECA5F00201630EC26FE6
:100F7000010EC36F0201020EC46F0101050E006F66
:100F800086ECA7F01DE1026A0101D05102E0010EDA
:100F9000026E0250030D65ECA7F0DA0E4B26020E2E
:100FA0004C220901BC51D7ECA7F0020E0901BC5D2F
:100FB00005E1190E84ECA5F040C000F001682F880F
:100FC000390E0101B55D0AE1D0C1E6FF1FEC0CF05E
:100FD000E552016818ECA6F00C0EC46F015002E057
:100FE00090ECE6F0140E0101B55D07E0160EB55D5C
:100FF00006E10101DF51400B02E00101158F390EBE
:101000000101B55D07E0160EB55D0AE10101DF5192
:10101000400B06E10101145102E1100E146F168F0E
:101020000B0E0101B55D1DE1150E0101565D0CE1D0
:101030000101006B670EE66EE80EE66E010EE66ECD
:1010400035ECE7F0E55206D056C100F090ECE6F042
:1010500003ECA7F0E552E5520201560EC26F010EF5
:10106000C36F3B0E0101B55D12E10101CDAB02D0B2
:10107000080E01D00E0EC2ECA5F02F800201CD0E9D
:10108000C26F010EC36F0201200EC46F2F88040EC1
:101090000101B55D0DE10701E3B102D00E0E01D0F3
:1010A000080EC2ECA5F018ECA6F0010EC46F2F805C
:1010B000050E0101B55D17E10701E3B306D0780E17
:1010C000E66EE80EE66E010E07D001010007620E23
:1010D000E66EE80EE66E010E1CECA5F018ECA6F02C
:1010E000020EC46F2F800F0E0101B55D1FE12CC1F0
:1010F000E6FF44DDE55213C10FF114C110F115C133
:1011000011F116C112F10101100E136F61ECA5F07F
:101110000101CEAB02D0290E01D02A0EE66E3BECC7
:10112000E7F0E5521FECA6F0200EC46F290E010176
:10113000B55D1AE16DECA5F061ECA5F00B0EC2EC0B
:10114000A5F00101CEA10BD061ECA5F05E0EE66E1C
:10115000E80EE66E010E1CECA5F00101168F1FECE7
:10116000A6F0010EC46F2F88200E0101B55D22E1AB
:101170006DECA5F028ECA8F0580EE66EE80EE66ED1
:10118000010E1CECA5F00101CC51010B06E0CC5185
:10119000020B03E00101030E04D0CCA303D0010134
:1011A000020E136F0201CC0EC26F010EC36F02015B
:1011B000030EC46FE3ECA6F02AE12350040B01E018
:1011C000010E010F01010F6F28ECA8F004902350CD
:1011D000040B01E0010E8BECA5F0EECF0FF0EDCF8C
:1011E00010F0BAEC24F00101100E126F2CB4166F3F
:1011F0002350040B01E0010E020DF3CFF3F6F4CF00
:10120000F4F6A00E0601F327020EF4232F88320E07
:101210000101B55D01E01FD125B80DD00101006BC2
:10122000FAEC60F0D4ECA7F061ECA5F003EC61F00F
:10123000D4ECA7F00FD109ECA8F035EC0FF00F506B
:101240000101D4271050D523D4C10FF0D5C110F01F
:10125000010E0F0B05E0D89010320F32E806FBE1CB
:1012600007010F500C5D10500D5905E20C510F5E37
:101270000D51105A02D00F6A106A0FC00EF710C03D
:101280000FF70201D2511DE0190E4B6E4BC045F015
:10129000D2C240F05CECFAF03C5004E193EC04F074
:1012A0000201D36FD3C200F00101136B0A0E84EC6C
:1012B000A5F040C014F13CC015F10101110E166FEC
:1012C000148FFAEC60F0026E006E2DA204D003ECD5
:1012D00061F0026E006E0201D2515CE0960E0101D7
:1012E000D46FD56B20A003D0F00ED46FD56BEFEC8C
:1012F00060F0000904E0320E0101D46FD56B0101EA
:10130000D4510F5CD551105811E20050DDECA5F01E
:1013100004E6F00E4B5C000E4C5808E2002A640E06
:101320000201D25D20E2190ED2271DD00C0E4C6AAC
:10133000D4254B6ED5514C220F504B5C10504C585D
:1013400005E20050640802E200060DD00201D2510D
:101350004B6E4C6A4C3407E24B50C808000E4C549C
:1013600002E2C80ED26F0250005C73E02DB208D0CA
:10137000E66A0050E66E0CEC61F0E552E66E07D0CE
:101380000050E66E1CEC61F0E552E66EE66AE2ECB7
:10139000A5F05FD02DB244D0FAEC60F04B6E640E35
:1013A0004B5C09E3FAEC60F04C6E4D6A4D340DE293
:1013B000A6ECA6F00AE2FAEC60F00701266F4E0EEA
:1013C000ABECA6F01AEC93F044D0E66AE66AE2ECE5
:1013D000A5F00201FA0ED26F49ECA5F005E0D89015
:1013E0000D330C33E806FBE103EC61F04B6E640E49
:1013F0004B5C09E303EC61F04C6E4D6A4D3408E23E
:10140000A6ECA6F005E2A00EE66E1CEC61F0E5523B
:1014100003EC61F0E66EE66AE2ECA5F02D8219D0ED
:101420001AEC93F003EC61F04B6E640E4B5C09E335
:1014300003EC61F04C6E4D6A4D340AE2A6ECA6F066
:1014400007E203EC61F00701266F510EABECA6F04A
:101450002D9226822F88350E0101B55D11E109EC30
:10146000A7F08BB102D00E0E006E33EC24F08AC1CF
:1014700000F0DEECA7F0168F10ECA7F0010EC46FA1
:10148000100E0101B55D2FE10101166B16C115F1BA
:10149000100E146F0D0E0101515D04E10101010EEA
:1014A000156F1ED0080E515D03E10101050E0BD032
:1014B000050E515D03E10101030E05D0030E515DE0
:1014C00004E10101020E166F0BD0510509E1010183
:1014D000010E166F0101006F0B0E006E33EC24F04D
:1014E0000101168F2F88370E0101B55D10E109EC5F
:1014F000A7F08BB302D00E0E006E33EC24F07BC14C
:1015000000F0DEECA7F010ECA7F0020EC46F020EA4
:101510000101B55D13E171C100F090ECE6F01E0E23
:101520000101715D06E143ECA6F00B0E006E33EC99
:1015300024F00201710EC26F010EC36F310E010162
:10154000B55D1AE10101865104E10B0EC2ECA5F074
:101550000ED086C100F08651780805E26C0E005E60
:1015600090ECE6F004D090ECE6F00101168F020159
:10157000860EC26F010EC36F030E0101B55D22E13D
:101580000201320EC26F010EC36FC3ECA6F00E0E45
:10159000C2ECA5F00101320507E10101020E006F66
:1015A000AF0E006E33EC24F0020E0101325D0AE151
:1015B0000101020E006F520EE66EE80EE66E010E9D
:1015C0001CECA5F0220E0101B55D0FE1CBECA6F0FD
:1015D000BBECA5F00101100E126F0101006B338C02
:1015E00002019B0EC26F020EC36F240E0101B55D96
:1015F00003E0340EB55D3CE1B8EC7CF0026A080E05
:10160000025C36E201500224E66EDAEC7CF0E55230
:10161000006E100E005C03E08EECA7F002E1020EFB
:1016200013D00050120802E2040E0ED00050100831
:1016300002E2030E09D00E0E005C02E2006A05D041
:10164000100E005C02E2010E006E410E0024E66EF8
:1016500019EC04F0E552D00FE66E0250EA6A0F0F63
:10166000E96E010EEA22E552E750EF6E022AC7D773
:10167000110E0101B55D11E10101100E156F15C1CB
:1016800014F1110E166F01012BAF02D00101162BC0
:1016900026ECA6F0800EC46F2F803F0E0101B55DD1
:1016A0000EE161ECA5F053C100F090ECE6F0010111
:1016B000158F0201530EC26F010EC36F2F88360EB5
:1016C0000101B55D18E10101006B4D0EE66EE80EFB
:1016D000E66E010E1CECA5F034B803D001010E0E2D
:1016E0000F6F61ECA5F031EC12F0B0ECA6F002E166
:1016F000100E146F2F882B0E0101B55D09E10FEC60
:1017000008F09C0E0F5C630E105802E2BBECA5F0D3
:1017100082ECA7F001E05CD10101006B0101E3ABB9
:101720002AD10A0E4B6E4C6ACEC73FF0CFC740F0AD
:101730004BC044F04CC045F002ECFAF03F50D4EC02
:10174000A7F00101240E0F6F9D0E6AECA7F0CCEC00
:1017500007F00FC0DEFF10C0DDFFC80E0F5C000EEB
:10176000105806E3840ED8800F54030E105406E27E
:101770000701080E266F240EABECA6F0BBECA5F01B
:101780000101100E126F160E136F09EC86F0F3CFE5
:1017900059F0F4CF5AF059C0E6FF5AC0E6FFC7EC43
:1017A000A6F0E7CF5AF0E552E7CF59F05950F324AD
:1017B000576E5A50F420586E57C0E6FF58C0E6FFE7
:1017C000C7ECA6F0E7CF58F0E552E7CF57F05750F7
:1017D000F324556E5850F420566E55C0E6FF56C09F
:1017E000E6FFC7ECA6F0E7CF56F0E552E7CF55F09D
:1017F0005550F324536E5650F420546E53C0E6FFF8
:1018000054C0E6FFC7ECA6F0E7CF54F0E552E7CFAF
:1018100053F05350F324516E5450F420526E51C083
:10182000E6FF52C0E6FFC7ECA6F0E7CF52F0E55264
:10183000E7CF51F05150F3244F6E5250F420506EC8
:101840004FC0E6FF50C0E6FFC7ECA6F0E7CF50F070
:10185000E552E7CF4FF04F50F3244D6E5050F42037
:101860004E6E4DC0E6FF4EC0E6FFC7ECA6F0E7CFD8
:101870004EF0E552E7CF4DF04D50F3244B6E4E50F5
:10188000F4204C6E030E0F0B05E0D8904C324B3217
:10189000E806FBE1020E4BC0DBFF030E4CC0DBFF92
:1018A0000101E3AD66D0450EE66EE80EE66E010E70
:1018B00039ECA5F0020EDBCFD4F1030EDBCFD5F16E
:1018C00001017F0ED880D455050ED55507E20701DA
:1018D000090E266F240EABECA6F04BD0D4C14BF012
:1018E000D5C14CF0070ED8904C324B32E804FBE1E6
:1018F0006A0E4B240A6ED4C14BF000014C6A4B9E19
:101900004B50E824016EBCEC38F0FF0E005C30E177
:10191000010EDB50006E77EC38F0012ADF50006ECC
:1019200077EC38F001012A0E1D6F400EE66EE80ECE
:10193000E66E010E80ECA5F0020EDBCFE6FF030E93
:10194000DBCFE6FF6FECA7F03C0EE66EE80EE66E2E
:10195000010E80ECA5F0DECFE6FFDDCFE6FF6FECF9
:10196000A7F0350EE66EE80EE66E010E80ECA5F0EF
:101970000A6A26822CD06AC11EF16BC11FF16CC1AC
:1019800020F16DC121F10A0E426E436A446A456A34
:101990001EC13DF01FC13EF020C13FF021C140F00B
:1019A00031ECF9F03DC01EF13EC01FF13FC020F107
:1019B00040C021F1CDECE6F0F7ECE6F00101128F2A
:1019C000158F0701E3BB03D00101100E166F2F889E
:1019D0000490170E0101B55D07E1010139BF0480D4
:1019E0005DECA6F0800EC46F0E0E0101B55D0AE13C
:1019F00001013F5101E00480F3ECA7F03F0EC26FFC
:101A0000010EC36F080E0101B55D0CE1010197BD28
:101A10000480F3ECA7F0970EC26F010EC36F0201B2
:101A2000400EC46F2E0E0101B55D27E1010137ADF7
:101A300018D0ADECE0F02E0EE66EE80EE66E010E6C
:101A40001CECA5F001013751070B050DF3500A0FEF
:101A5000006E0A0E84ECA5F040C015F13CC016F1F2
:101A600004D037BF048001EC86F00201370EC26F4C
:101A7000010EC36F0201C70EC46F250E0101B55DD3
:101A800007E1010139B504805DECA6F0040EC46FD6
:101A90003C0E0101B55D0CE1010138B10480F3ECAD
:101AA000A7F0380EC26F010EC36F0201010EC46FA2
:101AB0000A0E0101B55D24E10101855106E161ECE9
:101AC000A5F00B0EC2ECA5F015D0ADECE0F00101D5
:101AD000850506E1250EE66EE80EE66E010E08D0DD
:101AE000020E855D07E11C0EE66EE80EE66E010E45
:101AF0001CECA5F00201850EC26F010EC36F2F888A
:101B0000150E0101B55D16E161ECA5F00E0E006E3B
:101B100001013CA905D05C0E006E0101040E006FAE
:101B200002013C0EC26F010EC36F0201100EC46FA2
:101B3000F5EC85F01D0E0101B55D26E1010157A50B
:101B40000CD00101006B130EE66EE80EE66E010E7E
:101B50001CECA5F00101158F0ED057A108D00F0E77
:101B6000E66EE80EE66E010E1CECA5F004D00E0E3B
:101B7000006E33EC24F00201570EC26F010EC36FEA
:101B80000201050EC46F2F800101B55106E134B684
:101B9000048001EC86F02F88338C0101B50551E1FA
:101BA0000101006B060EE66EE80EE66E010E1CECFF
:101BB000A5F00101006B0101810507E1FD0EE66E54
:101BC000E70EE66E010E1CECA5F0020E0101815D30
:101BD00007E1F40EE66EE70EE66E010E1CECA5F0D2
:101BE000030E0101815D07E1EB0EE66EE70EE66E86
:101BF000010E1CECA5F0040E0101815D07E1E20E6F
:101C0000E66EE70EE66E010E1CECA5F0050E010176
:101C1000815D07E1D90EE66EE70EE66E010E1CEC63
:101C2000A5F0060E0101815D07E1D00EE66EE70E1C
:101C3000E66E010E1CECA5F00201810EC26F010ED2
:101C4000C36F0C0E0101B55D3FE10101845106E156
:101C500043ECA6F0440EC2ECA5F031D084050DE1B2
:101C600043ECA6F0C80EE66EE70EE66E010EE66ED9
:101C700035ECE7F0E552E55206D034AE06D0010E61
:101C8000E66E6EECEFF0E5521AD028ECA8F0C20E2A
:101C9000E66EE70EE66E010E1CECA5F00101840570
:101CA000040DF350006E0A0E84ECA5F040C012F152
:101CB0003CC013F10101125102E1100E126F02013A
:101CC000840EC26F010EC36F2A0E0101B55D12E1D1
:101CD0000B0E006E049001012BB3048004B004D0FD
:101CE00043ECA6F0440E006EF5EC85F026ECA6F071
:101CF000020EC46F2C0E0101B55D0EE10B0E006EDD
:101D0000010160AF02D0E00E006EF5EC85F017EC3B
:101D1000A7F0800EC46F2F882F0E0101B55D09E179
:101D200001012BB5048001EC86F026ECA6F0040E30
:101D3000C46FC3ECA6F01C0E0101B55D0EE161ECB1
:101D4000A5F002017CB90480F3ECA7F07C0EC26F11
:101D5000020EC36F0201100EC46F1F0E0101B55DAC
:101D600019E10101CEAF08D061ECA5F0700EE66E6E
:101D7000E80EE66E010E07D00101006BB90EE66EAB
:101D8000E70EE66E010E1CECA5F01FECA6F0800E2F
:101D9000C46F2F80180E0101B55D36E1ADECE0F0A7
:101DA000110E1EECA7F001010F6F130E1EECA7F031
:101DB0000101106F0F6A106A020173510DE1300EBC
:101DC000F66E850EF76E010EF86E0900F5CF0FF076
:101DD0000A00F5CF10F008D0730506E1076AA8ECF9
:101DE0001EF00101200E116F0E0ED8800F54270E29
:101DF000105402E20F6A106ABBECA5F00101125107
:101E000002E1100E126F158F090E0101B55D42E15E
:101E10003BECD9F043ECA6F001013B5102E1440E4A
:101E20000CD03B0504E1C3ECA6F02A0E06D0020E4E
:101E30003B5D06E1C3ECA6F05C0EC2ECA5F023D03E
:101E4000030E3B5D20E33B5113081DE3660EC2EC1D
:101E5000A5F0030E01013B5D006E080E005C05E27B
